:100000000C9444290C94654A0C943A4A0C940F4A77
:100010000C94E4490C94B9490C948E490C946349AE
:100020000C9438490C9475290C9475290C947529F5
:100030000C9475290C94E74A0C9475290C94752935
:100040000C9475290C9401E00C9475290C94752975
:100050000C9475290C9475290C94FB740C94CF4C5A
:100060000C9475290C94AB620C9445630C9475291F
:100070000C9475290C9475290C9475290C94752988
:100080000C9475290C9475290C9475290C94752978
:100090000C9475290C9475290C9475290C94752968
:1000A0000C9475290C9475290C9475290C94752958
:1000B0000C9475290C9475290C9475290C94752948
:1000C0000C9475290C9475290C9475290C94752938
:1000D0000C9475290C9475290C9475290C94752928
:1000E0000C947529D444D744C644CA44D0440E4520
:1000F000DB44DF44E544E944ED44F344F744FB4486
:100100000E45014505450945AC4BB14BB64BC04BBF
:10011000CA4B434CD44BDC4BE44BEE4BF84B024CFC
:10012000114C1B4C434C254C2F4C394CDE62E46285
:10013000F562006308631D630C631D631063146341
:100140001D631A63E800E800D400D400D400DA008C
:10015000DA00DA00EA00F400F400F400084AD73BC1
:100160003BCE016E84BCBFFDC12F3D6C74319ABD86
:1001700056833DDA3D00C77F11BED9E4BB4C3E91AA
:100180006BAAAABE000000803F05A84CCDB2D44E99
:10019000B93836A9020C50B9918688083CA6AAAA9B
:1001A0002ABE000000803F000D946F250D94E500ED
:1001B0000D94D8000D9476250D94E0000D945D0209
:1001C0000D94D4000D940C130D94E3000D94E813DA
:1001D0000D9468250D9483250D94701D0D94DC00FD
:1001E0000D9485190D9432040D947D254E414E4990
:1001F0004E495459494E46CDCCCC3D0AD7233C17E5
:10020000B7D13877CC2B329595E6241FB14F0A0031
:100210000020410000C84200401C4620BCBE4CCA21
:100220001B0E5AAEC59D74434F4D4D554E4943412B
:1002300054494F4E0044525952554E004552524F68
:10024000525300494E464F004543484F0020746FBB
:100250006F206C6F6E6720657874727573696F6E4E
:100260002070726576656E7465640A0020636F6C39
:100270006420657874727573696F6E20707265762C
:10028000656E7465640A0047322F473320626164EB
:1002900020706172616D65746572730A00536C65DC
:1002A00065702E2E2E00205A3A200020593A200048
:1002B00042656420583A2000526573756D696E6717
:1002C000207072696E74004D696E6920322072650B
:1002D0006164792E00436C69636B20746F207265D2
:1002E00073756D652E2E2E004E6F206D6F76652E08
:1002F00000456E642066696C65206C6973740A0041
:10030000426567696E2066696C65206C6973740A62
:10031000004D313235005344207072696E74696E3D
:1003200067206279746520004E6F742053442070FA
:1003300072696E74696E670A0046696C652064654F
:100340006C657465643A0044656C6574696F6E2011
:100350006661696C65642C2046696C653A20006FA3
:1003600070656E206661696C65642C2046696C65F9
:100370003A20005072696E742074696D653A2000ED
:10038000000125311D40FF24301CFF45232F1B0A8F
:1003900007FFFF040806FF06222B1AFFFF0438039D
:1003A000FF36FFFFFFFFFFFF50726F7465637465D8
:1003B000642050696E0A006D0046696C616D656E5F
:1003C0007420757365643A200053746174733A2025
:1003D000002C204C6F6E67657374206A6F623A2040
:1003E00000546F74616C2074696D653A2000537419
:1003F0006174733A20002C204661696C65643A2070
:10040000002C2046696E69736865643A200050725A
:10041000696E74733A200053746174733A20004516
:100420007874727564657220257300480243023C3B
:1004300002350227026F66660044454255473A007E
:100440006F6B00436F6F6C696E6720646F6E652E13
:100450000048656174696E6720646F6E652E0020C8
:10046000573A0045787472756465722025730020D0
:10047000643A0020693A0020703A00426564204CDA
:100480006576656C696E6720004661696C656420FD
:10049000746F20656E61626C6520426564204C65F6
:1004A00076656C696E670A00426564204C65766506
:1004B0006C20436F7272656374696F6E204D617456
:1004C0007269783A0020202020202846312E3020E2
:1004D0003D2066756C6C20636F7272656374696F22
:1004E0006E2C2046302E30203D206E6F20636F72C0
:1004F00072656374696F6E290A0020204661646525
:100500003A202020202020202020202020202020D1
:10051000202046002020536D6F6F7468696E67203D
:10052000286D6D293A2020202020202053002020F3
:1005300044697374616E636520286D6D293A2020CB
:100540002020202020205A004261636B6C61736878
:1005500020636F7272656374696F6E2069732061C6
:1005600063746976653A0A004261636B6C61736813
:1005700020636F7272656374696F6E20697320699E
:100580006E6163746976653A0A004261636B6C61FF
:100590007368206D6561737572656D656E74202872
:1005A0006D6D293A2020003A2000207A5F6D696E37
:1005B0003A20202D32207A5F6D61783A2020350A6A
:1005C0000050726F6265205A204F66667365740032
:1005D0004175746F0020452F443D00416476616E83
:1005E0006365204B3D0041637469766520457874EE
:1005F00072756465723A2000556E6B6E6F776E206F
:10060000636F6D6D616E643A20220000002000234C
:1006100000260029002C002F0032000001000003FA
:100620000106010901022569730025696D2025690C
:1006300073002569682025696D2025697300256987
:1006400064202569682025696D2025697300256966
:100650007920256964202569682025696D20256930
:1006600073007A5F6D61783A20007A5F6D696E3A47
:100670002000795F6D61783A2000785F6D696E3A8D
:1006800020005265706F7274696E6720656E6473C6
:10069000746F70207374617475730A00205A00209F
:1006A0005900580020204D61783A2000205A00203F
:1006B0005900580020204D696E3A20004F6E2000EE
:1006C0004F666600536F667420656E6473746F7056
:1006D000733A200050726F6265205A204F6666732D
:1006E00065743A200020643A0020693A0020703A8C
:1006F0000043290A0061626C656420286D696E20E0
:1007000074656D702000436F6C6420657874727539
:100710006465732061726520004B6420002364656A
:1007200066696E65202044454641554C545F004B38
:1007300069200023646566696E6520204445464152
:10074000554C545F004B70200023646566696E65EC
:10075000202044454641554C545F005049442041B7
:1007600075746F74756E652066696E69736865640B
:10077000212050757420746865206C617374204B5F
:10078000702C204B6920616E64204B6420636F6E77
:100790007374616E74732066726F6D2062656C6F26
:1007A0007720696E746F20436F6E6669677572613A
:1007B00074696F6E2E680A00504944204175746F49
:1007C00074756E65206661696C6564212074696D5D
:1007D000656F75740A00544845524D414C2052557E
:1007E0004E4157415900546865726D616C205275D5
:1007F0006E617761790048656174696E6720666132
:10080000696C65640048656174696E67206661693A
:100810006C656400504944204175746F74756E6551
:10082000206661696C6564212054656D7065726134
:100830007475726520746F6F20686967680A00209C
:100840004B643A2000204B693A2000204B703A203C
:10085000000A20436C617373696320504944200A85
:10086000002054753A2000204B753A2000206D611D
:10087000783A2000206D696E3A200020643A20000A
:1008800020626961733A20004F6666736574732055
:100890006170706C696564004572723A20546F6FC4
:1008A000206661722100546F6F206661722066724B
:1008B0006F6D207265666572656E636520706F6925
:1008C0006E740A004E6F2063617365206C696768FF
:1008D000740A001FFFFFFFFFFFFF60000000000120
:1008E000FF400000000000FF8000000000007F8348
:1008F000CF00000C303F87FF80000C301F867980CE
:10090000000C000F8C30C7838C30E78C30CFC7CC05
:1009100031F38C30DCECEC33B98C30D86C6C33199F
:100920008C30D06C0C33198C30D86C0C33198C3063
:10093000DC6C0E3B198C30CF7C079F198C30C77C48
:10094000038F19400000000000026000000000005A
:10095000061FFFFFFFFFFFF82020506C616E6E65E1
:100960007242756666657242797465733A2000203A
:1009700046726565204D656D6F72793A2000436F50
:100980006D70696C65643A204D6179203233203294
:100990003031380A00207C20417574686F723A202B
:1009A00028416C657068204F626A656374732049E2
:1009B0006E632E2C204C756C7A426F7420476974DC
:1009C000205265706F7369746F7279290A004D61E6
:1009D00079203233203230313831303A30313A33C5
:1009E0003000204C61737420557064617465643A02
:1009F0002000312E312E380A004D61726C696E0074
:100A000020536F6674776172652052657365740A4E
:100A100000205761746368646F6720526573657462
:100A20000A002042726F776E206F757420526573D2
:100A300065740A002045787465726E616C20526599
:100A40007365740A00506F77657255700A0073748D
:100A50006172740A006572726F72207772697469CC
:100A60006E6720746F2066696C650A00456E64735A
:100A7000746F707320256320256320256320256310
:100A800000205A3A0020593A0020583A00656E6416
:100A900073746F7073206869743A2000446F6E65D8
:100AA00020736176696E672066696C652E0A004D59
:100AB0003239004B494C4C45442E2000426564209D
:100AC000646F6E652E0020573A00426564206865A9
:100AD0006174696E672E0042656420636F6F6C6994
:100AE0006E672E004D31343520533C696E64657855
:100AF0003E206F7574206F662072616E67652028D6
:100B0000302D31290A004C756C7A426F7420486987
:100B1000626973637573204F66662E00205A3A002F
:100B200020593A0020436F756E7420583A002045D2
:100B30003A00205A3A0020593A00583A003A004305
:100B400061703A00454D455247454E43595F50410B
:100B50005253455200434153455F4C494748545F07
:100B60004252494748544E45535300544F47474C0F
:100B7000455F4C494748545300534F4654574152E0
:100B8000455F504F574552004255494C445F5045D0
:100B90005243454E54004C4556454C494E475F44E0
:100BA000415441005A5F50524F4245004155544F05
:100BB0004C4556454C005052494E545F4A4F4200F6
:100BC00050524F4752455353004155544F52455090
:100BD0004F52545F54454D5000564F4C554D45545F
:100BE00052494300454550524F4D005345524941EB
:100BF0004C5F584F4E5F584F4646004649524D573E
:100C00004152455F4E414D453A4D61726C696E20CF
:100C1000204649524D574152455F56455253494F20
:100C20004E3A312E312E382E3539204558545255F2
:100C30004445525F545950453A4165726F7374721E
:100C40007564657220534F555243455F434F444589
:100C50005F55524C3A68747470733A2F2F636F6407
:100C6000652E616C6570686F626A656374732E636C
:100C70006F6D2F646966667573696F6E2F4D415293
:100C80004C494E2050524F544F434F4C5F564552A3
:100C900053494F4E3A312E30204D414348494E453D
:100CA0005F545950453A4C756C7A426F74204869CC
:100CB0006269736375732045585452554445525FB9
:100CC000434F554E543A3120555549443A653535D0
:100CD00030323431312D643436642D343231642D68
:100CE000626133612D6132303132366437393330ED
:100CF000660A002F2F200053657474696E672054B4
:100D0000726176656C20416363656C6572617469BC
:100D10006F6E3A200053657474696E672052657473
:100D20007261637420416363656C65726174696F9D
:100D30006E3A200053657474696E67205072696E54
:100D40007420416363656C65726174696F6E3A20EB
:100D50000053657474696E67205072696E74206107
:100D60006E642054726176656C20416363656C65C6
:100D7000726174696F6E3A20001000C90210012C74
:100D8000014001220170011801B0010E01F00104BF
:100D9000015002FA00B002F0003003E600D003DC9C
:100DA000009004D2007005C800A006BE000008B480
:100DB00000B009AA00D00BA000600E960060118C54
:100DC000000015820020197800C01D6E00A022646A
:100DD00000B0275A00902C500000314600E0343C0F
:100DE0000010383200903A2800603C1E00A03D14EC
:100DF00000803E0A00203F00004572723A204D49B3
:100E00004E54454D5020424544004D494E54454DA9
:100E10005020747269676765726564004572723A42
:100E2000204D494E54454D50204531004572723A8F
:100E3000204D494E54454D50204530004572723A80
:100E4000204D415854454D5020424544004D415895
:100E500054454D502074726967676572656400453A
:100E600072723A204D415854454D5020453100454D
:100E700072723A204D415854454D50204530002063
:100E80002F002042403A0020403A007C3C3E5E2B3E
:100E90003D3F2F5B5D3B2C2A225C0020706F736905
:100EA00074696F6E206F7574206F662072616E6753
:100EB000652E0A003F50726F626520000A0A426583
:100EC00064204C6576656C20436F7272656374694B
:100ED0006F6E204D61747269783A00202B000A43CE
:100EE0006F72726563746564204265642048656949
:100EF0006768742076732E2042656420546F706F8B
:100F00006C6F67793A0A00202B000A42656420481A
:100F1000656967687420546F706F67726170687973
:100F20003A0A2020202B2D2D2D204241434B202DED
:100F30002D2B0A2020207C20202020202020202053
:100F400020207C0A204C207C20202020282B2920B7
:100F50002020207C20520A2045207C202020202098
:100F60002020202020207C20490A2046207C202888
:100F70002D29204E20282B29207C20470A20542070
:100F80007C20202020202020202020207C20480A97
:100F90002020207C20202020282D29202020207C7B
:100FA00020540A2020207C202020202020202020C7
:100FB00020207C0A2020204F2D2D2046524F4E54B9
:100FC000202D2D2B0A2028302C30290A004D656158
:100FD0006E206F662073616D706C656420706F6940
:100FE0006E74733A200020643A200020623A200098
:100FF00045716E20636F656666696369656E7473BB
:101000003A20613A20003474682070726F62652063
:10101000706F696E742C2064697374616E636520EF
:1010200066726F6D20706C616E653A2000202844F6
:10103000525952554E2900473239204175746F205C
:10104000426564204C6576656C696E6700284229AC
:1010500061636B00284629726F6E740028522969FB
:1010600067687400284C29656674003F4E756D6290
:101070006572206F662070726F626520706F696E96
:10108000747320697320696D706C61757369626C2B
:1010900065202832206D696E696D756D292E0A00F4
:1010A0003F2856296572626F7365206C6576656CA2
:1010B00020697320696D706C61757369626C65205D
:1010C00028302D34292E0A004D3630302042300091
:1010D0005072696E7420706175736564004D3132B1
:1010E0003500004D3234005072696E742061626FB9
:1010F00072746564004E6F20534420636172640013
:101100005072696E742066726F6D20534400537480
:101110006F70207072696E7400526573756D652012
:101120007072696E740041626F7574204669726DE9
:1011300077617265005061757365207072696E74B5
:10114000004368616E67652066696C616D656E74E9
:1011500000436F6E66696775726174696F6E0054E3
:10116000656D7065726174757265004D6F76656D41
:10117000656E740054756E6500496E666F2073630A
:101180007265656E004D6F76652061786973004405
:10119000697361626C652073746570706572730049
:1011A0004D3834004C6576656C2058204178697361
:1011B000004D313137204C6576656C696E6720587B
:1011C00020417869730A4732380A4730205831364F
:1011D000302046393939390A4730205A35204636C9
:1011E0003030300A4739310A4D3231312053300A1C
:1011F0004D3430300A4D393036205A3630300A47B7
:1012000030205A2D313520463530300A4730205AAB
:101210003520463530300A4739300A4D3430300AEF
:101220004D393036205A3936300A4D32313120535B
:10123000310A4D3430300A4732380A4D31313720C7
:101240004C6576656C696E6720646F6E652E004133
:1012500075746F20686F6D6500473238004D6169A5
:101260006E004D3530320A4D353030004C6F6164C0
:101270002073657474696E677300526573746F725E
:1012800065206661696C736166650053746F726591
:101290002073657474696E677300416476616E6370
:1012A00065642053657474696E6773004D61696E7F
:1012B000004572726F722077726974696E6720746C
:1012C0006F20454550524F4D210A00290A002062E7
:1012D000797465733B20637263200053657474698D
:1012E0006E67732053746F7265642028004F6666C2
:1012F000004F6E2000456E6473746F702061626FE2
:1013000072740053746570732F6D6D004A65726B53
:1013100000416363656C65726174696F6E00566548
:101320006C6F63697479005A204F66667365740048
:10133000416476616E6365642053657474696E6799
:10134000730043616E6E6F7420656E7465722073F6
:1013500075626469723A2000022E2E004D61696E3A
:101360000020204E6F7A7A6C653A2000200042619E
:10137000636B004D696E696D756D2054656D7020ED
:101380006973203132302E0048656174696E6720C0
:101390006661696C65640045787472756465206D7A
:1013A0006F726500526573756D65207072696E7439
:1013B00000524553554D45204F5054494F4E533AD6
:1013C0000020204E6F7A7A6C653A20006368616E67
:1013D0006765006F66207468652066696C616D657D
:1013E0006E74005761697420666F72207374617245
:1013F00074005052494E54205041555345440020EA
:10140000204E6F7A7A6C653A2000200066696C6124
:101410006D656E7420756E6C6F61640057616974E0
:1014200020666F72005052494E542050415553452A
:10143000440020204E6F7A7A6C653A2000200050DC
:101440006C6561736520776169742E2E2E00486586
:101450006174696E67206E6F7A7A6C6500505249CC
:101460004E54205041555345440020204E6F7A7A07
:101470006C653A2000200068656174206E6F7A7A8E
:101480006C652E00507265737320627574746F6E94
:1014900020746F005052494E5420504155534544DA
:1014A0000020204E6F7A7A6C653A2000746F2063BA
:1014B0006F6E74696E75652E2E2E00616E642070DD
:1014C0007265737320627574746F6E00496E736514
:1014D00072742066696C616D656E74005052494E7D
:1014E00054205041555345440020204E6F7A7A6C69
:1014F000653A2000200066696C616D656E74206C31
:101500006F6164005761697420666F7200505249C0
:101510004E54205041555345440020204E6F7A7A56
:101520006C653A2000200066696C616D656E742000
:1015300065787472756465005761697420666F72AE
:10154000005052494E5420504155534544003048B4
:10155000483025753A2530327500253032753A25E8
:10156000303275001A0025336400253464002520CC
:101570002000252000746F20726573756D6500571B
:1015800061697420666F72207072696E74005052C7
:10159000494E5420504155534544000000007E0000
:1015A0006000600060F87ECC60CC60CC60F860CCFD
:1015B00000CC00CC00CC00000000000000000000C7
:1015C000000000000000000000000000000000001B
:1015D00000FE7FFE7F06600000000000000000F0BB
:1015E0000FF81FF81FF81FF00FF00FF81FF81FF883
:1015F0001FE007C0038001000000000000FE7F0E16
:10160000702664724E7A5E324C8241324C7A5E723F
:101610004E26640E70FE7F000000000000FE7F0E6C
:1016200070C663C24382411A58BA5D1A588241C2D9
:1016300043C6630E70FE7F0000000000008808882B
:10164000081011202220221011880888081011008B
:101650000000000000000000000000000020221038
:1016600011880888081011202220221011880800F3
:1016700000000000000000000000004361726420D0
:1016800072656D6F766564004361726420696E7384
:1016900065727465640020202020004C696E65200E
:1016A0004E756D626572206973206E6F74204C6197
:1016B0007374204C696E65204E756D6265722B31B6
:1016C0002C204C617374204C696E653A2000535491
:1016D0004F505045442E20005072696E7465722040
:1016E00073746F707065642064756520746F206515
:1016F00072726F72732E2046697820746865206557
:1017000072726F7220616E6420757365204D393975
:101710003920746F20726573746172742E2028549E
:10172000656D70657261747572652069732072658C
:101730007365742E20536574206974206166746526
:10174000722072657374617274696E67290A004E43
:101750006F20436865636B73756D207769746820CB
:101760006C696E65206E756D6265722C204C6173BC
:1017700074204C696E653A2000636865636B73750D
:101780006D206D69736D617463682C204C61737496
:10179000204C696E653A20004D313130004D3331B7
:1017A0000053442072656164206572726F720A0092
:1017B000446F6E65207072696E74696E6720666929
:1017C0006C650A0020496E76616C696420657874E6
:1017D00072756465722000000040C00000A0C00067
:1017E000000000000023430000404300003743484E
:1017F0006F6D652025732573257320666972737478
:10180000002066697273740A005A00590058004833
:101810006F6D6520004D36303020486F74656E6402
:1018200020746F6F20636F6C6420746F2063686135
:101830006E67652066696C616D656E740A002F2F96
:10184000616374696F6E3A70617573650A000000B8
:1018500040C0000040430000374300004842000001
:10186000484200002042000000005761726E696E1D
:10187000673A20486F6D696E672042756D7020442D
:10188000697669736F72203C20310A0002020400FD
:10189000000000000000000000004000002643009F
:1018A00000454300003743FF01016265640A002CD4
:1018B0002073797374656D2073746F707065642123
:1018C000204865617465725F49443A20004865614B
:1018D00074696E67206661696C65642042454400E6
:1018E00048656174696E67206661696C656400486B
:1018F000656174696E67206661696C65640048653E
:101900006174696E67206661696C656420453000AA
:101910001000AD0330016A0150022B0170030A016F
:101920009004F500B005E500D006D800F007CE0021
:101930001009C500300ABE00500BB700700CB10092
:10194000900DAB00B00EA600D00FA200F0109D00CD
:1019500010129900301395005014920070158E00EB
:1019600090168B00B0178700D0188400F019810002
:10197000101B7E00301C7B00501D7900701E76000D
:10198000901F7300B0207000D0216E00F0226B0019
:10199000102469003025660050266300702761001E
:1019A00090285E00B0295C00D02A5900F02B560028
:1019B000102D5400302E5100502F4E0070304B002F
:1019C00090314800B0324500D0334200F0343E0040
:1019D00010363B00303737005038330070392E0056
:1019E000903A2900B03B2300D03C1B00F03D110091
:1019F000103F0100F03F0000436F6F6C646F776E23
:101A00000046616E2073706565640046616E2073E8
:101A1000706565640042656400426564004E6F7ADB
:101A20007A6C65004E6F7A7A6C65004D61696E0064
:101A30005654726176206D696E005654726176203C
:101A40006D696E005654726176206D696E00566D38
:101A5000696E00566D696E00566D696E00566D6157
:101A600078204500566D6178204500566D617820DC
:101A70004500566D6178205A00566D6178205A00F5
:101A8000566D6178205A00566D6178205900566D68
:101A90006178205900566D6178205900566D617843
:101AA000205800566D6178205800566D6178205896
:101AB000004D6F74696F6E00416D61782045004183
:101AC0006D6178204500416D6178205A00416D615B
:101AD00078205A00416D6178205900416D6178206D
:101AE0005900416D6178205800416D61782058009F
:101AF000412D74726176656C00412D74726176655A
:101B00006C00412D7265747261637400412D7265C1
:101B1000747261637400416363656C004163636563
:101B20006C004D6F74696F6E0056652D6A65726B3F
:101B30000056652D6A65726B0056652D6A65726B7D
:101B400000567A2D6A65726B00567A2D6A65726B43
:101B50000056792D6A65726B0056792D6A65726B35
:101B60000056792D6A65726B0056782D6A65726B26
:101B70000056782D6A65726B0056782D6A65726B17
:101B8000004D6F74696F6E004573746570732F6DCF
:101B90006D004573746570732F6D6D005A737465B5
:101BA00070732F6D6D005A73746570732F6D6D00B7
:101BB0005973746570732F6D6D005973746570730C
:101BC0002F6D6D005873746570732F6D6D005873B1
:101BD000746570732F6D6D004D6F74696F6E0020AA
:101BE000746F6F206C6F6E6720657874727573699F
:101BF0006F6E2070726576656E7465640A0020638E
:101C00006F6C6420657874727573696F6E20707282
:101C10006576656E7465640A0024F4D43050C38E12
:101C200020C2A24017828B7011127A910D816CD95B
:101C30000AA861E108C7586607615143061E4B5D5B
:101C400005C145A7041A411104093D9803713931B2
:101C5000034036DB0265339102D4305402802E1DDE
:101C600002632CEE01752AC501B028A0011027815E
:101C7000018F2564012B244B01E0223401AC211F8C
:101C8000018D200D01801FFC00841EED00971DDFDB
:101C900000B81CD200E61BC600201BBC00641AB2B0
:101CA00000B219A8000A19A0006A189900D117916A
:101CB0000040178B00B516840031167E00B31579ED
:101CC000003A157300C7146F0058146A00EE1366CB
:101CD000008813630025135E00C7125B006C125767
:101CE0000015125400C111510070114F0021114B09
:101CF00000D61049008D10470046104400021042E3
:101D000000C00F4000800F3E00420F3C00060F3B1A
:101D100000CB0E3800930E37005C0E3500270E34D2
:101D200000F30D3200C10D3100900D3000600D2E1A
:101D300000320D2D00050D2C00D90C2B00AE0C2906
:101D400000850C29005C0C2700350C27000E0C26A2
:101D500000E80B2400C40B2400A00B23007D0B2300
:101D6000005A0B2100390B2100180B2000F80A1F24
:101D700000D90A1E00BB0A1E009D0A1D00800A1D14
:101D800000630A1C00470A1B002C0A1B00110A1AD8
:101D900000F7091A00DD091900C4091900AB091977
:101DA00000920917007B091800630917004C0916F7
:101DB0000036091600200916000A091500F5081555
:101DC00000E0081400CC081400B8081400A408149B
:101DD00000900813007D0812006B081300580812C9
:101DE00000460812003408110023081100120811DF
:101DF0000001081100F0071000E0071000D00710E4
:101E000000C0071000B0070F00A107100091070ED7
:101E10000083070F0074070F0065070E0057070EB9
:101E20000049070E003B070D002E070E0020070D8E
:101E30000013070D0006070D00F9060C00ED060D56
:101E400000E0060C00D4060C00C8060C00BC060C12
:101E500000B0060C00A4060B0099060C008D060BC2
:101E60000082060B0077060B006C060B0061060A69
:101E70000057060B004C060A0042060A0038060A04
:101E8000002E060A0024060A001A060A0010060997
:101E90000007060A00FD050900F4050900EB050925
:101EA00000E2050900D9050900D0050900C70509A8
:101EB00000BE050900B5050800AD050800A5050927
:101EC000009C050800940508008C0508008405089E
:101ED000007C050800740508006C0507006505080E
:101EE000005D050700560508004E05070047050779
:101EF000004005080038050700310507002A0507DE
:101F000000230507001C050600160507000F05073E
:101F1000000805060002050700FB040600F504079B
:101F200000EE040600E8040600E2040700DB0406F5
:101F300000D5040600CF040600C9040600C3040649
:101F400000BD040600B7040600B1040500AC040699
:101F500000A6040600A00405009B040600950405E5
:101F600000900406008A040500850405008004062C
:101F7000007A04050075040500700405006B040573
:101F80000066040500610405005C040500570405B3
:101F900000520405004D04050048040500430405F3
:101FA000003E0404003A0405003504050030040432
:101FB000002C04050027040400230405001E04046B
:101FC000001A04040016040500110404000D0404A2
:101FD00000090405000404040000040400FC0304D8
:101FE00000F8030400F4030400F0030400EC03040D
:101FF00000E8030400E4030400E0030400DC03043D
:1020000000D8030400D4030400D0030400CC03046C
:1020100000C8030300C503030024F404D9201BC433
:102020000C5C0E9804C4095F0265077101F405F9A0
:1020300000FB04B30048048700C10369005803553E
:102040000003034500BE023A008402310053022A15
:10205000002902250004022000E4011C00C8011927
:1020600000AF0117009801140084011300710110E2
:10207000006101100051010E0043010D0036010BFB
:10208000002B010B0020010B00150109000C0109B8
:102090000003010800FB000800F3000800EB000744
:1020A00000E4000600DE000600D8000600D20006AC
:1020B00000CC000500C7000500C2000500BD0004FB
:1020C00000B9000400B5000400B1000400AD000434
:1020D00000A9000400A5000300A20003009F000463
:1020E000009B00030098000300950002009300038A
:1020F00000900003008D0002008B000300880002A6
:10210000008600020084000300810002007F0002BC
:10211000007D0002007B00020079000200770001D0
:1021200000760002007400020072000100710002DB
:10213000006F0002006D0001006C0002006A0001E7
:1021400000690002006700010066000100650001EF
:1021500000640002006200010061000100600001F3
:10216000005F0002005D0001005C0001005B0001F7
:10217000005A0001005900010058000100570001F9
:1021800000560001005500010054000100530000FA
:1021900000530001005200010051000100500001F5
:1021A000004F0001004E0000004E0001004D0001F4
:1021B000004C0001004B0000004B0001004A0001F0
:1021C00000490001004800000048000100470001EC
:1021D00000460000004600010045000000450001E7
:1021E00000440001004300000043000100420000E1
:1021F00000420001004100000041000100400001D8
:10220000003F0000003F0001003E0000003E0001D2
:10221000003D0000003D0001003C0000003C0000CB
:10222000003C0001003B0000003B0001003A0000C0
:10223000003A0001003900000039000100380000B8
:1022400000380000003800010037000000370001AE
:1022500000360000003600000036000100350000A6
:10226000003500000035000100340000003400009B
:10227000003400010033000000330000003300018F
:102280000032000000320000003200010031000086
:10229000003100000031000100300000003000007B
:1022A00000300001002F0000002F0000002F000070
:1022B000002F0001002E0000002E0000002E000163
:1022C000002D0000002D0000002D0000002D000159
:1022D000002C0000002C0000002C0000002C00014D
:1022E000002B0000002B0000002B0000002B000141
:1022F000002A0000002A0000002A0000002A000135
:102300000029000000290000002900000029000029
:10231000002900010028000000280000002800001B
:10232000002800000028000100270000002700000E
:102330000027000000270000002700010026000001
:1023400000260000002600000026000000260001F4
:1023500000250000002500000025000000250000E9
:1023600000250000002500010024000000240000DA
:1023700000240000002400000024000100230000CD
:1023800000230000002300000023000000230000C1
:1023900000230000002300010022000000220000B2
:1023A00000220000002200000022000000220001A4
:1023B0000021000000210000002100000021000099
:1023C0000021000000210000002100010020000089
:1023D000002000000020000000200000002000007D
:1023E000002000000020000000200001001F00006D
:1023F000001F0000001F0000001F0000001F000061
:10240000001F0000001F0001001E0000001E000051
:10241000001E0000001E0000004D383420582059D6
:10242000204500204500205A0020204D393037201B
:10243000580053746570706572206D6F746F7220F0
:1024400063757272656E74733A0A00205200202020
:102450004D393030204B004C696E6561722041640B
:1024600076616E63653A0A00205900205800536572
:102470006E736F726C65737320686F6D696E672021
:102480007468726573686F6C643A0A002045302086
:1024900000205A2000205920002058200053746545
:1024A00070706572206472697665722063757272ED
:1024B000656E743A0A0020204D383531205A005A92
:1024C0002D50726F6265204F666673657420286DAB
:1024D0006D293A0A0020440020490020204D333065
:1024E0003420500020440020490020204D3330315A
:1024F0002050005049442073657474696E67733AC4
:102500000A0020460020420020480020204D31349F
:10251000352053004D6174657269616C2068656196
:1025200074757020706172616D65746572733A0ABA
:102530000020204D3432302053004175746F20420A
:102540006564204C6576656C696E673A0A00205AAE
:102550000020590020204D323036205800486F6D41
:1025600065206F66667365743A0A00204500205A3C
:102570000020590020580020420020540020204D07
:10258000323035205300416476616E6365643A20D1
:10259000533C6D696E5F66656564726174653E206B
:1025A000543C6D696E5F74726176656C5F666565DB
:1025B00064726174653E20423C6D696E5F7365674D
:1025C0006D656E745F74696D655F75733E20583C10
:1025D0006D61785F78795F6A65726B3E205A3C6DF9
:1025E00061785F7A5F6A65726B3E20453C6D617809
:1025F0005F655F6A65726B3E0A00205400205200DE
:1026000020204D323034205000416363656C657288
:102610006174696F6E2028756E6974732F73322927
:102620003A20503C7072696E745F616363656C3E02
:1026300020523C726574726163745F616363656CA0
:102640003E20543C74726176656C5F616363656CB7
:102650003E0A00204500205A0020590020204D321B
:1026600030312058004D6178696D756D204163638C
:10267000656C65726174696F6E2028756E6974731C
:102680002F7332293A0A00204500205A00205900B1
:1026900020204D3230332058004D6178696D756DC2
:1026A000206665656472617465732028756E69744F
:1026B000732F73293A0A00204500205A0020590040
:1026C00020204D3932205800537465707320706596
:1026D0007220756E69743A0A0020204D3230302025
:1026E00044300A0020204D3230302044002044691C
:1026F0007361626C65640A0046696C616D656E7435
:102700002073657474696E67733A0020204D31340C
:10271000392043203B20556E69747320696E204335
:10272000656C736975730A002020473231202020C0
:10273000203B20556E69747320696E206D6D0A0010
:1027400053442063617264206F6B0A006F70656E82
:10275000526F6F74206661696C65640A00766F6CF5
:10276000756D652E696E6974206661696C65640AB1
:1027700000534420696E6974206661696C0A0061C7
:1027800075746F25692E6700206178697320647203
:10279000697665722063757272656E743A20007492
:1027A0007275650066616C736500206178697320DD
:1027B00074656D706572617475726520707265778D
:1027C00061726E207472696767657265643A200091
:1027D000207072657761726E20666C616720636C31
:1027E00065617265640A0020737465616C74684386
:1027F000686F70206D617820737065656420736503
:102800007420746F20002064726976657220686F8E
:102810006D696E672073656E736974697669747922
:102820002073657420746F2000656E717565756521
:10283000696E672022002F2F616374696F6E3A7290
:102840006573756D650A000A003B20454550524F7F
:102850004D20496E6465783A200055706461746952
:102860006E67207A6F666673657420696E204545D1
:1028700050524F4D3A20000E000E000E000E000E7A
:10288000000E000E000E007FC03F801F000E0004EF
:102890000004000E001F003F807FC00E000E000EDF
:1028A000000E000E000E000E000E0007F8000C0CCB
:1028B000001002002001006001804000804003E021
:1028C0004001C04000804000004000006000002047
:1028D00000001000000C0C0007F80001FE000303CC
:1028E000000400800800401800601000207C0020D8
:1028F00038002010002000002000002000006000B0
:10290000004000008003030001FE00FFFFFF7F8006
:10291000FFC0FFC0FFC07F807F80FFC0FFC0FFC03F
:102920003F001E000C005A204F6666736574005A03
:10293000204F666673657400466C6F7700466C6F57
:10294000770046616E2073706565640046616E2095
:1029500073706565640042656400426564004E6F93
:102960007A7A6C65004E6F7A7A6C65005370656593
:1029700064005370656564004D61696E004D6F764B
:10298000652058004D6F76652059004D6F766520A3
:102990005A004578747275646572004D6F766520D3
:1029A000302E316D6D004D6F766520316D6D004DAF
:1029B0006F76652031306D6D004D6F7665206178E2
:1029C0006973004578747275646572004D6F766541
:1029D000205A004D6F76652059004D6F766520585E
:1029E000004578747275646572004175746F206873
:1029F0006F6D6500473238004D6F7665205A004D87
:102A00006F76652059004D6F76652058004D6F76C2
:102A1000656D656E74004D3234004D323320257380
:102A20000057726974696E6720746F2066696C65FF
:102A30003A20006F70656E206661696C65642C20B9
:102A400046696C653A20006F70656E206661696C3E
:102A500065642C2046696C653A200046696C6520E7
:102A600073656C65637465640A002053697A653A1E
:102A7000200046696C65206F70656E65643A2000C1
:102A80006F70656E206661696C65642C2046696CA8
:102A9000653A20002066696C653A2000646F696EB3
:102AA00067006672657368004E6F772000454E447C
:102AB00020535542524F5554494E450A002220702A
:102AC0006F73002220706172656E743A2200535554
:102AD00042524F5554494E452043414C4C2074615D
:102AE000726765743A22004B494C4C45442E2000D5
:102AF000747279696E6720746F2063616C6C2073E7
:102B000075622D67636F64652066696C65732077F5
:102B100069746820746F6F206D616E79206C6576C2
:102B2000656C732E204D4158206C6576656C20696C
:102B3000733A004572726F723A0043616E6E6F7441
:102B4000206F70656E207375626469722000656322
:102B5000686F3A00544845524D414C2052554E4101
:102B60005741592042454400546865726D616C209C
:102B700052756E6177617900544845524D414C2041
:102B800052554E4157415920453100544845524D08
:102B9000414C2052554E4157415920453000202884
:102BA00063616C63756C6174656429210A0020217E
:102BB0003D2000454550524F4D20435243206D6902
:102BC000736D61746368202D202873746F7265645F
:102BD000292000290A002062797465733B20637202
:102BE0006320002073746F72656420736574746968
:102BF0006E6773207265747269657665642028005B
:102C0000204D61726C696E3D563437290A002845A3
:102C10004550524F4D3D00454550524F4D20766531
:102C20007273696F6E206D69736D617463682000E3
:102C300048617264636F6465642044656661756CA5
:102C4000742053657474696E6773204C6F6164659A
:102C5000640A002823000028230000C8000000E8C0
:102C600003000000009643000096430000964300D6
:102C70000020420000C8420000C842000048430053
:102C800000D24300060900FE06018902FE20FFFE75
:102C900007FE06FE00000006000701060606020009
:102CA000808080800080030303060103A0A0A005AC
:102CB00007070600FF5050F850F850500509090664
:102CC00000FE2070A8A07028A87020060808060042
:102CD000FF40A84810204854080507070600FF6079
:102CE0009090609890680103030602038080800240
:102CF00007070602FF4080808080804002070706A9
:102D000002FF8040404040408005050506000088E5
:102D100050F850880505050600002020F820200204
:102D200004040602FEC0404080050101060002F8CE
:102D3000020202060200C0C00406060601001010CE
:102D4000204080800406060601006090909090600C
:102D500003060606010040C0404040E004060606A7
:102D600001006090102040F0040606060100F020EB
:102D7000601010E005060606000010305090F810B4
:102D8000040606060100F080E01010E004060606C6
:102D900001006080E0909060040606060100F010DB
:102DA000102040400406060601006090609090608C
:102DB000040606060100609090701060020505068A
:102DC0000200C0C000C0C00207070602FEC0C0006B
:102DD000C0404080050505060000186080601805A9
:102DE0000303060001F800F8050505060000C030E1
:102DF0000830C004070706010060901060400040E2
:102E00000506060600007090A8B08070050606064C
:102E10000000205088F88888050606060000F08823
:102E2000F08888F0040606060100609080809060BB
:102E3000040606060100E090909090E00406060665
:102E40000100F080E08080F0040606060100F080BA
:102E5000E0808080040606060100609080B09060EB
:102E60000406060601009090F09090900306060676
:102E70000100E040404040E0050606060000381032
:102E80001010906004060606010090A0C0A090906B
:102E90000406060601008080808080F00506060694
:102EA000000088D8A8A8888804060606010090D0EB
:102EB000B09090900506060600007088888888709B
:102EC000040606060100E09090E0808004070706F3
:102ED00001FF609090D0B06010040606060100E08B
:102EE0009090E090900406060601006090402090CB
:102EF00060050606060000F82020202020040606B3
:102F000006010090909090906004060606010090E3
:102F10009090F060600506060600008888A8A8D892
:102F20008805060606000088502020508805060601
:102F3000060000888850202020040606060100F0C4
:102F400010204080F0030606060100E080808080AB
:102F5000E0040606060100808040201010030606EB
:102F6000060100E020202020E005030306000320E6
:102F700050880501010600FEF802020206020480E4
:102F800040040404060100709090700406060601D7
:102F9000008080E09090E0040404060100708080CE
:102FA000700406060601001010709090700404046E
:102FB00006010060B0C07004060606010020504003
:102FC000E040400406060601FE6090907010600428
:102FD00006060601008080E0909090030606060138
:102FE000004000C04040E00308080601FE200060E9
:102FF000202020A0400406060601008080A0C0A07A
:1030000090030606060100C040404040E00504046D
:10301000060000D0A8A888040404060100E09090EF
:103020009004040406010060909060040606060106
:10303000FEE09090E080800406060601FE7090900D
:10304000701010040404060100A0D0808004040461
:1030500006010070C030E00406060601004040E0B2
:103060004050200404040601009090907004040471
:103070000601009090606005040406000088A8A87E
:1030800050040404060100906060900406060601E6
:10309000FE909090709060040404060100F02040BF
:1030A000F003070706010020404080404020010750
:1030B000070602FF8080808080808003070706016A
:1030C000008040402040408004020206010350A0DE
:1030D000FFFFFFFFFFFFFFFFFFFFFFFFFFFFFFFF00
:1030E000FFFFFFFFFFFFFFFFFFFFFFFFFFFFFFFFF0
:1030F000FF000000060007010606060200800080AF
:103100008080800406060601FF2070A0A0702005C4
:1031100007070600FF304840F04040F80505050667
:103120000000A8508850A80506060600008850F840
:1031300020F8200107070602FF8080800080808041
:103140000407070601FF708060906010E003010132
:10315000060105A0060707060000788494A494845D
:103160007803050506010160A06000E0050505067D
:1031700000002850A05028040303060100F010109E
:10318000040101060102F00607070600007884B476
:10319000A4A48478040101060105F00403030601D8
:1031A000026090600507070600FF2020F82020003D
:1031B000F803050506010140A02040E003050506CF
:1031C0000101C0204020C002020206020440800427
:1031D00005050601FF9090B0D080050606060000A8
:1031E00078E8E8682828010101060202800202024C
:1031F0000602FE408003050506010140C04040E094
:1032000003050506010140A04000E0050505060094
:1032100000A0502850A00508080600FF40C04050FC
:10322000703078100508080600FF40C0405068085C
:1032300010380508080600FFC0204030F030781034
:103240000407070601002000206080906005070742
:1032500006000040202050708888050707060000FF
:103260001020205070888805070706000020502095
:103270005070888805070706000028502050708885
:103280008805070706000050002050708888050751
:1032900007060000205020507088880506060600AA
:1032A0000078A0F0A0A0B80408080601FE60908095
:1032B00080906020400407070601004020F080E075
:1032C00080F00407070601002040F080E080F00451
:1032D00007070601002050F080E080F00407070691
:1032E00001005000F080E080F00307070601008035
:1032F00040E0404040E00307070601002040E04076
:103300004040E003070706010040A0E0404040E0E5
:10331000030707060100A000E0404040E005060664
:103320000600007048E8484870040707060100508E
:10333000A090D0B090900407070601004020609054
:103340009090600407070601002040609090906014
:103350000407070601002050609090906004070762
:1033600006010050A06090909060040707060100DD
:103370005000609090906005050506000088502080
:1033800050880408080601FF1070B0B0D0D0E0806B
:103390000407070601004020909090906004070702
:1033A00006010020409090909060040707060100FD
:1033B0002050909090906004070706010050009004
:1033C000909090600507070600001020885020208C
:1033D0002004060606010080E09090E080040606C6
:1033E0000601006090A0A090A0040707060100401D
:1033F00020007090907004070706010020400070C4
:1034000090907004070706010020500070909070A3
:1034100004070706010050A0007090907004060693
:10342000060100500070909070040707060100200C
:1034300050207090907005040406000070A8B078C9
:103440000406060601FE708080702040040707060F
:10345000010040200060B0C0700407070601002092
:10346000400060B0C07004070706010020500060F3
:10347000B0C070040606060100500060B0C07003C2
:103480000707060100804000C04040E00307070630
:103490000100204000C04040E00307070601004053
:1034A000A000C04040E0030606060100A000C040A6
:1034B00040E004070706010030601070909060043F
:1034C000070706010050A000E0909090040707064F
:1034D0000100402000609090600407070601002072
:1034E00040006090906004070706010020500060D3
:1034F00090906004070706010050A0006090906063
:10350000040606060100500060909060050505065F
:1035100000002000F8002004040406010070B0D070
:10352000E004070706010040200090909070040717
:1035300007060100204000909090700407070601E4
:103540000020500090909070040606060100500084
:10355000909090700409090601FE20400090909020
:103560007090600408080601FE8080E09090E08082
:10357000800408080601FE50009090907090600052
:10358000060900FE0701920321207FFF07FF07FFC6
:10359000000000060000010707060200808080800E
:1035A000800080030202060105A0A00507070600AF
:1035B000005050F850F850500507070600002078DA
:1035C000A07028F020050707060000C0C8102040A2
:1035D00098180507070600006090A040A8906802B0
:1035E0000303060104C040800307070601002040D2
:1035F00080808040200307070601008040202020B3
:10360000408005050506000120A870A820050505D5
:103610000600012020F820200203030602FFC0401C
:1036200080050101060003F8020202060200C0C084
:103630000505050600010810204080050707060063
:10364000007088888888887003070706010040C0DA
:1036500040404040E0050707060000708808708081
:1036600080F8050707060000F81020100808F0058C
:10367000070706000010305090F8101005070706E5
:103680000000F880F0080888700507070600007041
:103690008080F0888870050707060000F808102071
:1036A0002020200507070600007088887088887031
:1036B000050707060000708888780808700205056D
:1036C000060200C0C000C0C00206060602FFC0C05D
:1036D00000C0408004070706000010204080402002
:1036E00010050303060002F800F8040707060100AE
:1036F00080402010204080050707060000708808E1
:103700001020002005070706000070880868A8A898
:1037100070050707060000708888F8888888050704
:1037200007060000F08888F08888F0050707060083
:103730000070888080808870050707060000F08888
:1037400088888888F0050707060000F88080F080E8
:1037500080F8050707060000F88080F0808080056B
:103760000707060000708880B8888870050707067C
:103770000000888888F8888888010707060200808A
:1037800080808080808005070706000038101010B8
:103790001090600507070600008890A0C0A09088E0
:1037A000050707060000808080808080F8050707F5
:1037B00006000088D8A888888888050707060000C2
:1037C0008888C8A898888805070706000070888838
:1037D00088888870050707060000F08888F08080D8
:1037E0008005070706000070888888A8906805078C
:1037F00007060000F08888F0A090880507070600FB
:1038000000788080700808F0050707060000F8209F
:103810002020202020050707060000888888888847
:10382000887005070706000088888888885020056A
:1038300007070600008888888888A85005070706BB
:1038400000008888502050888805070706000088F7
:10385000888850202020050707060000F80810205F
:103860004080F8030707060100E08080808080E048
:103870000505050600018040201008030707060122
:1038800000E02020202020E0050303060004205053
:1038900088050101060000F80202020602058040C8
:1038A00005050506000070087888780507070600FA
:1038B000008080B0C88888F005050506000070808B
:1038C00080887005070706000008086898888878CF
:1038D0000505050600007088F880700507070600DA
:1038E000003048E0404040400506060600FF708872
:1038F000887808700507070600008080B0C88888AF
:10390000880107070602008000808080808003080D
:10391000080601FF200020202020A0400407070601
:103920000000808090A0C0A090030707060100C09F
:103930004040404040E0050505060000D0A8A8A88A
:10394000A8050505060000B0C88888880505050695
:10395000000070888888700506060600FFF08888D9
:10396000F080800506060600FF788888780808053C
:103970000505060000B0C88080800505050600002A
:1039800070807008F00407070600004040E04040E7
:1039900040300505050600008888889868050505FB
:1039A00006000088888850200505050600008888E4
:1039B000A8A8500505050600008850205088050677
:1039C000060600FF8888887808700505050600004F
:1039D000F8102040F803070706010020404080400F
:1039E00040200107070602008080808080808003DD
:1039F0000707060100804040204040800502020683
:103A00000002689000000006000000060900FE00A9
:103A10000000000001090008FE000005080806007B
:103A20000040F0C88888987810050808060000C093
:103A3000F88888888888F80505050600012030F890
:103A400030200508080600002070F820202020E023
:103A50000509090600FF2070A8A8B888887020050D
:103A600009090600FFE080C0B0A828302828050911
:103A7000090600FFF8A88888888888A8F8050A0A37
:103A80000600FE205050505088A8A88870030303F9
:103A900006000340A04001050800FF060121023591
:103AA00020FFFF07FF06FF09005022165680808086
:103AB000800080153353A0A0A00257575050F850F3
:103AC000F850500257572070A070287020133555B9
:103AD00080A040A02002475740A0A040A0A05025B1
:103AE00013538080801226564080808080401226AA
:103AF000568040404040800245559060F060900202
:103B000055552020F8202011335360408004415146
:103B1000F011335340E040024656101020408080A0
:103B200012365640A0A0A0A04012365640C04040D9
:103B300040E00246566090106080F0024656F02049
:103B4000601090600246562060A0F0202002465689
:103B5000F080E01090600246566080E09090600235
:103B60004656F010202040400246566090609090EB
:103B700060024656609090701060122555C0C000DB
:103B8000C0C011365660600060408012365620403A
:103B900080804020034353F000F0123656804020CE
:103BA00020408012365640A0204000400158583036
:103BB0004898A8A8904030024656609090F09090A7
:103BC000024656E090E09090E00246566090808079
:103BD0009060024656E090909090E0024656F08049
:103BE000E08080F0024656F080E0808080024656F9
:103BF000609080B090600246569090F09090901245
:103C00003656E040404040E002465670202020A05A
:103C10004002465690A0C0A0A090024656808080E8
:103C20008080F002465690F0F090909002465690B8
:103C3000D0F0B0B0900246566090909090600246EE
:103C400056E09090E08080014757609090D0B0603F
:103C500010024656E09090E09090024656609040E8
:103C6000209060123656E040404040400246569058
:103C700090909090600246569090909060600246BE
:103C800056909090F0F09002465690906060909020
:103C9000025656888850202020024656F0102040B8
:103CA00080F0123656E080808080E00246568080A8
:103CB00040201010123656E020202020E01632520C
:103CC00040A0014151F016225280400244547090AD
:103CD00090700246568080E09090E01234546080EC
:103CE000806002465610107090907002445460B08C
:103CF000C060024656205040E0404001455560906B
:103D00007010600246568080E090909012365640C7
:103D100000C04040E01137572000202020A0400282
:103D20004656808090E09090123656C04040404009
:103D3000E0025454D0A8A8A8024454E09090900205
:103D4000445460909060014555E090E080800145CA
:103D5000557090701010024454A0D08080123454DA
:103D600060C020C00246564040E04050200244540B
:103D700090909070123454A0A0A04002545488A88F
:103D8000A850024454906060900145559090709006
:103D900060024454F02040F0024757304020C020D9
:103DA0004030221656808080808080024757C02095
:103DB00040304020C006425250A0FFFFFFFFFFFFEF
:103DC000FFFFFFFFFFFFFFFFFFFFFFFFFFFFFFFF03
:103DD000FFFFFFFFFFFFFFFFFFFFFF09005022165D
:103DE000568000808080800146562070A0A0702000
:103DF0000246562050E04050A00255558870507041
:103E0000880256568850F820F82022175780808064
:103E1000008080800247577080E0907010E017317A
:103E200051A002565670A8C8C8A87014355560A095
:103E30006000E003435350A050123353E02020149D
:103E40003151E002565670E8D8E8D870173151E089
:103E500015335340A04012355540E04000E0143582
:103E60005540A02040E0143555C020C020C0162287
:103E7000524080014555909090E08002565678E877
:103E8000E8682828241151801122524080143555A9
:103E900040C04040E014355540A04000E00343538B
:103EA000A050A0024757808080A060F020024757B2
:103EB0008080A0D010207002475780408060A0F022
:103EC0002012365640004080A040024757402060F4
:103ED00090F0909002475720406090F090900247F9
:103EE0005760906090F0909002475750A06090F01B
:103EF000909002475790006090F090900247576072
:103F0000906090F0909002465670A0A0F0A0B00192
:103F10004757609080809060400247574020F08073
:103F2000E080F00247572040F080E080F0024757E1
:103F30006090F080E080F00247579000F080E080D1
:103F4000F01237578040E0404040E01237572040A1
:103F5000E0404040E012375740A0E0404040E012CF
:103F60003757A000E0404040E00256567048E8480D
:103F7000487002475750A090D0B0909002475740E9
:103F80002060909090600247572040609090906031
:103F90000247576090609090906002475750A06031
:103FA000909090600247579000609090906012331C
:103FB00053A040A002465670B0B0D0D0E0024757A0
:103FC00040209090909060024757204090909090B1
:103FD0006002475760909090909060024757900021
:103FE0009090909060025757102088502020200217
:103FF000465680E09090E0800246566090A0A090E7
:10400000A002475740200070909070024757204010
:10401000007090907002475720500070909070028E
:10402000475750A000709090700246565000709014
:10403000907002475760906070909070025454F0F6
:1040400068B0781135556080806040024757402045
:104050000060B0C06002475720400060B0C06002FE
:10406000475760900060B0C060024656500060B094
:10407000C060123757804000C04040E012375720E0
:104080004000C04040E012375740A000C04040E030
:10409000123656A000C04040E0024757A040A01092
:1040A00070906002475750A000E0909090024757F0
:1040B0004020006090906002475720400060909040
:1040C000600247576090006090906002475750A090
:1040D00000609090600246569000609090601235AB
:1040E000554000E0004002445470B0D0E002475711
:1040F0004020009090907002475720400090909090
:104100007002475760900090909070024656900061
:1041100090909070014858204000909070906001FD
:1041200047578080E090E080800147579000909052
:1041300070906001050700FE0500FB01F220FFFE04
:1041400005FE05FE020040021525808080008005E6
:104150003242A0A002556550F850F8500146562052
:1041600070C030E02002556590102040480255652F
:10417000608068906805122280800225354080802A
:1041800080400225358040404080043343A040A059
:1041900003334340E0400122324080043141E002D9
:1041A000112180025565081020408002455560901D
:1041B000909060022535C040404040024555E010D7
:1041C0006080F0024555E0106010E0024555206027
:1041D000A0F020024555F080E010E00245556080D7
:1041E000E09060024555F010204040024555609037
:1041F000609060024555609070106003132380004A
:1042000080021424800080800235452040804020B8
:10421000033343E000E00235458040204080024502
:1042200055E0106000400255657088B8A8700245DE
:1042300055609090F090024555E090E090E0023596
:10424000456080808060024555E0909090E00235A6
:1042500045E080E080E0023545E080E08080024576
:10426000557080B090700245559090F09090023556
:1042700045E0404040E00245553010109060024556
:104280005590A0C0A09002354580808080E0025506
:104290006588D8A8888802455590D0B0909002458E
:1042A000556090909060024555E09090E080014606
:1042B00056609090906010024555E09090E090021A
:1042C000455570806010E0023545E04040404002B6
:1042D000455590909090600245559090A0A0400266
:1042E000556588A8A8A85002455590906090900206
:1042F00045559090701060023545E0204080E00206
:104300002535C0808080C00255658040201008029D
:104310002535C0404040C005324240A0024151F026
:1043200005223280400244547090907002455580BE
:10433000E09090E002344460808060024555107047
:1043400090907002445460B0C0600235452040E057
:10435000404000465670909070106002455580E0D5
:1043600090909002152580008080800027374000C3
:1043700040404040800245558090A0E090021525C5
:104380008080808080025464F0A8A8A8024454E091
:1043900090909002445460909060004656E0909057
:1043A000E08080004656709090701010023444A057
:1043B000C0808002445470C030E002354540E04087
:1043C0004020024454909090700244549090A04039
:1043D000025464A8A85050023444A04040A00046B3
:1043E00056909090701060024454F02040F00235D6
:1043F00045604080406002152580808080800235C5
:1044000045C0402040C005425250A0FFFFFFFFFFC3
:10441000FFFFFFFFFFFFFFFFFFFFFFFFFFFFFFFFAC
:10442000FFFFFFFFFFFFFFFFFFFFFFFF020040FF57
:10443000FFFFFFFFFFFFFFFFFFFFFFFFFFFFFFFF8C
:10444000FFFFFFFFFFFFFFFFFFFFFFFFFFFFFFFF7C
:10445000FFFFFFFFFFFFFFFFFFFFFFFFFFFFFFFF6C
:10446000FFFFFFFFFFFFFFFFFFFFFFFFFFFFFFFF5C
:10447000FFFFFFFFFFFFFFFFFFFFFFFFFFFFFFFF4C
:10448000FFFFFFFFFFFFFFFFFFFFFFFFFFFF010633
:104490000D00FE09016602D620FFFE0BFE0AFE0D8E
:1044A00000602219698080808080808000801833BD
:1044B00063A0A0A00357675050F850F8505002591D
:1044C000692078A0A0702828F02002596948A850D7
:1044D00010204050A89002586840A0A040A098909A
:1044E00068281363808080113B6B2040408080806F
:1044F0008080404020113B6B8040402020202020C5
:1045000040408006556520A870A8200455652020ED
:10451000F82020113363604080065161F811336345
:1045200040E0400259690808101020404080800295
:1045300059692050888888888850200259692060ED
:10454000A02020202020F8025969708888081020B7
:104550004080F8025969F808102070080888700235
:104560005969101030505090F81010025969F880B5
:1045700080B0C80808887002596970888080F08807
:10458000888870025969F8081010202040404002C5
:10459000596970888888708888887002596970881D
:1045A0008888780808887011386840E0400000402A
:1045B000E04011386840E0400000604080025969E6
:1045C000081020408040201008045464F80000F8CF
:1045D00002596980402010081020408002596970FB
:1045E000888808102020002002596970888898A8BF
:1045F000A8B080780259692050888888F88888880F
:10460000025969F048484870484848F002596970B2
:104610008880808080808870025969F048484848C6
:10462000484848F0025969F8808080F0808080F81E
:10463000025969F8808080F080808080025969701A
:10464000888080809888887002596988888888F86E
:1046500088888888123969E040404040404040E006
:1046600002596938101010101010906002596988B2
:104670008890A0C0A090888802596980808080803E
:10468000808080F80259698888D8A8A88888888896
:1046900002596988C8C8A8A898988888025969707A
:1046A0008888888888888870025969F0888888F0A6
:1046B00080808080015A6A70888888888888A8707D
:1046C00008025969F0888888F0A0908888025969A2
:1046D000708880807008088870025969F82020204E
:1046E0002020202020025969888888888888888826
:1046F0007002596988888888505050202002596972
:1047000088888888A8A8A8A8500259698888505025
:1047100020505088880259698888505020202020D5
:1047200020025969F808101020404080F8113B6BB6
:10473000E0808080808080808080E0025969808075
:1047400040402010100808113B6BE0202020202062
:1047500020202020E0085363205088015161F82A6E
:10476000226280400256667008788898680259690B
:10477000808080F088888888F00256667088808003
:1047800088700259690808087888888888780256ED
:10479000667088F880887002596930484040F0405F
:1047A00040404000586870888888780888700259AE
:1047B00069808080B0C8888888881238684000C0C6
:1047C00040404040E0004A6A100030101010109045
:1047D000906002596980808090A0C0A090881239B2
:1047E00069C040404040404040E0025666D0A8A822
:1047F000A8A888025666B0C888888888025666705D
:104800008888888870005868F0888888F080808060
:104810000058687888888878080808025666B0C802
:1048200080808080025666708860108870025868A8
:104830004040F0404040483002566688888888985A
:10484000680256668888885050200256668888A874
:10485000A8A85002566688502020508800586888C2
:1048600088889868088870025666F810204080F89A
:10487000015B6B1820202020C02020202018221946
:1048800069808080808080808080015B6BC0202078
:1048900020201820202020C008536348A890FFFF44
:1048A000FFFFFFFFFFFFFFFFFFFFFFFFFFFFFFFF18
:1048B000FFFFFFFFFFFFFFFFFFFFFFFFFFFFFF0DFA
:1048C0000060221969800080808080808080035889
:1048D000682070A8A0A0A870200259693048404004
:1048E000E0404048B00356668870505070880259C6
:1048F0006988885050F820F820202219698080802B
:10490000800080808080124A6A6090806090906011
:104910001090601A3262A0A00359697088A8D8C8A4
:10492000D8A88870045767700878887800F803560C
:10493000662850A0A05028045363F8080816316177
:10494000E00359697088E8D8D8E8D888700A5161BE
:10495000F8174464609090600357672020F8202087
:1049600000F807356540A02040E007356540A040CD
:1049700020C02A226240800058688888888898E889
:10498000808002596978E8E8E8E868282828262124
:1049900061C0202262408007356540C04040E0048D
:1049A0005767708888887000F8035666A0502828DA
:1049B00050A0025A6A40C04040E008182838080257
:1049C0005A6A40C04040E01028081038025A6A4035
:1049D000A04020A04818283808025969200020204B
:1049E0004080888870025A6A40200020508888F8E9
:1049F0008888025A6A10200020508888F888880227
:104A00005A6A30480020508888F88888025A6A28F4
:104A1000500020508888F88888025A6A5050002038
:104A2000508888F88888025A6A2050202050888848
:104A3000F8888802596958A0A0A0B0E0A0A0B800EA
:104A40005B6B7088808080808088702040025A6A0A
:104A5000402000F88080F08080F8025A6A10200020
:104A6000F88080F08080F8025A6A304800F8808030
:104A7000F08080F8025A6A505000F88080F0808000
:104A8000F8123A6A804000E04040404040E0123A6C
:104A90006A204000E04040404040E0124A6A609096
:104AA00000E04040404040E0123A6AA0A000E040F0
:104AB00040404040E0025969F0484848E8484848CA
:104AC000F0025A6A2850008888C8A8988888025A34
:104AD0006A40200070888888888870025A6A10208E
:104AE0000070888888888870025A6A304800708808
:104AF0008888888870025A6A285000708888888858
:104B00008870025A6A5050007088888888887003BC
:104B100055658850205088015B6B08709898A8A84C
:104B2000A8C8C87080025A6A40200088888888888F
:104B30008870025A6A1020008888888888887002E5
:104B40005A6A30480088888888888870025A6A5073
:104B5000500088888888888870025A6A10200088E7
:104B600088502020202002596980F0888888F080B1
:104B70008080025969609090A0A0908888B0025906
:104B800069402000700878889868025969102000F0
:104B900070087888986802596930480070087888E9
:104BA00098680259692850007008788898680259F6
:104BB00069505000700878889868025A6A30483006
:104BC00000700878889868025666702870A0A8500F
:104BD00000586870888080887020400259694020A1
:104BE000007088F88088700259691020007088F879
:104BF0008088700259693048007088F88088700297
:104C000059695050007088F8808870123969804066
:104C100000C040404040E0123969204000C04040A0
:104C20004040E0124969609000C040404040E012BE
:104C30003969A0A000C040404040E0025A6A5020BC
:104C40006010708888888870025969285000B0C840
:104C50008888888802596940200070888888887010
:104C6000025969102000708888888870025969305C
:104C700048007088888888700259692850007088B8
:104C800088888870025969505000708888888870B8
:104C9000035767202000F80020200158680870980A
:104CA000A8A8C87080025969402000888888889820
:104CB00068025969102000888888889868025969B4
:104CC0003048008888888898680259695050008860
:104CD0008888889868005B6B1020008888889868AE
:104CE000088870005A6A8080B0C88888C8B0808000
:104CF000005B6B50500088888898680888700000B6
:104D000000000000000000000000000000000000A3
:104D10000000000000000000000000000000000093
:104D2000000C000000000000000C0000000000006B
:104D3000001200000000000000230000000000003E
:104D40000021000000000000004C80000000000076
:104D5000005E8000000000000092400000000000A3
:104D600000A1400000000000012120000000000020
:104D7000027F900000000000020010000000000010
:104D800007FFF80000000000040008000000000019
:104D900008000400000000000800060000000000F9
:104DA0001000020000000000301E010000000000A2
:104DB000207F81000000000041FFE0800000000033
:104DC00043FCF08000000000873B784000000001B9
:104DD0008EDBFC60000000010FEBCC200000000225
:104DE0001FEDB610000000021FDEB6100000000428
:104DF00039CD7F080000000436E0FF0800000008FD
:104E00007EC0BB84000000187F005D86000000109B
:104E10007FC0ED82000000203CC073010000002034
:104E20003B337F01000000701BE77E03800000C859
:104E30001DEEDE04C00000880FDEDC04400001240B
:104E40000FDF3C092000012607DBF8192000027261
:104E500003E7F0139000025101FFE0229000048963
:104E6000007F802448000904801E004824000BFEB7
:104E7000400000DFF40010004000008002001FFF2F
:104E8000FFFFFFFFFE000000000000000000000028
:104E900000000000000000000000000000001022E0
:104EA000103C3C0E1F00102210042211040010229E
:104EB000100822110400102210083C1104001022D6
:104EC00010102211040010221020221104001E1CB8
:104ED0001E3C3C0E0400000000000000000000002A
:104EE00000000000000000000000000000000000C2
:104EF00000000000000000000000000000000000B2
:104F000000000000000000000000000000000000A1
:104F10000000000000000000000000000000000091
:104F20000000000000000000000000000000000081
:104F300000000000000000000000000052657365E2
:104F40006E643A20002042002050006F6B004B49F5
:104F50004C4C45442E20004B494C4C2063617573EA
:104F6000656420627920746F6F206D7563682069B5
:104F70006E6163746976652074696D65202D2063A8
:104F8000757272656E7420636F6D6D616E643A2028
:104F900000506C65617365207265736574005052D2
:104FA000494E5445522048414C5445440050726982
:104FB0006E7465722068616C7465642E206B696C18
:104FC0006C28292063616C6C6564210A0050726F43
:104FD00062696E67206661696C6564004D313137C6
:104FE00020426564206C6576656C696E6720666139
:104FF000696C65642E0A4730205A31300A473020E8
:1050000045300A4D33303020503235205338383057
:105010000A4D333030205035302053300A4D333074
:10502000302050323520533838300A4D333030205C
:105030005035302053300A4D333030205032352037
:10504000533838300A4734205331004D313137203E
:1050500050726F6265207375636365737366756CF8
:105060000A0050524F4245204641494C20434C458E
:10507000414E204E4F5A5A4C450A004D313137208F
:105080004C6576656C696E67205820417869730AB3
:105090004732380A473020583136302046393939BE
:1050A000390A4730205A352046363030300A4739E1
:1050B000310A4D3231312053300A4D3430300A4DEF
:1050C000393036205A3630300A4730205A2D3135A3
:1050D00020463530300A4730205A352046353030AA
:1050E0000A4739300A4D3430300A4D393036205AAB
:1050F0003936300A4D3231312053310A4D34303097
:105100000A4732380A4D313137204C6576656C6973
:105110006E6720646F6E652E0A4D313137205265FF
:10512000776970696E67206E6F7A7A6C650A4731AD
:1051300032205030205331322054300A4D31313733
:105140002050726F62696E67206265640000002201
:1051500000250028002B002E003100340002010041
:1051600000050108010B0100002100240027002A8E
:10517000002D003000330001010000040107010A86
:105180000105050505070508080808020202020ACC
:105190000A080804040404010101010101010103DA
:1051A00003030303030303040707070C0C0C0C0C95
:1051B0000C0C0C0202020206060606060606060B88
:1051C0000B0B0B0B0B0B0B010210202008081020FF
:1051D0004010204080020102010804020101020483
:1051E0000810204080804020100804020180040242
:1051F0000180402010080402010804020101020499
:105200000810204080010204081020408000000A9D
:105210000B02090C0D0E080703040100000000003A
:10522000000000000000000000000000000000007E
:10523000000000000000000000121110000000003B
:10524000000000000000000000000000000000005E
:1052500000000050726F62696E67206661696C655C
:10526000640A0050726F62696E67206661696C65DE
:105270006400205A3A200020593A200042656420F8
:10528000583A2000F000DFF911241FBECFEFD1E221
:10529000DEBFCDBF00E00CBF14E0A0E0B2E0E2E270
:1052A000F4E602E00BBF02C007900D92AC34B107E8
:1052B000D9F728E1ACE4B4E001C01D92A436B207EE
:1052C000E1F719E2C3E4D9E200E006C02197010941
:1052D000802FFE010F947C31C234D10780E0080793
:1052E000A9F70E9410580D9400320C9400002F92E0
:1052F0003F924F925F926F927F928F929F92AF9266
:10530000BF92CF92DF92EF92FF920F931F93CF93B2
:10531000DF93CDB7DEB7C158D1090FB6F894DEBF21
:105320000FBECDBFC158DF4F8883CF57D04080918B
:1053300071088D3411F40C947C32843511F40C9482
:105340002B40873411F00C946B40E0906F08F09084
:1053500070082AE1E216F10409F4ABC7CCF444E08A
:10536000E416F1044CF452E0E516F1040CF060C0D0
:10537000F7FE32C00C94854084E0E816F10409F48D
:1053800025C69CE0E916F10409F467C60C94854033
:10539000AEE1EA16F10409F4CFC744F4ECE1EE16ED
:1053A000F10409F4C0C70CF48BC7C2C72BE5E216A1
:1053B000F10411F40C940A323CE5E316F10411F403
:1053C0000C940F324AE5E416F10411F00C94854078
:1053D000109254040C94854080912002882311F48B
:1053E0000C9485408AE50E947BB8482F89E5CF5709
:1053F000DF4F4883C158D0400E947BB8682F88E5B2
:10540000C058DF4F6883C058D0400E947BB8CF5748
:10541000DF4F4881C158D040C058DF4F6881C05825
:10542000D0400E942DB181110C9485400C94904085
:1054300041E061E081E00E942DB181110C94854032
:1054400080912002882311F40C94854011E082E0C1
:10545000E816F10409F010E00E94B6B882E50E9457
:10546000AAB8882309F45CC10E9444B86B017C018E
:105470004090F70E5090F80E6090F90E7090FA0E72
:105480002091FB0E3091FC0E4091FD0E5091FE0ECE
:105490002B962CAF3DAF4EAF5FAF2B9780913F085F
:1054A00090914008A0914108B09142082F968CAF8E
:1054B0009DAFAEAFBFAF2F97209143083091440806
:1054C000409145085091460863962CAF3DAF4EAFD2
:1054D0005FAF639720E030E0A901C701B6010F94E8
:1054E000172A882309F458C5A30192012F966CADA1
:1054F0007DAD8EAD9FAD2F970F94172A811111C0EE
:105500002B962CAD3DAD4EAD5FAD2B9763966CAD3C
:105510007DAD8EAD9FAD63970F94172A882309F454
:105520003BC520E030E0A901C701B6010F94172A5E
:10553000881F8827881F18130BC080E090E0A0E820
:10554000BFE3A3968CAF9DAFAEAFBFAFA3970AC02A
:1055500020E030E040E85FEBA3962CAF3DAF4EAFCC
:105560005FAFA397A30192012F966CAD7DAD8EAD79
:105570009FAD2F970F94802E6B966CAF7DAF8EAF43
:105580009FAF6B972B962CAD3DAD4EAD5FAD2B977E
:1055900063966CAD7DAD8EAD9FAD63970F94802EFD
:1055A0006F966CAF7DAF8EAF9FAF6F976B962CAD44
:1055B0003DAD4EAD5FAD6B97CA01B9010F947C2A2A
:1055C0004B015C016F962CAD3DAD4EAD5FAD6F975D
:1055D000CA01B9010F947C2A9B01AC01C501B40139
:1055E0000F94812E0F94EC3067966CAF7DAF8EAF29
:1055F0009FAF679720E030E040E05FE30F947C2AA4
:105600004B015C01A7019601C701B6010F947C2AEA
:105610006B017C01A5019401C501B4010F947C2AA2
:105620009B01AC01C701B6010F94802E0F94EC30A2
:105630009B01AC01A3966CAD7DAD8EAD9FADA397E4
:105640000F947C2A4B015C012F962CAD3DAD4EADE5
:105650005FAD2F97C301B2010F94812E20E030E09F
:1056600040E05FE30F947C2A6B017C016F966CAD88
:105670007DAD8EAD9FAD6F97905867962CAD3DADCB
:105680004EAD5FAD67970F945D2F9B01AC01C501D7
:10569000B4010F947C2A9B01AC01C701B6010F94A1
:1056A000812EA30192010F94802E6B017C016396E1
:1056B0002CAD3DAD4EAD5FAD63972B966CAD7DAD22
:1056C0008EAD9FAD2B970F94812E20E030E040E00F
:1056D0005FE30F947C2A2B013C0167962CAD3DAD16
:1056E0004EAD5FAD67976B966CAD7DAD8EAD9FADEA
:1056F0006B970F945D2F9B01AC01C501B4010F9412
:105700007C2A9B01AC01C301B2010F94812E2B9620
:105710002CAD3DAD4EAD5FAD2B970F94802E14C0D8
:1057200089E40E94AAB8882329F00E9444B86B013A
:105730007C0103C0C12CD12C76018AE40E94AAB856
:105740008823F9F00E9444B863966CAF7DAF8EAFAA
:105750009FAF639720E030E0A901C701B6010F9425
:10576000172A81111EC020E030E0A90163966CADBC
:105770007DAD8EAD9FAD63970F94172A811111C037
:105780000BC420E030E0A901C701B6010F94172A2D
:10579000882309F401C463961CAE1DAE1EAE1FAE75
:1057A0006397D701C601B0582B968CAF9DAFAEAFB3
:1057B000BFAF2B9763962CAD3DAD4EAD5FAD6397FC
:1057C00050582F962CAF3DAF4EAF5FAF2F979C0137
:1057D000AD01BC01CD010F947C2A4B015C012F96D9
:1057E0002CAD3DAD4EAD5FAD2F97CA01B9010F9401
:1057F0007C2A9B01AC01C501B4010F94812E0F944A
:10580000EC30E3966CAF7DAF8EAF9FAFE3978091A6
:10581000F70E9091F80EA091F90EB091FA0E6796DE
:105820008CAF9DAFAEAFBFAF6797A7019601BC012C
:10583000CD010F94812EA3966CAF7DAF8EAF9FAF3D
:10584000A3972091FB0E3091FC0E4091FD0E5091DC
:10585000FE0E6F962CAF3DAF4EAF5FAF6F97639666
:105860002CAD3DAD4EAD5FAD63976F966CAD7DAD2C
:105870008EAD9FAD6F970F94812EA7966CAF7DAFC5
:105880008EAF9FAFA79780913F0890914008A0915D
:105890004108B0914208AB968CAF9DAFAEAFBFAFA1
:1058A000AB97A3962CAD3DAD4EAD5FADA397BC01BC
:1058B000CD010F94802E6B017C0120914308309123
:1058C00044084091450850914608AF962CAF3DAF33
:1058D0004EAF5FAFAF97A7962CAD3DAD4EAD5FAD70
:1058E000A797AF966CAD7DAD8EAD9FADAF970F9482
:1058F000802E4B015C018091FF0E9091000FA091D2
:10590000010FB091020FEB968CAF9DAFAEAFBFAF62
:10591000EB979C01AD016091470870914808809118
:10592000490890914A080F94802E6B966CAF7DAF1A
:105930008EAF9FAF6B9720914B0830914C084091F0
:105940004D0850914E08E7962CAF3DAF4EAF5FAF7C
:10595000E7978091030F9091040FA091050FB091EC
:10596000060FEF968CAF9DAFAEAFBFAFEF97A7011D
:1059700096012B966CAD7DAD8EAD9FAD2B970F94A0
:105980007C2A2B013C01A50194012F966CAD7DADC5
:105990008EAD9FAD2F970F947C2A9B01AC01C30164
:1059A000B2010F94812E2B013C01A50194012B968D
:1059B0006CAD7DAD8EAD9FAD2B970F947C2A4B01C6
:1059C0005C01A70196012F966CAD7DAD8EAD9FADAC
:1059D0002F970F947C2A9B01AC01C501B4010F9451
:1059E000802EA30192010F94F42E6B017C0120E024
:1059F00030E0A9010F94172A87FF0AC02BED3FE082
:105A000049EC50E4C701B6010F94812E6B017C0173
:105A1000112351F02BED3FE049EC50E4C701B601F2
:105A20000F94802E6B017C0120E030E0A901C701BA
:105A3000B6010F94172A811128C0AB962CAD3DAD4D
:105A40004EAD5FADAB9767966CAD7DAD8EAD9FAD46
:105A500067970F94172A811118C0AF962CAD3DADF2
:105A60004EAD5FADAF976F966CAD7DAD8EAD9FAD1A
:105A70006F970F94172A811108C06BEDC62E6FE047
:105A8000D62E69ECE62E60E4F62EE3962CAD3DAD05
:105A90004EAD5FADE397C701B6010F947C2A9B0121
:105AA000AC010F947C2A4B015C016B962CAD3DAD93
:105AB0004EAD5FAD6B97CA01B9010F947C2A9B0173
:105AC000AC01C501B4010F94812E0F94EC304B0151
:105AD0005C012FE632E143E85AE30F94172A87FD71
:105AE00057C2C501B4010F94F62F0F94CA2F1B01A2
:105AF000672B19F422242394312CB10180E090E02B
:105B00000F941B2A4B015C019B01AC01C701B6013C
:105B10000F945D2F67966CAF7DAF8EAF9FAF679789
:105B2000A50194016B966CAD7DAD8EAD9FAD6B976D
:105B30000F945D2FE3966CAF7DAF8EAF9FAFE39771
:105B4000EF962CAD3DAD4EAD5FADEF97E7966CADEA
:105B50007DAD8EAD9FADE7970F94802EA50194018A
:105B60000F945D2FE7966CAF7DAF8EAF9FAFE79739
:105B700067962CAD3DAD4EAD5FAD6797CA01B901DB
:105B80000F947C2A20E030E040E05FE30F947C2A11
:105B90009B01AC0160E070E080E89FE30F94802EF1
:105BA000AB966CAF7DAF8EAF9FAFAB97EB962CAD46
:105BB0003DAD4EAD5FADEB9729873A874B875C874C
:105BC000EF968CAD9DADAEADBFADEF978D879E8747
:105BD000AF87B88B6091010270910202072E000C12
:105BE000880B990B0F941D2A2091A3023091A402D7
:105BF0004091A5025091A6020F947C2A2AE037ED2D
:105C000043E25CE30F947C2A6BAF7CAF8DAF9EAF19
:105C10000E94844C9B01AC0128533F4F4F4F5F4F74
:105C2000AF962CAF3DAF4EAF5FAFAF9728964FAC5E
:105C3000289729965FAC29972A966FAC2A972B96BE
:105C40007FAC2B9741E050E06D965FAF4EAF6D9704
:105C500059E168965FAF68976D96AEADBFAD6D9731
:105C6000A215B30509F459C10E94C4BE0E94844C18
:105C7000DC01CB01AF962CAD3DAD4EAD5FADAF9726
:105C8000821B930BA40BB50BB7FD11C00E94844C73
:105C90009B01AC0128533F4F4F4F5F4FAF962CAF46
:105CA0003DAF4EAF5FAFAF9780E00F94311668966F
:105CB0003FAD6897315068963FAF6897332309F43A
:105CC0004BC0AB962CAD3DAD4EAD5FADAB972F96B7
:105CD0006CAD7DAD8EAD9FAD2F970F947C2A6B017F
:105CE0007C0167962CAD3DAD4EAD5FAD6797B201BF
:105CF000C3010F947C2AA70196010F94812E7B018A
:105D00008C01AB962CAD3DAD4EAD5FADAB97B20106
:105D1000C3010F947C2A4B015C0167962CAD3DAD0D
:105D20004EAD5FAD67972F966CAD7DAD8EAD9FADDF
:105D30002F970F947C2A9B01AC01C501B4010F94ED
:105D4000802E2B013C01C701D8012F968CAF9DAF4F
:105D5000AEAFBFAF2F9761C06D964EAD5FAD6D9783
:105D6000BA0180E090E00F941B2A67962CAD3DAD00
:105D70004EAD5FAD67970F947C2A4B015C010F9489
:105D80005A2F6B017C01C501B4010F94E2304B0125
:105D90005C01A70196012B966CAD7DAD8EAD9FADDC
:105DA0002B970F947C2A2B013C01A501940163964B
:105DB0006CAD7DAD8EAD9FAD63970F947C2A9B013A
:105DC000AC01C301B2010F94812E2B013C01A5014E
:105DD00094012B966CAD7DAD8EAD9FAD2B970F943E
:105DE0007C2A4B015C01A701960163966CAD7DADE9
:105DF0008EAD9FAD63970F947C2A9B01AC01C501CA
:105E0000B4010F94802E2F966CAF7DAF8EAF9FAFF5
:105E10002F9759E168965FAF68979201A301A39607
:105E20006CAD7DAD8EAD9FADA3970F94812E698330
:105E30007A838B839C832F962CAD3DAD4EAD5FADA9
:105E40002F97A7966CAD7DAD8EAD9FADA7970F94A4
:105E5000812E6D837E838F839887E3962CAD3DAD35
:105E60004EAD5FADE39769857A858B859C850F94F0
:105E7000812E69877A878B879C87E7962CAD3DAD0D
:105E80004EAD5FADE7976D857E858F8598890F94C0
:105E9000812E6D877E878F87988B80910002882363
:105EA00021F0CE0101960E9403F8E0904F04898111
:105EB0009A81AB81BC8188A399A3AAA3BBA38D813E
:105EC0009E81AF81B8858CA39DA3AEA3BFA3898516
:105ED0009A85AB85BC8588A799A7AAA7BBA7CE0141
:105EE00080960E9456A58E01055C1F4F9E01235F80
:105EF0003F4FAE01485D5F4FBE016C5D7F4FCE01ED
:105F000080960E9430DA6D968EAD9FAD6D970196AA
:105F10006D969FAF8EAF6D979FCEE0904F048091AE
:105F20003F0890914008A0914108B091420888A391
:105F300099A3AAA3BBA38091430890914408A09180
:105F40004508B09146088CA39DA3AEA3BFA3809142
:105F5000470890914808A0914908B0914A0888A73D
:105F600099A7AAA7BBA7CE0180960E9456A58E012D
:105F7000055C1F4F2BE438E0AE01485D5F4FBE016A
:105F80006C5D7F4FCE0180960E9430DA0E94CFB9BF
:105F90000E945EA50C948540E3E3FBE284918F01AF
:105FA0000F5F1F4F882321F00E944961F801F6CF4F
:105FB000E7E8F2E084918F010F5F1F4F882311F40F
:105FC0000C9485400E944961F801F4CF80E50E945D
:105FD000AAB8882329F00E9404B86B017C0103C091
:105FE000C12CD12C760183E50E94AAB8882361F0E8
:105FF0000E9444B820E030E04AE754E40F947C2A41
:106000000F94CA2F6B017C010E94A9DF80915C0272
:10601000811105C060E08DE992E00E94A2AB0E9470
:106020005EA580917C1290917D12A0917E12B0911C
:106030007F12C80ED91EEA1EFB1E0E94844CDC0192
:10604000CB018C199D09AE09BF09B7FD02C00C94A4
:10605000854080E00F943116F0CF41E061E081E0AF
:106060000E942DB181110C94854080E50E94AAB850
:10607000882321F00E9414B8F62E01C0F12C83E58C
:106080000E94AAB8882321F00E9414B88B0102C094
:106090000CE010E084E50E94AAB881110E9414B8B7
:1060A00082E50E94AAB8882329F00E9444B84B01D7
:1060B0005C0106C0812C912C40EDA42E40E4B42E4E
:1060C000B1E0FB1611F40C948540E2E0FE128DC0A5
:1060D00080E090E0A4E3B2E489839A83AB83BC833D
:1060E00080E090E0A0E3B3E48D839E83AF83B88724
:1060F00080E090E0A0E8BFE389879A87AB87BC8700
:10610000002311F40C94854018A219A21AA21BA214
:106110009E01205E3F4FAE01475F5F4FBE016B5F48
:106120007F4FCE0101960E9413B210E0E12CF12CBA
:1061300018A219A21AA21BA2B7010F2C000C880BDF
:10614000990B0F941D2A2CE739ED40E25FE30F9481
:106150007C2A2B013C010F945A2FA50194010F9426
:106160007C2A20E030E040E353E40F94812E6BAFB3
:106170007CAF8DAF9EAFC301B2010F94E230A50199
:1061800094010F947C2A20E030E044E352E40F9421
:10619000812E23966CAF7DAF8EAF9FAF2397AE015C
:1061A000405E5F4FBE01655C7F4FCE01CF960E947F
:1061B0003EB3FFEFEF1AFF0A2AE0E216F10409F0FE
:1061C000B7CF1F5F101708F4B1CF18A219A21AA2F7
:1061D0001BA2AE01405E5F4FBE016B5F7F4FCE01E1
:1061E00001960E943EB30C94854080E090E0A6EEBC
:1061F000B2E489839A83AB83BC8340E050E060E3E0
:1062000073E44D835E836F83788780E090E0A0E83D
:10621000BFE389879A87AB87BC87C12CD12C24E345
:10622000E22E22E4F22EC8A2D9A2EAA2FBA24CA33B
:106230005DA36EA37FA388A799A7AAA7BBA71BAE40
:106240001CAE1DAE1EAE9E01255C3F4FAE01485DEB
:106250005F4FBE016C5D7F4FCE0180960E9413B2EE
:10626000112715950795F12C8F2D90E08017910738
:1062700014F00C9485401BAE1CAE1DAE1EAEAE01DC
:10628000455C5F4FBE016B5F7F4FCE0101960E9460
:106290003EB31BAE1CAE1DAE1EAEAE01455C5F4FE5
:1062A000BE016C5D7F4FCE0180960E943EB3F39499
:1062B000DBCF81E0809320021092B3120C948540D2
:1062C00041E061E081E00E942DB181110C94854094
:1062D00080E090E0A0E2B1E489839A83AB83BC8341
:1062E00080E090E0A6E3B3E48D839E83AF83B8871C
:1062F00080E090E0A0EAB1E489879A87AB87BC8709
:1063000080E50E94AAB8882319F00E9414B801C041
:1063100060E068A3BE016F5F7F4FCE0180960F944F
:106320004A220C94854080E00E946F870C9485403F
:106330000F94EF150C948540C090F70ED090F80E96
:10634000E090F90EF090FA0E88E50E94AAB881114B
:1063500008C020E030E0A901C701B6010F94812EEA
:1063600002C00E9444B868A379A38AA39BA3C090EB
:10637000FB0ED090FC0EE090FD0EF090FE0E89E535
:106380000E94AAB8811108C020E030E0A901C7012D
:10639000B6010F94812E02C00E9444B86B017C01AB
:1063A00069837A838B839C8388A099A0AAA0BBA0D1
:1063B00022E630E140E450ECC501B4010F94A7306F
:1063C00087FF02C00C94854022E430E043E253E4AE
:1063D000C501B4010F94172A181614F40C948540C3
:1063E00021E338E040E850ECC701B6010F94A73034
:1063F00087FF02C00C94854022E430E048E253E479
:10640000C701B6010F94172A181614F40C9485408E
:106410000C94454181E0809354040C9485400E9483
:10642000A9DF43E353E029965FAF4EAF2997E7EF2B
:10643000EE2EEEE0FE2EF2E5CF2EF8E1DF2E312C2F
:1064400000E010E02996AEADBFAD29978D91299659
:10645000BFAFAEAF29970E94AAB88823B9F10E94B6
:1064600044B82B013C01133049F0F6012081318101
:10647000428153810F94802E2B013C01D7012D9135
:106480003D914D915C91C301B2010F94802E4B015F
:106490005C012DEB37E346E855EB0F94A73087FD01
:1064A0000AC02DEB37E346E855E3C501B4010F946C
:1064B000172A18165CF4133011F001E002C03324DF
:1064C0003394F70140825182628273821F5FF4E04D
:1064D000EF0EF11C24E0C20ED11C143009F0B2CF33
:1064E000002319F00E94D8B603C031100E9407F7AC
:1064F0000E946A680C94854080916F0890917008A2
:106500008D37910509F480C70CF0E1C08D349105F9
:1065100009F41FC50CF059C08931910509F402C373
:106520001CF58431910509F47BC27CF4813191051D
:1065300009F46BC22CF4029708F4E3C10C94854073
:10654000429709F46AC70C9485408631910509F495
:10655000AEC20CF4A8C28731910509F4AEC24897C7
:1065600009F4C1C20C9485408F31910509F45DC4D2
:106570007CF48B31910509F4F3C20CF4E3C28C3145
:10658000910509F429C34E9709F430C30C94854052
:106590008934910509F4CCC44CF48032910509F496
:1065A00033C48A9709F46DC40C9485408B349105EB
:1065B00009F4CBC48C34910511F00C94854080E033
:1065C00095E10E94BB4C0C9485408B36910509F4F3
:1065D00018C7ECF58435910509F41FC7CCF4813553
:1065E000910509F414C734F48E34910509F4B5C447
:1065F0000C9485408235910509F40CC783359105CB
:1066000011F00C94854081E0809353040C948540F4
:106610008836910509F4B0C56CF48535910509F407
:10662000FFC68C35910511F00C9485400E943869A5
:106630000C9485408936910509F48CC68A369105FB
:1066400011F00C9485400E947D6C0C94854083373A
:10665000910509F4E8C6D4F48E36910509F4C8C54D
:1066600034F48D36910509F4B4C60C9485408F3608
:10667000910509F4CEC58237910511F00C9485403F
:106680000E94A9DF0E946A680C94854087379105B3
:1066900009F4D4C66CF48537910509F4C7C686376A
:1066A000910511F00C9485400E94E7670C94854099
:1066B0008837910509F4D0C68937910511F00C94FB
:1066C000854010924C1810924B180C9485408039DC
:1066D00031E0930709F485C70CF084C0833D910530
:1066E00009F4CFC6E4F5883C910509F4BEC6C4F4AC
:1066F0008139910509F4B6C634F48C38910509F452
:106700000FC60C9485408B39910509F43DC68E3B2C
:10671000910511F00C9485400E94CB6A0C94854041
:106720008C3C910509F4A7C66CF4893C910509F4E9
:106730009FC68B3C910511F00C9485400E94CA665F
:106740000C9485408D3C910509F498C68E3C9105CA
:1067500011F00C9485400E9429570C9485408C328E
:1067600051E0950709F496C6DCF48D3D910509F4D6
:106770008BC64CF48C3D910511F00C9485400E9421
:106780003F560C948540823E910509F480C68232C2
:10679000914011F00C9485400E9415550C94854051
:1067A0008F32E1E09E0709F419C774F48D3221E0BD
:1067B000920709F472C68E32914011F00C94854014
:1067C0000E940B540C948540803341E0940709F4F7
:1067D00002C78336914011F00C9485400E94194DF8
:1067E0000C9485408835A2E09A0711F40C945E3C25
:1067F000D4F58C3AE1E09E0709F4FCC794F48239A1
:1068000021E0920709F4F4C60CF4EEC6843A41E0A4
:10681000940709F4F1C6893A914009F46DC70C94C4
:106820008540863FA1E09A0709F4EAC774F4843FE3
:10683000E1E09E0709F4E1C7853F914011F00C9417
:1068400085400F94BA0C0C948540873F21E0920755
:1068500009F4D9C78C31924011F00C9485400E9404
:10686000674D0C9485408F3843E0940711F40C94E5
:10687000093FE4F48438A3E09A0711F40C94773DBF
:1068800044F48335934011F00C948540EEE4FBE230
:10689000BDC78A38F3E09F0711F40C94B23E8B38E1
:1068A000934011F40C94793E0C948540823933E086
:1068B000930711F40C941340C4F4803953E0950706
:1068C00011F40C94223F8139934011F00C948540CF
:1068D00083E3E82E83E0F82E8E010F5F1F4F6E01D9
:1068E000F9E0CF0ED11C0C94783F803AB3E09B07BF
:1068F00009F48EC2873E934011F40C9416400C9418
:106900008540A0906D08B0906E0880E50E94AAB8FE
:10691000882359F00E9404B86B017C0111E0672BB9
:10692000682B692B31F410E004C010E0C12CD12C8D
:10693000760183E50E94AAB88823F1F00E9444B84A
:1069400020E030E04AE754E40F947C2A0F94CA2FE9
:106950006B017C01111112C0672B682B692B71F43C
:10696000A114B10459F0D5018C91882339F061E06C
:10697000C5010E94C0AB07C0112391F360E085ED13
:1069800092E00E94A2AB81E0809384060E94A9DF7E
:106990000E945EA5C114D104E104F104F1F08091DC
:1069A0007C1290917D12A0917E12B0917F12C80E40
:1069B000D91EEA1EFB1E0E94844CDC01CB018C19FF
:1069C0009D09AE09BF09B7FF1CC0809184068823CA
:1069D000C1F080E00F943116EECF809184068823B9
:1069E00021F080E00F943116F8CF8091001560E01F
:1069F000823019F487EC92E002C088EB92E00E94AA
:106A0000A2AB109284060C94854060E088EE92E080
:106A10000E94A2AB17981698159814980C9485406C
:106A2000E0E0F3E084918F010F5F1F4F882321F096
:106A30000E944961F801F6CF1092061840E050E03C
:106A4000BA0182EB95E10E940D648BE1E2EBF5E186
:106A5000DE01159601900D928A95E1F78091B015AF
:106A60009091B1159C838B8381E394E09A83898311
:106A700040E050E0BE016F5F7F4F8DEC93E00F94DC
:106A80003406CE0101960E94FCF9E1EFF2E0849118
:106A90008F010F5F1F4F882311F40C9485400E94D3
:106AA0004961F801F4CF0E94BAF10C94854010922C
:106AB0005A1510925B150C948540E0916D08F09189
:106AC0006E088081882329F0803209F41082319683
:106AD000F8CF40E061E080916D0890916E080F94CE
:106AE0006E080C94854019821A821B821C8218A29F
:106AF00019A21AA21BA280912F08882341F040E01E
:106B0000BE016F5F7F4FCE0180960E94D6F88091C4
:106B10005B15882319F081E080935A150F94821C2D
:106B20000C94854010925A1580E095E10E94BB4C70
:106B300081E193E090935411809353110E94F7B335
:106B40000C94854080915B15882311F40C9485404A
:106B500083E50E94AAB881110C949C410C94854055
:106B600080915B15882351F1E6E1F3E084918F0178
:106B70000F5F1F4F882321F00E944961F801F6CF73
:106B80006091FD177091FE178091FF17909100188A
:106B90004AE00E94A2618FE20E9449616091F91768
:106BA0007091FA178091FB179091FC174AE00E94B0
:106BB000A2618AE00E9449610C948540E8E2F3E01A
:106BC00084918F010F5F1F4F882311F40C9485402F
:106BD0000E944961F801F4CF40E060E080916D08C7
:106BE00090916E080F946E080C94854080915B150F
:106BF000882311F40C9485408CE497E10E94DA63B9
:106C00008CE497E10E949A6F1092591510925815D2
:106C1000E0906D08F0906E0880915B15882311F468
:106C20000C9485400F9463081D8218861C821B8279
:106C300081E394E09A8389838EEA95E19093CE155F
:106C40008093CD15F70180818F3209F068C06FE223
:106C500070E0C7010F94C6318C010F5F1F4F9E017A
:106C60002F5F3F4F59010115110509F45EC06FE216
:106C700070E0C8010F94C6316C01009709F456C04A
:106C80000817190708F052C04C01801A910AA40194
:106C9000B801CE0180960F94E631E0E2F0E0EC0F0F
:106CA000FD1FE80DF91D10828E01005E1F4FD801F7
:106CB0008D918D01882319F00E944961F8CF8AE0F7
:106CC0000E9449616091CD157091CE1561157105D5
:106CD00011F06C5F7F4F21E0AE01405E5F4FCE014F
:106CE00005960E94E272811112C0BE01605E7F4F64
:106CF0008FE593E00E94D9A58EE20E9449618AE067
:106D00000E944961C5010E94FCF90C948540B09233
:106D1000CE15A092CD1586010F5F1F4FA4CF8FEC2B
:106D200095E19093CE158093CD1587016091CD1597
:106D30007091CE156115710511F06C5F7F4F18A22F
:106D40001BA222E0A801CE0180960E94E27281116E
:106D500002C0F12C14C0CE0180960F94A2058823A6
:106D6000C1F361E0CE0180960E94A36F009789F382
:106D700025EEFC0120831BA20F945B20F82ECE0190
:106D800080960E94B6B9FF2009F1E9E3F3E084910F
:106D90007F012FEFE21AF20A882321F00E94496155
:106DA000F701F5CFD8018D918D01882319F00E944C
:106DB0004961F8CF8AE00E9449611092FD17109254
:106DC000FE171092FF171092001818C0E7E4F3E0C6
:106DD00084917F01BFEFEB1AFB0A882321F00E9408
:106DE0004961F701F5CFF80181918F01882319F0EE
:106DF0000E944961F8CF8EE20E944961CE0101965E
:106E00000E94FCF90C9485400E94A06C0C94854073
:106E100080916D0890916E0821E02093591540E013
:106E200060E00F946E080C94854080E095E10E942C
:106E3000904C68A379A38AA39BA3BE016F5F7F4F89
:106E4000CE0180960E94D84560E0CE0101960E9456
:106E5000C0ABEEE4FBE284918F010F5F1F4F8823EC
:106E600021F00E944961F801F6CFBE016F5F7F4FAC
:106E700083E793E00E94D9A58AE00E9449610C94BF
:106E8000854083E50E94AAB8882311F40C948540BC
:106E90000E9424B8E82E80E50E94AAB8811112C091
:106EA00081E0E11001C080E080937304882329F021
:106EB00024982C9A149A0C948540249A2C9814980F
:106EC0000C94854080E50E94AAB8882341F00E9476
:106ED00014B88B0177FF02C00C94854002C00DE00E
:106EE00010E0902FE0E8F3E088E28E0F24919217F3
:106EF00029F031968E13FACF0C94AD41E3E3FBE217
:106F000084918F010F5F1F4F882321F00E944961F8
:106F1000F801F6CFE8EAF3E084918F010F5F1F4F8D
:106F2000882311F40C9485400E944961F801F4CF44
:106F300080915A1581110C94854080E50E947BB8A0
:106F400081110C94C2410C9485400F94821C0C94C6
:106F500085400F94D51C0C94854083E50E94AAB807
:106F6000882359F00E9414B86E34710531F480E022
:106F700095E10E94C3450C94854018A219A21AA25B
:106F80001BA2E7E1F4E084918F010F5F1F4F88237C
:106F900021F00E944961F801F6CFEEE0F4E084911F
:106FA0008F010F5F1F4F882321F00E944961F80174
:106FB000F6CF60910D1570910E1580E090E04AE0DB
:106FC0000E94A261E1E0F4E084918F010F5F1F4F06
:106FD000882321F00E944961F801F6CF60910F15D6
:106FE0007091101580E090E04AE00E94A261E6EF07
:106FF000F3E084918F010F5F1F4F882321F00E94DF
:107000004961F801F6CF60910D1570910E158091D0
:107010000F1590911015681B790B80910015815008
:1070200021E030E0823010F020E030E0621B730B92
:1070300080E090E04AE00E94A2618AE00E944961FB
:10704000EEEEF3E084918F010F5F1F4F882321F054
:107050000E944961F801F6CF8091111590911215A7
:10706000A0911315B091141588A399A3AAA3BBA34B
:10707000BE016F5F7F4FCE0180960E94D845E1EE42
:10708000F3E084918F010F5F1F4F811106C09E01B5
:107090002F5F3F4F7901890104C00E944961F801C7
:1070A000F0CFD8018D918D01882319F00E9449619C
:1070B000F8CF8091151590911615A0911715B091E4
:1070C000181588A399A3AAA3BBA3BE016F5F7F4F26
:1070D000CE0180960E94D845E1EDF3E084918F01C6
:1070E0000F5F1F4F882321F00E944961F801F6CFFE
:1070F000F70181917F01882319F00E944961F8CF3F
:107100008AE00E944961E9ECF3E084918F010F5F0E
:107110001F4F882321F00E944961F801F6CFE9EB67
:10712000F3E084918F010F5F1F4F882321F00E94AD
:107130004961F801F6CF20E030E04AE754E460917D
:10714000191570911A1580911B1590911C150F94AB
:107150005D2F42E00E942262E7EBF3E084918F0111
:107160000F5F1F4F882321F00E944961F801F6CF7D
:107170008AE00E944961C9C788E690E00E9476B91A
:107180008111C3C78091E50883FF01C0BEC783E5B5
:107190000E94AAB8882309F4B8C70E9444B80F9483
:1071A000C52F709354076093530780E00E942CBD55
:1071B0000E9444B82091D8083091D9084091DA084B
:1071C0005091DB080F94A73018160CF09EC783EE81
:1071D00092E09F938F938FE194E09F938F931F9200
:1071E0000F944E1D0F900F900F900F900F908DC722
:1071F0008EE40E94AAB8882309F487C70E9414B8B5
:1072000060932D0F70932E0F80932F0F9093300F5C
:107210007CC783E50E947BB8882359F083E50E94F0
:10722000AAB8882319F00E9424B801C080E0809396
:10723000E508EEE4FBE284918F010F5F1F4F882386
:1072400021F00E944961F801F6CFE9E3F4E084916E
:107250008F010F5F1F4F882321F00E944961F801C1
:10726000F6CF8091E5088823A1F17BE2C72E74E078
:10727000D72EE12CF12C20E08091E50890E00E2C37
:1072800002C0959587950A94E2F780FF17C0BB244A
:10729000B394B20E222319F08CE20E944961F601E8
:1072A00025913491F901849189010F5F1F4F882343
:1072B00021F00E9449619801F5CF2B2DFFEFEF1AC5
:1072C000FF0A32E0C30ED11C45E0E416F104A1F63A
:1072D00023C0E5E3F4E084918F010F5F1F4F882303
:1072E000D9F00E944961F801F6CFC0905C0ED090B1
:1072F0005D0EE0905E0EF0905F0E20E030E0A901A0
:10730000C701B6010F94172A882309F4E5C442E0A7
:10731000C701B6010E9422628AE00E944961F5C657
:107320008091E50883FDF1C683E50E94AAB8882311
:1073300009F4EBC60E9444B80F94C52F6739710554
:1073400014F066E970E070935207609351070E9451
:10735000E1BCDBC689E690E00E9476B981110C940D
:10736000E743E0E4F4E084918F010F5F1F4F88232F
:1073700021F00E944961F801F6CF0E9478748AE0FA
:107380000E9449610C94E74383E50E94AAB88823D0
:1073900009F4BBC60E9424B8182F8D3308F01CE3F3
:1073A00010936F120E94844C6B017C01212F30E0FE
:1073B000A8EEB3E00F94712EC60ED71EE81EF91E7C
:1073C000C0926B12D0926C12E0926D12F0926E121B
:1073D0009CC68DE690E00E9476B9811196C6809198
:1073E000E50883FD92C683E50E94AAB828968FAF70
:1073F00028978111D2C782E50E94AAB88111CDC712
:1074000084C60E946E6C81C60E945A677EC60E9426
:107410003F6A7BC61092530478C60E94EE6975C617
:107420000E94D66972C60E9424686FC660E080918F
:107430006D0890916E080E94C0AB67C681E0809392
:10744000730424982C9A149A0E9434451092730461
:10745000249A2C98149859C681E080934C188093F4
:107460004B1853C60E94546A50C60E9411674DC6FD
:107470000E94EC664AC60E94656647C60E94525743
:1074800044C60E944B5641C60E94F5553EC60E9416
:10749000AA553BC60E94E05438C685E40E94AAB8AB
:1074A000811110C080E50E947BB8882391F00E9472
:1074B00044B86093780E7093790E80937A0E90930F
:1074C0007B0E07C00E9424B8882361F3E3E3FBE24C
:1074D00071C089E40E947BB8882381F00E9444B87F
:1074E0002CEA35EC47E25EE30F947C2A6093740E3D
:1074F0007093750E8093760E9093770E84E40E94BD
:107500007BB8882381F00E9444B82CEA35EC47E22E
:107510005EE30F945D2F6093700E7093710E8093F5
:10752000720E9093730EEEE4FBE284918F010F5F75
:107530001F4F882321F00E944961F801F6CF409146
:10754000780E5091790E60917A0E70917B0E87E7DC
:1075500094E00E94A3A52CEA35EC47E25EE360913B
:10756000740E7091750E8091760E9091770E0F9437
:107570005D2FAB01BC0183E794E00E9486A52CEA55
:1075800035EC47E25EE36091700E7091710E809170
:10759000720E9091730E0F947C2AAB01BC018FE6A2
:1075A00094E00E9486A58AE00E944961AEC50E94CF
:1075B0004961F80184918F010F5F1F4F8111F7CF4F
:1075C00001E013E0F80181918F01882309F4A4CE32
:1075D0000E944961F7CF0E94615497C50E94BF4E37
:1075E00094C50E94A9DF91C581E00E94F8B28DC5C3
:1075F00080E00E94F8B289C58091F70E9091F80E54
:10760000A091F90EB091FA0E89839A83AB83BC8363
:107610008091FB0E9091FC0EA091FD0EB091FE0E9C
:107620008D839E83AF83B8878091FF0E9091000F6A
:10763000A091010FB091020F89879A87AB87BC8711
:1076400086E50E947BB8882321F088EA94E00F94B5
:10765000162583E50E947BB8882331F00E9435B857
:10766000182F0E94C0B701C010E0F090880E1111D1
:1076700003C0EEE4FBE21AC0F110FBCFE3E3FBE250
:1076800084918F010F5F1F4F882321F00E94496171
:10769000F801F6CFE9E8F4E084918F010F5F1F4F06
:1076A000882339F30E944961F801F6CF84918F0154
:1076B0000F5F1F4F882321F00E944961F801F6CF28
:1076C000F11003C06DEF72E002C069EF72E08BE76A
:1076D00094E00E94D9A58AE00E9449614CE050E004
:1076E00067EF7EE0CE0101960F949231892B09F469
:1076F0000CC50E946A6809C58AE50E947BB8882388
:1077000029F180914D0490914E04892B19F00E942B
:1077100044B808C060914E1870914F18809150186D
:10772000909151186093C9087093CA088093CB0850
:107730009093CC0880E090E0A0E8BFE38093CD0870
:107740009093CE08A093CF08B093D00886E40E940F
:107750007BB8882381F10E9444B820E030E040E803
:107760005FE30F94A73018166CF40E9444B820E031
:1077700030E040E85FE30F94A730181684F00E94D1
:1077800044B811C00E9444B820E030E0A9010F9431
:10779000172A87FFEACF60E070E0CB0104C060E009
:1077A00070E080E89FE36093CD087093CE088093EB
:1077B000CF089093D00883E50E947BB8882351F0CE
:1077C0000E9444B86093250270932602809327029A
:1077D000909328028AE50E947BB8811196C486E4C2
:1077E0000E947BB8811191C483E50E947BB881110E
:1077F0008CC462C70E947C4D88C40E94A18F85C43E
:107800000F94020B82C40E94714D7FC484918F013A
:107810000F5F1F4F882321F00E944961F801F6CFC6
:10782000E1ECF5E084918F010F5F1F4F882321F079
:107830000E944961F801F6CF8AE50E947BB888234F
:1078400069F10E9444B86B017C0120E030E040E027
:1078500050EC0F94A73087FF03C0EAEAF5E013C0AD
:1078600020E030E040EA50E4C701B6010F94172A47
:1078700018169CF3C092E30ED092E40EE092E50E4F
:10788000F092E60E0BC084918F010F5F1F4F88238B
:1078900009F43BC40E944961F801F5CF4091E30E21
:1078A0005091E40E6091E50E7091E60E87EA95E046
:1078B0000E94A3A58AE00E94496127C480E090E06D
:1078C000A0E2B1E489839A83AB83BC8380E090E03B
:1078D000A6E3B3E48D839E83AF83B88780E090E016
:1078E000A0EAB1E489879A87AB87BC8741E061E071
:1078F00081E00E942DB1882319F081E00E946F87FA
:1079000085E40E947BB8882319F00E9444B804C023
:1079100060E070E080E090EC27966CAF7DAF8EAFBA
:107920009FAF27978AE50E94AAB8882379F08AE555
:107930000E94AAB8882319F00E9444B803C060E0EE
:1079400070E0CB0169877A878B879C8788E50E94E6
:10795000AAB8882379F088E50E94AAB8882319F08C
:107960000E9444B803C060E070E0CB0169837A8371
:107970008B839C8389E50E94AAB8882379F089E5E6
:107980000E94AAB8882319F00E9444B803C060E09E
:1079900070E0CB016D837E838F83988785E50E949D
:1079A0007BB8882319F00E9444B804C060E070E0FE
:1079B00088EC92EC23966CAF7DAF8EAF9FAF239790
:1079C0008CE40E947BB8882319F00E9444B803C05D
:1079D00060E070E0CB016BAF7CAF8DAF9EAF82E417
:1079E0000E94AAB8882321F00E9414B8162F01C063
:1079F00015E0F090001580912F08811172C001E010
:107A0000212FAE01415C5F4FBE016F5F7F4FCE0102
:107A10008D5B9F4F0E94ACC2882309F462C081E055
:107A20008093840680918406882309F446C060E030
:107A3000812F0E94756D809160118823D1F1009390
:107A4000641189E49BE90F94710480918406882372
:107A500021F081E00F943116F8CF1092B008109207
:107A6000B1081092B2081092B308109260110E94EF
:107A70002CBD0E94186D0093641182EF9AE90F9457
:107A800071040E94844CDC01CB0188539045AF4FB8
:107A9000BF4F8093B0089093B108A093B208B09301
:107AA000B308109260110093840661E0812F0E9458
:107AB000756D81E00F943116B5CF80E090E0A0EABB
:107AC000B1E488A399A3AAA3BBA380912F0888231C
:107AD00041F0412FBE01605E7F4FCE01CB960E94E8
:107AE000D6F8F1E0FF1211C30F94821C0EC30E945E
:107AF000A9DF8BE40E94AAB8882399F00E9444B8B9
:107B00006B017C0120E030E0A9010F94A73087FDD4
:107B100008C0C092600ED092610EE092620EF092A8
:107B2000630E82E50E94AAB8882361F00E9444B8DF
:107B30006B017C0120E030E0A9010F94172A87FF38
:107B400091C006C0C12CD12C40E8E42E4FEBF42E9E
:107B500084E40E94AAB8882329F00E9444B84B010B
:107B60005C0106C0812C912C30E8A32E3FEBB32E94
:107B700087E50E94AAB8882329F00E9444B82B0107
:107B80003C0106C0412C512C20E8622E2FEB722EB6
:107B900088E40E94AAB8882349F00E9444B82B9632
:107BA0006CAF7DAF8EAF9FAF2B970AC020E030E067
:107BB00040E85FEB2B962CAF3DAF4EAF5FAF2B97FE
:107BC00020E030E0A901C501B4010F94A73087FD82
:107BD00049C020E030E0A901C301B2010F94A730F1
:107BE00087FD40C020E030E0A9012B966CAD7DAD53
:107BF0008EAD9FAD2B970F94A73087FD33C020E04B
:107C000030E0A901C501B4010F94172A8823A1F11E
:107C100020E030E040E05FE3C501B4010F947C2A2E
:107C20006B017C012B962CAD3DAD4EAD5FAD2B971E
:107C3000C301B2010F947C2A4B015C01A70196019C
:107C4000C701B6010F947C2A2BED3FE049E450E4D4
:107C50000F947C2A9B01AC01C501B4010F945D2FE8
:107C60006B017C0120E030E0A901C701B6010F944F
:107C7000A73087FF04C00BC0C12CD12C7601C09265
:107C80005C0ED0925D0EE0925E0EF0925F0EEEE41E
:107C9000FBE284918F010F5F1F4F882321F00E9428
:107CA0004961F801F6CF4091600E5091610E6091EC
:107CB000620E7091630E8BED95E00E94A3A5E5ED39
:107CC000F5E084918F010F5F1F4F882309F40DCBDE
:107CD0000E944961F801F5CFE0EDF5E084918F0154
:107CE0000F5F1F4F882309F417CB0E944961F801E9
:107CF000F5CF88E50E947BB88823F1F00E9414B884
:107D00008B01072E000C220B330B0093500E1093A7
:107D1000510E2093520E3093530EDB012FEF30E0C3
:107D20000F94843120ED37E040E050E00F94452E71
:107D3000B9018EE20E94854B8AE50E947BB88823B8
:107D400029F00E9414B881E00E94059A85E40E94FF
:107D50007BB8882309F4D9C10E9414B882E00E943C
:107D6000059AD3C193E3E92E93E0F92E8E010F5FBC
:107D70001F4F6E0139E0C30ED11CD7018D917D01DB
:107D80000E94AAB8882319F00E9414B802C060E0CB
:107D900070E0F801619371938F01EC15FD0569F7AF
:107DA00049815A8162E173E08DE694E14115510504
:107DB00019F00E9450FB02C00E9428FB4B815C819D
:107DC00068E173E088EF93E14115510519F00E94D5
:107DD00050FB02C00E9428FB4D815E816EE173E082
:107DE00083E893E14115510519F00E9450FB02C050
:107DF0000E9428FB4F81588564E273E08EE093E196
:107E00004115510519F00E9450FB7FC10E9428FBCB
:107E10007CC162E173E08DE694E10E94F8FA68E1CA
:107E200073E088EF93E10E94F8FA6EE173E083E873
:107E300093E10E94F8FA64E273E08EE093E10E941D
:107E4000F8FA63C188E50E947BB8182F89E50E9483
:107E50007BB8E82E8AE50E947BB8F82E85E40E9464
:107E60007BB8082F111108C0E11019C0F11024C00F
:107E70008111A9C411E007C0EE2011F0F11002C079
:107E800010E001C0182F62E173E08DE694E10E94DA
:107E9000DFFAE11005C0112309F493C401C010E01A
:107EA00068E173E088EF93E10E94DFFAF11005C00A
:107EB000112309F488C401C010E06EE173E083E887
:107EC00093E10E94DFFA002339F064E273E08EE070
:107ED00093E10E94DFFA19C11111F7CF16C160E0DA
:107EE00070E0F801619371938F01EC15FD0551F07D
:107EF000D7018D917D010E94AAB8882381F30E9449
:107F000014B8EFCF09811A816091070F7091080FA3
:107F10008091090F90910A0F0115110571F00F94CE
:107F2000CA2F980140E050E07B018C0162E173E0D0
:107F30008DE694E10E948DFA09C00F94CA2FAB011F
:107F400062E173E08DE694E10E943FFA0B811C81AF
:107F500060910B0F70910C0F80910D0F90910E0F8F
:107F60000115110571F00F94CA2F980140E050E0FF
:107F70007B018C0168E173E088EF93E10E948DFA48
:107F800009C00F94CA2FAB0168E173E088EF93E159
:107F90000E943FFA0D811E8160910F0F7091100FAA
:107FA0008091110F9091120F0115110571F00F942E
:107FB000CA2F980140E050E07B018C016EE173E034
:107FC00083E893E10E948DFA09C00F94CA2FAB0198
:107FD0006EE173E083E893E10E943FFA0F81188518
:107FE0006091130F7091140F8091150F9091160FDF
:107FF0000115110571F00F94CA2F980140E050E06F
:108000007B018C0164E273E08EE093E10E948DFAC3
:108010007CC00F94CA2FAB0164E273E08EE093E161
:108020000E943FFA72C00E94344D6FC081E080937D
:1080300020021092B31283E50E94AAB8882319F097
:108040000E9435B803C083E50E947BB881115DC0F2
:108050000F9428195AC0F0906F08FF2021F1EEE428
:10806000FBE284918F010F5F1F4F882321F00E9454
:108070004961F801F6CF84E50E9449616F2D70E0F7
:1080800080E090E04AE00E94A26180E20E944961A3
:1080900001E013E0D8018D918D01882309F43CC9DA
:1080A0000E944961F7CF10924F04EEE4FBE2849105
:1080B0008F010F5F1F4F882321F00E944961F80153
:1080C000F6CF60E070E086EE95E00E94C0A58AE001
:1080D0000E9449611AC0EEE4FBE284918F010F5FB8
:1080E0001F4F882321F00E944961F801F6CF60916B
:1080F00072087091730888EF95E00E94D9A582E21A
:108100000E9449618AE00E944961C158DF4FB881ED
:10811000CF57D040BB2309F45AC30F94BA1857C3A2
:108120000E94B6B880910002882321F08FE398E086
:108130000E9403F80E945EA58091E50883FD86C039
:10814000C0904B08D0904C08E0904D08F0904E083D
:108150002091030F3091040F4091050F5091060FAD
:10816000C701B6010F94172A882309F46FC00E9433
:10817000B6F8882301F1C092030FD092040FE09269
:10818000050FF092060FEEE4FBE284918F010F5F82
:108190001F4F882321F00E944961F801F6CFECE6D9
:1081A000F2E084918F010F5F1F4F882321F00E941E
:1081B0004961F801F6CFC0904B08D0904C08E09090
:1081C0004D08F0904E082091030F3091040F40911C
:1081D000050F5091060FC701B6010F94802E9F77AF
:1081E000E0914F0454E0E59FF0011124E55DFD4F5F
:1081F00020813181428153810F947C2A20E030E03C
:1082000048E453E40F94A730181604F5C092030F06
:10821000D092040FE092050FF092060FEEE4FBE21D
:1082200084918F010F5F1F4F882321F00E944961C5
:10823000F801F6CFEDE4F2E084918F010F5F1F4F5C
:10824000882321F00E944961F801F6CF6091010274
:1082500070910202072E000C880B990B0F941D2AB7
:108260002091A3023091A4024091A5025091A60250
:108270000F947C2A2AE037ED43E25CE30F947C2ADA
:108280000E9449B30E94CFB940CF80E00E94C0B79E
:108290000E94F3B185E40E94AAB8882319F00E94D5
:1082A00035B803C085E40E947BB821E0482FBE01A9
:1082B0006F5F7F4FCE0180960F94DF226B017C01B0
:1082C0009B01AC010F942D31811131C02CEA35ECAA
:1082D00047E257E368A179A18AA19BA10F94812E5F
:1082E000AB01BC0180EB92E00E9486A52CEA35EC44
:1082F00047E257E369817A818B819C810F94812EBB
:10830000AB01BC018BEA92E00E9486A52CEA35EC19
:1083100047E257E3C701B6010F94812EAB01BC01C0
:1083200086EA92E00E9486A58AE00E9449610E9446
:10833000D9B10E946A68E9CE0E9414B8AB01BC01B1
:108340004093FD175093FE176093FF17709300182A
:108350008CE497E10E940D64D8CE802F0F941F1BF0
:108360006E2D802F0E94B84AF12CB701802F0E94F9
:10837000854B0830110509F0C8CEF092D708E0927D
:10838000D608C3CE0E9424B8853620F084E68093B8
:108390004C04BBCE80934C04B8CE0E9444B80F94DA
:1083A000C52F709354076093530780E00E942CBD43
:1083B0006091530770915407072E000C880B990B9E
:1083C0000F941D2A2091D8083091D9084091DA08DD
:1083D0005091DB080F94A73018160CF065C183EE9E
:1083E00092E09F938F9383E694E09F938F931F92E5
:1083F0000F944E1D0F900F900F900F900F9081E0F3
:1084000080931A022F961CAE1DAE1EAE1FAE2F9784
:1084100067961CAE1DAE1EAE1FAE6797312C6896D8
:108420001FAE68975CE36C965FAF6C978CE1A0968B
:108430008FAFA09796E4A4969FAFA497C12CD12CA0
:1084400050E8E52E6FEBF62E812C912C54016091B3
:10845000530770915407072E000C880B990B0F944B
:108460001D2A162F072F782E692E262F372F482FDB
:10847000592FB601C7010F94172A8823E1F02091E4
:10848000D8083091D9084091DA085091DB08612F63
:10849000702F872D962D0F94172A382E331C3324D6
:1084A000331C2896AFAD2897AA2349F0332039F022
:1084B00033243394E7C01C2D0D2D7E2C6F2C0E948D
:1084C000844C6B017C01DC01CB0167962CAD3DAD8A
:1084D0004EAD5FAD6797821B930BA40BB50BB7FD39
:1084E0003DC0D701C60188519C4FAF4FBF4F679623
:1084F0008CAF9DAFAEAFBFAF67970E947874EFE5CA
:10850000F4E084912F019FEF491A590A882321F042
:108510000E944961F201F5CF81149104A104B104D4
:10852000B9F0D501C40188519C4FAF4FBF4FBC017A
:10853000CD016C197D098E099F0928EE33E040E0DA
:1085400050E00F94232ECA01B9010E94086203C0B3
:108550008FE30E9449618AE00E94496180E00F94A4
:1085600031160E945EA52090D808A091D908609687
:10857000AFAF60974090DA085090DB08222D3A2F79
:10858000A201612F702F872D962D0F94802E9F773B
:1085900020E030E040E251E481149104A104B104F0
:1085A00029F40F94172A87FF07C004C00F94A7303F
:1085B000181614F446015701332009F449C02F96C8
:1085C0002CAD3DAD4EAD5FAD2F9721153105410569
:1085D000510541F0D701C601821B930BA40BB50BCB
:1085E000B7FD36C0222D60963FAD6097A201689618
:1085F0006FAD68976C967FAD6C97A0968FADA09786
:10860000A4969FADA4970F94802E20E030E040EC1C
:108610005FE30F94172A87FD4BCFD701C601805A1D
:108620009541AF4FBF4F2F968CAF9DAFAEAFBFAF51
:108630002F9768962FAE689760969FAD60976C965F
:108640009FAF6C97A0964FAEA097A4965FAEA497ED
:1086500080911A028823B1F081149104A104B1041D
:1086600029F4C12ED02EE72CF62CF1CEA8EECA1A92
:10867000A3E0DA0AE108F108C818D908EA08FB08FB
:10868000F7FCEFCF80911A02882309F43ECD60E019
:10869000332029F083E494E00E94A2AB36CD81E53B
:1086A00094E00E94A2AB31CD2896EFAD2897E1115E
:1086B000A6CE8EEE92E095CE40914E1850914F1876
:1086C00060915018709151188AE895E00E94A3A516
:1086D0008AE00E9449618AE00E94496120E030E01E
:1086E000A9016091C9087091CA088091CB08909146
:1086F000CC080F94A73018160CF056C020E030E0DC
:10870000A9016091CD087091CE088091CF08909119
:10871000D0080F94A73018160CF046C0E8E4F5E036
:1087200084918F010F5F1F4F882321F00E944961C0
:10873000F801F6CF4091C9085091CA086091CB0862
:108740007091CC088EE295E00E94A3A58AE00E9479
:108750004961409125025091260260912702709153
:10876000280284E195E00E94A3A58AE00E94496165
:108770004091CD085091CE086091CF087091D008FB
:108780008AEF94E00E94A3A58AE00E944961E5EC8B
:10879000F4E084918F010F5F1F4F882309F4B5CC5B
:1087A0000E944961F801F5CFE8E6F5E084918F0178
:1087B0000F5F1F4F882309F4BDCF0E944961F80164
:1087C000F5CFF1107ACB002309F49FCC7ECBCF57A5
:1087D000DF4F0FB6F894DEBF0FBECDBFDF91CF9154
:1087E0001F910F91FF90EF90DF90CF90BF90AF90CF
:1087F0009F908F907F906F905F904F903F902F90C1
:108800000895CF92DF92EF92FF920F931F93CF9331
:10881000DF936C017A018B01C0E0D0E0CE15DF055B
:1088200089F0D8016D918D01D601ED91FC910190F7
:10883000F081E02DC6011995892B11F47E0102C04B
:108840002196ECCFC701DF91CF911F910F91FF903F
:10885000EF90DF90CF900895089580E090E0089524
:1088600080E008950B96FC01849108950A96FC011E
:1088700084910895FC0184910895FCDF882321F000
:10888000823011F083E0089586E00895FC01E60F40
:10889000F11D849190E0982F88273196E4918E0FF6
:1088A000911D089568E0F2CF66E0F0CF0895FC01D5
:1088B000A681B7818281481B8581483018F0A80FB6
:1088C000B11D4770382F369536953695562F57700F
:1088D00080E890E002C0959587955A95E2F7439F0E
:1088E000402D1124669566956695E62FF0E0E40F1D
:1088F000F11DEA0FFB1F3081222311F0832B02C0F0
:108900008095832380830895FB014181DC011296C9
:108910002C911297421760F013962C9113972417FD
:1089200038F0608115962C91621710F42481BFCF26
:108930000895FC0180819281980F92832181921782
:1089400060F494819F5F94839381890F821710F064
:108950008FEF820F838381E0089580E00895FC010A
:1089600012828081815083831482089581E008956A
:10897000089590E0FC013197E231F10508F04EC016
:108980008827EE58FF4F8F4F0D947C3180918000E7
:108990008F7703C0809180008F7D80938000089541
:1089A00080918000877FF9CF84B58F7702C084B52E
:1089B0008F7D84BD08958091B0008F7703C0809132
:1089C000B0008F7D8093B0000895809190008F77E4
:1089D00007C0809190008F7D03C080919000877FB9
:1089E0008093900008958091A0008F7707C08091B8
:1089F000A0008F7D03C08091A000877F8093A0009E
:108A00000895809120018F7707C0809120018F7D8C
:108A100003C080912001877F8093200108953FB794
:108A2000F89480915A0490915B04A0915C04B091F9
:108A30005D0426B5A89B05C02F3F19F00196A11D26
:108A4000B11D3FBFBA2FA92F982F8827820F911DE4
:108A5000A11DB11DBC01CD0142E0660F771F881F2B
:108A6000991F4A95D1F70895CF93DF93E2E8F6E096
:108A70008491EF012196882321F00E944961FE0133
:108A8000F7CFEAE7F6E08491EF012196882321F001
:108A90000E944961FE01F7CF8091060182FF03C069
:108AA000C7E3D3E002C0CCE3D3E08991882319F077
:108AB0000E944961FACF8AE00E944961E2E7F6E04C
:108AC0008491EF012196882321F00E944961FE01E3
:108AD000F7CF8091060187FF03C0C7E3D3E002C050
:108AE000CCE3D3E08991882319F00E944961FACF41
:108AF0008AE00E944961EAE6F6E08491EF0121965E
:108B0000882321F00E944961FE01F7CF1C9B03C01E
:108B1000C7E3D3E002C0CCE3D3E08991882319F006
:108B20000E944961FACF8AE00E944961E2E6F6E0DC
:108B30008491EF012196882321F00E944961FE0172
:108B4000F7CF8091000184FD03C0C7E3D3E002C0EA
:108B5000CCE3D3E08991882319F00E944961FACFD0
:108B60008AE0DF91CF910C944961FC0127A1222377
:108B700049F0658D768D6F5F7F4F40E150E00D9637
:108B80000D94E52D0895CF93DF93EC0181E08FA341
:108B9000FE013D9680E1DF011D928A95E9F7CE0145
:108BA000E4DF66E18D8D9E8DDF91CF910D94062ED1
:108BB0004F925F926F927F92AF92BF92CF92DF926D
:108BC000EF92FF92CF93DF93EB01FC016081718103
:108BD000828193812CE3C22ED12CE12CF12CA701B0
:108BE00096010F94232EB62EA72ECA01B901A70114
:108BF00096010F94232E6B017C01CA01B90128E173
:108C000030E040E050E00F94232E2B013C01C901DD
:108C10006DE671E00F94553161157105D9F0AF9291
:108C2000BF92DF92CF925F924F929F938F937F93E9
:108C30006F938EE496E09F938F93DF93CF930F947F
:108C4000B0298DB79EB70E960FB6F8949EBF0FBE93
:108C50008DBF61C00097C9F0AF92BF92DF92CF92F3
:108C60005F924F929F938F938EE396E09F938F93A3
:108C7000DF93CF930F94B029EDB7FEB73C960FB6B4
:108C8000F894FEBF0FBEEDBF46C04114510461040D
:108C90007104B9F0AF92BF92DF92CF925F924F9280
:108CA00082E396E09F938F93DF93CF930F94B02945
:108CB0008DB79EB70A960FB6F8949EBF0FBE8DBFB4
:108CC0002AC0C114D104E104F104A9F0AF92BF920B
:108CD000DF92CF928AE296E09F938F93DF93CF93B8
:108CE0000F94B029EDB7FEB738960FB6F894FEBFD3
:108CF0000FBEEDBF10C0AF92BF9286E296E09F9389
:108D00008F93DF93CF930F94B0290F900F900F9014
:108D10000F900F900F90DF91CF91FF90EF90DF9029
:108D2000CF90BF90AF907F906F905F904F900895DD
:108D3000CF92DF92FF920F931F93CF93DF931F92F7
:108D40001F92CDB7DEB76901DB0112960D911C9120
:108D50001397423309F470C0B8F4453109F477C071
:108D6000473109F487C0443109F09DC0D8011596F8
:108D70002C9115971696ED91FC911797CF01820FC4
:108D8000911D820F911D5CC0463409F483C04734A5
:108D900009F484C04B3309F086C0F90181819381C5
:108DA000913029F0933031F4482F885004C048E0C6
:108DB000480F01C0482F21E0D80113963C91381785
:108DC00008F420E031E0F8015281451708F430E062
:108DD00051E0481708F050E0822F852B382319F412
:108DE000252309F460C0D6011296FC90913051F011
:108DF00030F0923049F0933051F42FEF09C020E069
:108E000031E007C021E004C020E03FEF02C020E0D5
:108E100030E0F7FE07C0B601C8012A83398374DD4C
:108E200039812A81F6018081830F80838181820FBD
:108E30008183FF0C71F737C0B901C80165DD33C00C
:108E40001192E817F907E1F7C80189DD2CC0C801C4
:108E500070DD882349F1F80125810680F781E02D36
:108E6000CF01820F911D820F911D1192E817F90712
:108E7000E1F719C0D9011C92F801828111968C93F7
:108E800011978581815012968C9312978381139646
:108E90008C9309C0D80115968C9103C0D801119606
:108EA0008C91F601808381E00F900F90DF91CF913C
:108EB0001F910F91FF90DF90CF90089588E290E08E
:108EC0000197F1F708952EE93FE0009729F0F901A5
:108ED0003197F1F70197F9CF08950F93FC010150F5
:108EE000040F84A996A9941718F0081728F402C053
:108EF000081750F0041740F42150260F83A995A9B4
:108F0000961720F4281720F480E007C0281720F4D3
:108F100081E0261710F0F8CF81E00F910895DB0172
:108F2000ED91FC9119942F923F925F926F927F92F4
:108F30008F929F92AF92BF92CF92DF92EF92FF9269
:108F40000F931F93CF93DF931F92CDB7DEB71C0112
:108F5000C62E142FD22EDC011496ED90FC9015979E
:108F6000C70188DC082FF1018481958186DC982E69
:108F7000013019F48FE0A82E02C0AA24AA94D101CE
:108F800014968D919C91159771DC082FF1018481C5
:108F9000958168DCB82ED10114968D919C9115971E
:108FA00081DCB0E6BD1530F4009721F0E80EF91E23
:108FB00001E610C0F1018481958176DCF0E4FD15B5
:108FC00030F4009721F0E80EF91E01E403C021E11E
:108FD000E20EF11CBD1480F4D10150961C92509702
:108FE00053961C92539754961C92549751961C92E8
:108FF000519752961C92C3C0B01670F3892D90E021
:10900000F70124912F3F21F4FFEFEF1AFF0A59C017
:109010000D114EC0D10114968D919C9115972ADCAB
:1090200097012F5F3F4FF701882311F08230E1F461
:109030008491D10153968C935397F90124915496BE
:109040002C935497F7013396E4915096EC935097F4
:10905000F7013496E4915196EC935197F7013596C8
:10906000E4915296EC9320C08491982F9F70925077
:10907000D10152969C93529782958F7051968C9302
:109080005197F9012491822F8F7054968C935497A5
:1090900022952F7053962C935397F7013296E491B3
:1090A000E295EF705096EC93E114F10479F467C007
:1090B000F7013296E491EA219C012E0F311DE20E58
:1090C000F31E0B1509F488CF0F5F9ACFF10184814D
:1090D0009581D3DBB82ED10153969C90539754962B
:1090E000DC90549751968C915197C80E52969C9152
:1090F0009D0D512E591A0D2D292D452D6C2DC10177
:10910000ECDE8823C9F1C7018B0D911D5C0187E05E
:10911000890DF82EF694F694F694D50C41019CE155
:10912000890E911C6F2C712C5D1431F15C2D850121
:10913000802F8A198F15E0F4F8018491D1011296DD
:109140006D917C9113975C965C935C975D965C92B5
:109150005D975F961C925F975E968C9394014BE3AC
:10916000C1015983DCDE0F5F1F4F5981585FE0CF8B
:10917000A60CB71C5394D8CFF101808901C080E0C0
:109180000F90DF91CF911F910F91FF90EF90DF90A3
:10919000CF90BF90AF909F908F907F906F905F9097
:1091A0003F902F900895EF92FF920F931F93CF93CC
:1091B000DF931F92CDB7DEB78C01DC011296ED90E4
:1091C000FC901397D196ED91FC91D29782E019957E
:1091D00020E030E04AE0B701C801A1DEF82ED80156
:1091E000D196ED91FC91D29783E01995D801D19653
:1091F000ED91FC91D29780E01995FF2081F1F80163
:10920000628173819E012F5F3F4F46E4C80187DE74
:109210008981D8018C9312966D917C9113979E0150
:109220002F5F3F4F47E4C8017ADE8981F8018183CF
:109230006281738120E030E048E4C80170DED8012B
:109240001B968C931B9798012D5C3F4F12966D9146
:109250007C91139747E1C80162DE81E001C080E0A4
:109260000F90DF91CF911F910F91FF90EF90089594
:109270001F920F920FB60F9211240BB60F922F93DD
:109280003F934F935F936F937F938F939F93AF938E
:10929000BF93EF93FF93E0911102F09112021995A1
:1092A000FF91EF91BF91AF919F918F917F916F91BE
:1092B0005F914F913F912F910F900BBE0F900FBE7A
:1092C0000F901F9018951F920F920FB60F921124B6
:1092D0000BB60F922F933F934F935F936F937F93B0
:1092E0008F939F93AF93BF93EF93FF93E0910F0200
:1092F000F09110021995FF91EF91BF91AF919F915D
:109300008F917F916F915F914F913F912F910F902E
:109310000BBE0F900FBE0F901F9018951F920F92CB
:109320000FB60F9211240BB60F922F933F934F93CA
:109330005F936F937F938F939F93AF93BF93EF93BD
:10934000FF93E0910502F09106021995FF91EF91CC
:10935000BF91AF919F918F917F916F915F914F914D
:109360003F912F910F900BBE0F900FBE0F901F904B
:1093700018951F920F920FB60F9211240BB60F92F1
:109380002F933F934F935F936F937F938F939F930D
:10939000AF93BF93EF93FF93E0910302F091040228
:1093A0001995FF91EF91BF91AF919F918F917F910F
:1093B0006F915F914F913F912F910F900BBE0F9046
:1093C0000FBE0F901F9018951F920F920FB60F921D
:1093D00011240BB60F922F933F934F935F936F938C
:1093E0007F938F939F93AF93BF93EF93FF93E091FE
:1093F0000D02F0910E021995FF91EF91BF91AF917F
:109400009F918F917F916F915F914F913F912F919C
:109410000F900BBE0F900FBE0F901F9018951F92CC
:109420000F920FB60F9211240BB60F922F933F930A
:109430004F935F936F937F938F939F93AF93BF935C
:10944000EF93FF93E0910B02F0910C021995FF91BD
:10945000EF91BF91AF919F918F917F916F915F91AC
:109460004F913F912F910F900BBE0F900FBE0F9019
:109470001F9018951F920F920FB60F9211240BB6E2
:109480000F922F933F934F935F936F937F938F939D
:109490009F93AF93BF93EF93FF93E0910902F091F5
:1094A0000A021995FF91EF91BF91AF919F918F9112
:1094B0007F916F915F914F913F912F910F900BBED4
:1094C0000F900FBE0F901F9018951F920F920FB61E
:1094D0000F9211240BB60F922F933F934F935F93EC
:1094E0006F937F938F939F93AF93BF93EF93FF936C
:1094F000E0910702F09108021995FF91EF91BF9159
:10950000AF919F918F917F916F915F914F913F911B
:109510002F910F900BBE0F900FBE0F901F901895BC
:10952000CF93DF93282F30E0F901E35FFD4A849168
:10953000F901E953FE4AD491F901EF57FE4AC4916B
:10954000CC2389F0811115DAEC2FF0E0EE0FFF1F2C
:10955000E55FF94FA591B491EC91ED2381E090E0A6
:1095600021F480E002C080E090E0DF91CF91089587
:109570001F93CF93DF93282F30E0F901E35FFD4A7B
:109580008491F901E953FE4AD491F901EF57FE4A5B
:10959000C491CC23C1F0162F8111EBD9EC2FF0E050
:1095A000EE0FFF1FE35BFE4AA591B4918FB7F894CD
:1095B000111105C09C91ED2FE095E92302C0EC91BB
:1095C000ED2BEC938FBFDF91CF911F9108951F92E8
:1095D0000F920FB60F9211240BB60F922F933F9359
:1095E0004F935F936F937F938F939F93AF93BF93AB
:1095F000EF93FF938091610490916204A0916304C2
:10960000B0916404892B8A2B8B2B59F180916004D3
:10961000E0915E04F0915F049081892780838091BE
:10962000610490916204A0916304B09164041816DF
:1096300019061A061B060CF055C080916104909122
:109640006204A0916304B09164040197A109B10977
:109650008093610490936204A0936304B0936404C4
:1096600041C080911302E5E2F6E0E4919FEF909310
:109670001302E230C9F050F4EE2399F0E13081F5A5
:1096800090916F009D7F90936F002AC0E43019F194
:10969000E0F0E53029F5909173009D7F9093730081
:1096A0001FC010926E001CC0909170009D7F90931F
:1096B000700091E09093B0009091B100987F946019
:1096C0009093B1001092B3000BC0909171009D7FF8
:1096D0009093710005C0909172009D7F90937200ED
:1096E00060E046DFFF91EF91BF91AF919F918F9125
:1096F0007F916F915F914F913F912F910F900BBE92
:109700000F900FBE0F901F9018951F93CF93DF936C
:10971000182FEB010F941F1B209711F460E004C079
:10972000CF3FD10531F461E0812FDF91CF911F91BF
:109730001FCFE12FF0E0E35FFD4AE4914E2F50E0B0
:10974000FA013197E231F10508F09DC08827EC5706
:10975000FF4F8F4F0D947C3184B5806884BDC7BDA9
:1097600097C084B5806284BDC8BD92C080918000DE
:10977000806880938000D0938900C093880088C05F
:1097800080918000806280938000D0938B00C09392
:109790008A007EC080918000886080938000D09392
:1097A0008D00C0938C0074C08091B000806880935D
:1097B000B000C093B3006CC08091B0008062809311
:1097C000B000C093B40064C0809190008068809322
:1097D0009000D0939900C09398005AC08091900057
:1097E000806280939000D0939B00C0939A0050C0F9
:1097F00080919000886080939000D0939D00C093EA
:109800009C0046C08091A00080688093A000809159
:10981000A0008F7B8093A000D093A900C093A800E4
:1098200037C08091A00080628093A000D093AB00ED
:10983000C093AA002DC08091A00088608093A000F2
:10984000D093AD00C093AC0023C08091200180680C
:1098500080932001D0932901C093280119C08091E1
:109860002001806280932001D0932B01C0932A01B4
:109870000FC080912001886080932001D0932D013A
:10988000C0932C0105C0C038D1050CF04CCF46CF99
:10989000DF91CF911F9108958F929F92AF92BF92C7
:1098A000CF92DF92EF92FF926B017C01B8D84B010F
:1098B0005C01C114D104E104F104E9F0B0D8DC0189
:1098C000CB0188199909AA09BB09883E9340A105D3
:1098D000B10578F321E0C21AD108E108F10888EE59
:1098E000880E83E0981EA11CB11CC114D104E104B0
:1098F000F10421F7DECFFF90EF90DF90CF90BF9083
:10990000AF909F908F9008952FB7F8946091560470
:109910007091570480915804909159042FBF089575
:109920000F931F93CF93DF93EC018881813011F463
:10993000EBDF04C069857A858B859C850D811E814E
:109940002F813885601B710B820B930B28EE33E05F
:1099500040E050E00F94232E89819A81AB81BC8135
:10996000BC01CD01620F731F841F951FDF91CF9142
:109970001F910F910895CF93DF93FC012081213037
:1099800051F4EC0182E08083BFDF69877A878B879F
:109990009C8781E001C080E0DF91CF9108951F9204
:1099A0000F920FB60F9211242F933F938F939F9393
:1099B000AF93BF938091560490915704A09158049F
:1099C000B09159043091550423E0230F2D3720F432
:1099D0000196A11DB11D05C026E8230F0296A11D09
:1099E000B11D209355048093560490935704A0937F
:1099F0005804B093590480915A0490915B04A0914B
:109A00005C04B0915D040196A11DB11D80935A04C0
:109A100090935B04A0935C04B0935D04BF91AF91FD
:109A20009F918F913F912F910F900FBE0F901F909C
:109A30001895CF93DF93E3E3FBE28491EF01219646
:109A4000882321F00E944961FE01F7CFE4ECF8E0A1
:109A50008491EF012196882321F00E944961FE0143
:109A6000F7CFDF91CF91089588E50E947BB88823D6
:109A700031F00E9414B88DE694E10E94E35762E150
:109A800073E08DE694E10E9404FA89E50E947BB8B8
:109A9000882331F00E9414B888EF93E10E94E357C5
:109AA00068E173E088EF93E10E9404FA85E40E9484
:109AB0007BB8882331F00E9414B88EE093E10E94B5
:109AC000E35764E273E08EE093E10C9404FA83E5DB
:109AD0000E947BB8882321F00E9435B880938504CA
:109AE000089583E50E947BB8882321F00E9435B851
:109AF00091E089270C942EEA2F923F924F925F9229
:109B00006F927F928F929F92AF92BF92CF92DF928D
:109B1000EF92FF920F931F93CF93DF93CDB7DEB7F2
:109B200063970FB6F894DEBF0FBECDBF41E061E092
:109B300081E00E942DB18111CFC09EE4892E98E171
:109B4000992E87EF9EE09A8B898BFE0131965F01FB
:109B500007EA18E11F01F3E0F00FFB8BF4016591B8
:109B6000759185919491E989FA89C190D190E1909C
:109B7000F190FA8BE98BA70196010F94802E2B01AF
:109B80003C0120E030E040EA51EC0F94A73087FD23
:109B900010C020E030E040EA51E4C301B2010F946C
:109BA000172A181634F0F1014082518262827382C2
:109BB0000DC0F80184911816B4F7F7FAF094F7F88D
:109BC000F094F101C082D182E282F382F101C1906E
:109BD000D190E190F1901F0120E030E040EA51EC9B
:109BE000C701B6010F94A73087FF03C0E3E3FBE290
:109BF0000BC020E030E040EA51E4C701B6010F9409
:109C0000172A18163CF5F2CF84918F010F5F1F4F72
:109C1000882321F00E944961F801F6CFE6EAF8E0D6
:109C200084918F010F5F1F4F882321F00E944961AB
:109C3000F801F6CF61E088E998E00E94A2AB0E94AB
:109C4000688988E290E0988B8F8788EC90E09E8707
:109C50008D873BC0F4E08F0E911C0F5F1F4F8B89E7
:109C600080137CCF84E7E82E84E0F82E10E0F50125
:109C700081919191A191B1915F01F70181939193AC
:109C8000A193B1937F01812F0E949BB31F5F13307B
:109C900071F70E946A6860E088E898E00E94A2ABD1
:109CA00083E992E0988B8F8704E610E01E870D878A
:109CB000BE01615F7F4FCE010D960E9440F38AEB9B
:109CC00092E0988B8F871E870D87BE01615F7F4F63
:109CD000CE010D960E9440F363960FB6F894DEBF56
:109CE0000FBECDBFDF91CF911F910F91FF90EF90ED
:109CF000DF90CF90BF90AF909F908F907F906F90AC
:109D00005F904F903F902F90089588E893E1909353
:109D10004F0E80934E0E80916F008D7F80936F0069
:109D20000E94BCB9882359F00E94BCB98823C1F3B2
:109D300080910D138F5F8F7080930D13F1CF109270
:109D40004D0E10924C0E80916F00826080936F00D8
:109D50008FB7F8941092FA081092FB081092FC0842
:109D60001092FD088FBF0E94A9DF0F949E1886ED08
:109D70009EE00E9445DD0E94F9F70C94D8B62F9220
:109D80003F924F925F926F927F928F929F92AF928B
:109D9000BF92CF92DF92EF92FF920F931F93CF93D8
:109DA000DF93CDB7DEB7C654D1090FB6F894DEBF46
:109DB0000FBECDBF85E40E94AAB8882321F00E947F
:109DC00014B84B0102C0812C912C83E40E94AAB8E4
:109DD000882321F00E9414B868A302C045E048A37C
:109DE00085E50E94AAB8882319F00E9435B803C0FF
:109DF00085E50E947BB88CA797FC07C0C12CD12CAD
:109E000026E1E22E23E4F22E06C0C12CD12C9CE8E0
:109E1000E92E92E4F92E83E50E94AAB8882321F066
:109E20000E9444B86B017C018114910411F41092DA
:109E30004C07182D69DD2B013C0187FE0DC080E029
:109E400090E0A0E0B1E421968CAF9DAFAEAFBFAF84
:109E500021978CE3B82E0CC020E030E040E551E4BF
:109E600021962CAF3DAF4EAF5FAF219704E1B02EEE
:109E700081E0880D823028F4BAE48B2EB3E09B2E6B
:109E800026C00DE513E0D8018D918D01882319F0CE
:109E90000E944961F8CF8AE0CA5BDF4F0FB6F894A1
:109EA000DEBF0FBECDBFDF91CF911F910F91FF900D
:109EB000EF90DF90CF90BF90AF909F908F907F906A
:109EC0006F905F904F903F902F900C944961F401F8
:109ED00081914F01882319F00E944961F8CF8AE0EF
:109EE0000E9449610E94B07617FF04C08FE78093FB
:109EF0004B0708C0E12F012E000CFF0BE65BF84F6B
:109F00008FE78083C701B6010F94C52F072E000C81
:109F1000880B990B0F941D2A062F79878A879B87B8
:109F20002B2D30E0A8EEB3E00F94712E6DA77EA725
:109F30008FA798AB9B01AC01240D351D461D571D05
:109F400029AF3AAF4BAF5CAF81E080931A024CA2CD
:109F50005DA26EA27FA249AA5AAA6BAA7CAA1BA2E2
:109F60001DAA1EAA1FAA18AE1E8A30E43F8B4CE120
:109F7000488F56E4598F1A8E1B8E1C8E1D8E1A8A9E
:109F80001B8A1C8A1D8A1E861F86188A198AC12C64
:109F9000D12C7601FFE78F2E912CA12CB12C8FE7CD
:109FA00090E0A0E0B0E08D839E83AF83B88718A6D1
:109FB00019A61AA61BA691E09AA31D861C86212C21
:109FC000312C26961FAE269727961FAE2797812FF6
:109FD000012E000C990BDC01A65BB84F2396BFAF96
:109FE000AEAF2397880F991F880F991FFC01E85285
:109FF000F74FFF8FEE8F28A1022E000C330B39A3F1
:10A0000028A380911A02882309F4ECC07DDC6983BF
:10A010007A838B839C8380913907882309F4C3C09A
:10A020000E9416BE17FF0FC020904D0730904E07BC
:10A0300030914F0726963FAF2697409150072796BD
:10A040004FAF279711C0AE8DBF8D2C9011963C90CD
:10A0500011971296BC912696BFAF2697EE8DFF8D75
:10A06000F3812796FFAF2797910126964FAD26974C
:10A0700027965FAD27976A8D7B8D8C8D9D8D0F9474
:10A08000172A87FF0AC02A8E3B8E26962FAD269769
:10A090002C8F27963FAD27973D8F910126964FAD88
:10A0A000269727965FAD27976E897F89888D998D32
:10A0B0000F94A730181654F42E8A3F8A26964FAD77
:10A0C0002697488F27965FAD2797598F8AA1202F13
:10A0D00039854A855B85B101882309F446C02696F7
:10A0E0008FAD269727969FAD27970F94A730181608
:10A0F0000CF059C049815A816B817C814419550902
:10A1000066097709DB01CA0188589341A109B109A1
:10A11000B7FD49C08D819E81AF81B88588199909A5
:10A12000AA09BB09B595A7959795879517FF03C011
:10A1300080934B0705C02396EEADFFAD2397808338
:10A1400048A759A76AA77BA70A8FF985FB8F2A859D
:10A150002C8F3B853D8F89819A81AB81BC818CA3FB
:10A160009DA3AEA3BFA31AA21EC026968FAD2697AD
:10A1700027969FAD27970F94172A87FF14C08981D0
:10A180009A81AB81BC812CA13DA14EA15FA1821B14
:10A19000930BA40BB50BAC01BD01485853416109A9
:10A1A000710977FFB6C120E030E040EA51E4602F4A
:10A1B00079858A859B850F94812E9B01AC01B10125
:10A1C00026968FAD269727969FAD27970F94A73099
:10A1D00018163CF5E4E1F8E084918F010F5F1F4F02
:10A1E00081111BC0CA5BDF4F0FB6F894DEBF0FBEF4
:10A1F000CDBFDF91CF911F910F91FF90EF90DF9036
:10A20000CF90BF90AF909F908F907F906F905F9016
:10A210004F903F902F900C94B0760E944961F801C6
:10A22000DBCF89819A81AB81BC8129A93AA94BA94D
:10A230005CA9821B930BA40BB50BB7FD93C00E94C6
:10A2400078748AE00E94496189819A81AB81BC81DE
:10A250008053984FAF4FBF4F89AB9AABABABBCAB02
:10A260009BA1911161C02DA93EA94FA958ADB10183
:10A2700026968FAD269727969FAD27970F94A730E8
:10A2800018160CF03EC021962CAD3DAD4EAD5FAD25
:10A290002197602F79858A859B850F94802E9B015D
:10A2A000AC01A1E0ABA3B10126968FAD269727960E
:10A2B0009FAD27970F94A73018160CF01BA220E033
:10A2C00030E040E050E4B10126968FAD2697279606
:10A2D0009FAD27970F94812E6DAB7EAB8FAB98AF60
:10A2E00029813A814B815C818DA59EA5AFA5B8A936
:10A2F000280F391F4A1F5B1F29AF3AAF4BAF5CAF26
:10A3000031C089819A81AB81BC8129AD3AAD4BAD19
:10A310005CAD821B930BA40BB50BB7FD23C046EFBE
:10A3200057E065E078E01BC020E030E040EA51E40F
:10A33000602F79858A859B850F94802E9B01AC01C7
:10A34000B10126968FAD269727969FAD27970F943C
:10A35000172A87FF07C046ED57E066EE77E0812FAA
:10A360000E9439BE89819A81AB81BC81880F991F77
:10A37000AA1FBB1F2CA13DA14EA15FA1821B930B65
:10A38000A40BB50B84199509A609B70981389F4418
:10A39000A241B10568F0E8EBF7E084918F010F5F0F
:10A3A0001F4F882309F41ECF0E944961F801F5CFA1
:10A3B0004C855D8588A199A1841795070CF0A6C0EE
:10A3C000EBE5F7E084915F019FEFA91AB90A8823B2
:10A3D00021F00E944961F501F5CF17FD05C09DEC04
:10A3E000A92E93E0B92E04C086E4A82E83E0B82EEF
:10A3F000B50189E497E00E94D9A5B701A60185E4DB
:10A4000097E00E94A3A58AE00E944961B50183E319
:10A4100097E00E94D9A54E855F85688979898FE28A
:10A4200097E00E94A3A58AE00E944961B5018DE1F1
:10A4300097E00E94D9A54A895B896C897D8989E169
:10A4400097E00E94A3A58AE00E944961ACA5AA23D7
:10A4500009F4C7C117FF2DC0C0926C0ED0926D0ECB
:10A46000E0926E0EF0926F0E2CEA35EC47E25EE35E
:10A470006E857F85888999890F947C2A6093680E00
:10A480007093690E80936A0E90936B0E2CEA35ECF4
:10A4900047E25EE36A897B898C899D890F945D2FF1
:10A4A0006093640E7093650E8093660E9093670EB2
:10A4B00098C1C092780ED092790EE0927A0EF09206
:10A4C0007B0E2CEA35EC47E25EE36E857F8588895A
:10A4D00099890F947C2A6093740E7093750E809303
:10A4E000760E9093770E2CEA35EC47E25EE36A89AC
:10A4F0007B898C899D890F945D2F6093700E70937A
:10A50000710E8093720E9093730E6BC10E94D0AB4C
:10A5100078CD4C855D85452B09F439C148A459A4F3
:10A520006AA47BA4480E591E6A1E7B1E28A539A565
:10A530004AA55BA5281B390B4A0B5B0BCA01B90165
:10A54000A50194010F94142EA30192010F94452E9E
:10A550008D809E80AF80B884820E931EA41EB51E8F
:10A5600034E183169104A104B1040CF14CEE84167D
:10A570009104A104B1043CF450E885169104A104AF
:10A58000B10434F422C05BEE852E912CA12CB12CA9
:10A590008D829E82AF82B8868EEF90E0A0E0B0E020
:10A5A00088199909AA09BB094C015D0112C024E16F
:10A5B00030E040E050E02D833E834F83588744E1F4
:10A5C000842E912CA12CB12C04C08D829E82AF824E
:10A5D000B886E0E8F8E084919F012F5F3F4F882321
:10A5E00081F024962FAF249725963FAF25970E94A0
:10A5F000496124962FAD249725963FAD2597F90103
:10A60000EACF6D817E818F8198850E940862EBE799
:10A61000F8E084919F012F5F3F4F882381F02496BB
:10A620002FAF249725963FAF25970E944961249626
:10A630002FAD249725963FAD2597F901EACFC501A7
:10A64000B4010E9408624E895F89688D798D84E724
:10A6500098E00E94A3A54A8D5B8D6C8D7D8D8DE663
:10A6600098E00E94A3A54C855D85433051050CF40C
:10A670008EC0C501B4010F941D2A20E030E040E8EF
:10A6800050E40F947C2A6B017C012E893F89488D10
:10A69000598D6A8D7B8D8C8D9D8D0F94802E2BED29
:10A6A0003FE049E450E40F947C2A20E030E040E0B1
:10A6B0005FE30F947C2A9B01AC01C701B6010F94A4
:10A6C0005D2F6B017C01C301B2010F941D2A2FE69F
:10A6D00032E143E85AE30F947C2A2B013C01B70195
:10A6E000A60187E698E00E94A3A5B301A20181E636
:10A6F00098E00E94A3A52AE939E949E15FE3C7018F
:10A70000B6010F947C2A6B017C019B01AC010F9474
:10A71000812EA30192010F945D2F6E877F87888B16
:10A72000998BA3019201C701B6010F947C2A20E006
:10A7300030E040E05EE30F947C2A6A8B7B8B8C8B4D
:10A740009D8BE1E5F8E084913F015FEF651A750AA2
:10A75000882321F00E944961F301F5CFB701A601DA
:10A760008BE498E00E94A3A54E855F85688979896E
:10A7700085E498E00E94A3A54A895B896C897D895C
:10A780008FE398E00E94A3A58AE00E9449618D8131
:10A790009E81AF81B885880D991DAA1DBB1DB595F9
:10A7A000A7959795879517FF03C080934B0705C022
:10A7B0002396EEADFFAD239780832C853D852F5FDB
:10A7C0003F4F3D872C870E8B39853F8B4A85488FBD
:10A7D0005B85598F49805A806B807C8081E08AA399
:10A7E000E2CCCA5BDF4F0FB6F894DEBF0FBECDBF21
:10A7F000DF91CF911F910F91FF90EF90DF90CF905D
:10A80000BF90AF909F908F907F906F905F904F9090
:10A810003F902F900895CF93DF9383E50E947BB8FC
:10A82000C82F882371F00E9444B80F94C52F7093ED
:10A830002A026093290221E0672B09F020E020938F
:10A84000DC0880E50E947BB8882359F0209129021A
:10A8500030912A02232B11F00E9435B88093DC0836
:10A860002DC0C1112BC0EEE4FBE28491EF012196D3
:10A87000882321F00E944961FE01F7CF8091DC0816
:10A88000811103C066E873E002C069E373E086E00B
:10A8900097E00E94D9A56091290270912A0285EF64
:10A8A00096E00E94C0A5E1EFF6E08491EF012196C9
:10A8B000882321F00E944961FE01F7CFDF91CF91FB
:10A8C0000895CF93DF9380E50E947BB8882351F0F1
:10A8D0000E9444B860936C0E70936D0E80936E0E60
:10A8E00090936F0E89E40E947BB8882381F00E94C8
:10A8F00044B82CEA35EC47E25EE30F947C2A60937F
:10A90000680E7093690E80936A0E90936B0E84E4C8
:10A910000E947BB8882381F00E9444B82CEA35EC71
:10A9200047E25EE30F945D2F6093640E7093650EB3
:10A930008093660E9093670EEEE4FBE28491EF0144
:10A940002196882321F00E944961FE01F7CF4091B2
:10A950006C0E50916D0E60916E0E70916F0E8DEEBB
:10A9600096E00E94A3A52CEA35EC47E25EE36091F5
:10A97000680E7091690E80916A0E90916B0E0F9423
:10A980005D2FAB01BC0189EE96E00E9486A52CEA02
:10A9900035EC47E25EE36091640E7091650E809144
:10A9A000660E9091670E0F947C2AAB01BC0185EE78
:10A9B00096E00E9486A58AE0DF91CF910C944961D0
:10A9C000CF93DF9300D01F92CDB7DEB783E50E940F
:10A9D000AAB8882319F00E9414B802C064E071E09C
:10A9E0007C836B8380E50E94AAB8882339F00E949B
:10A9F00014B8693883E1780730F402C068EE73E078
:10AA00007A83698304C088E893E19A838983BE01CD
:10AA10006D5F7F4FCE0101960E9440F30F900F9023
:10AA20000F900F90DF91CF910895CF92DF92EF9228
:10AA3000FF92CF93DF938AE50E94AAB8811106C0E6
:10AA400083E50E94AAB8882309F47DC00E9444B817
:10AA500020E030E040E050EC0F94172A87FD15C04D
:10AA60000E9444B820E030E040E050E40F94A7306A
:10AA700018162CF00E9444B86B017C010BC0C12C4D
:10AA8000D12CE12C90E4F92E05C0C12CD12CE12C65
:10AA900080ECF82E20910F0F3091100F4091110F84
:10AAA0005091120F80917204882381F0C091330776
:10AAB000D0913407C701B6010F947C2A0F94C52F9B
:10AAC000C60FD71FD0933407C093330780E50E9489
:10AAD0007BB8882321F00E9435B88823A1F1A70113
:10AAE00096016091E30E7091E40E8091E50E9091D5
:10AAF000E60E0F94812E6093E30E7093E40E809324
:10AB0000E50E9093E60EEEE4FBE28491EF012196D0
:10AB1000882321F00E944961FE01F7CF4091E30EA6
:10AB20005091E40E6091E50E7091E60E84ED96E092
:10AB30000E94A3A58AE0DF91CF91FF90EF90DF9074
:10AB4000CF900C944961DF91CF91FF90EF90DF900F
:10AB5000CF900895CF92DF92EF92FF92CF93DF9341
:10AB600080E50E947BB88823C9F10E9414B86B016C
:10AB70007C0183E50E94AAB8882321F00E9414B8C2
:10AB8000EB0102C0CFEFDFEF9E012F5F3F4F23307D
:10AB9000310520F5D7FC22C00E94A9DFCF3F8FEFFF
:10ABA000D80729F0219771F4C1E0D0E00DC08C2DB9
:10ABB0000E94904A31E020E0892B09F030E0C32F59
:10ABC000D22F02C0C0E0D0E08C2D0E94904A8C179A
:10ABD0009D0721F080E00F943116F6CFDF91CF91E1
:10ABE000FF90EF90DF90CF9008950F931F93CF9336
:10ABF000DF938DED90E00E9476B981113BC083E533
:10AC00000E94AAB88823B1F1C0914C07D0E00E94FD
:10AC100014B8CC0FDD1FCD5DDD4F79836883809143
:10AC20004C0790E0EC01CC0FDD1FCC0FDD1F8E0137
:10AC3000055D1D4F880F991FFC01ED5DFD4F608183
:10AC40007181072E000C880B990B0F941D2A2AE0A6
:10AC500037ED43E25CE30F947C2AC054D74F288140
:10AC600039814A815B810F947C2AF801608371836A
:10AC700082839383DF91CF911F910F91089583E594
:10AC80000E94AAB8882331F00E9414B8709302027F
:10AC9000609301020895CF93DF93EEE4FBE2849189
:10ACA000EF012196882321F00E944961FE01F7CF30
:10ACB00083E50E947BB8882321F00E9435B88093F9
:10ACC0000002E4ECF6E08491EF012196882321F064
:10ACD0000E944961FE01F7CF80910002811103C0FB
:10ACE000E0ECF6E002C0ECEBF6E08491EF01219697
:10ACF000882321F00E944961FE01F7CFE4EBF6E0E2
:10AD00008491EF012196882321F00E944961FE0180
:10AD1000F7CF209152183091531840915418509108
:10AD2000551860913C1170913D1180913E119091A8
:10AD30003F110F94812EAB01BC0182EB96E00E9483
:10AD4000A3A520915618309157184091581850914A
:10AD50005918609140117091411180914211909168
:10AD600043110F94812EAB01BC018FEA96E00E9443
:10AD7000A3A520915A1830915B1840915C1850910E
:10AD80005D18609144117091451180914611909128
:10AD900047110F94812EAB01BC018CEA96E00E9412
:10ADA000A3A5E4EAF6E08491EF012196882321F03F
:10ADB0000E944961FE01F7CF20915218309153183B
:10ADC00040915418509155186091390270913A028F
:10ADD00080913B0290913C020F94812EAB01BC010B
:10ADE00082EA96E00E94A3A5209156183091571848
:10ADF000409158185091591860913D0270913E024F
:10AE000080913F02909140020F94812EAB01BC01D2
:10AE10008FE996E00E94A3A520915A1830915B1803
:10AE200040915C1850915D1860914102709142020E
:10AE300080914302909144020F94812EAB01BC019A
:10AE40008CE996E00E94A3A58AE0DF91CF910C9453
:10AE50004961EF92FF920F931F93CF9383E3E82E04
:10AE600083E0F82E04E714E0C0E0F70181917F0150
:10AE70000E947BB8882351F00E9444B8F801608397
:10AE80007183828393838C2F0E949BB3CF5F0C5F6F
:10AE90001F4FC33051F7CF911F910F91FF90EF904B
:10AEA0000C946A6883E50E947BB8882351F00E9465
:10AEB00044B86093A10E7093A20E8093A30E90935A
:10AEC000A40E84E50E947BB8882351F00E9444B808
:10AED00060939D0E70939E0E80939F0E9093A00E94
:10AEE00082E40E947BB8882351F00E9404B86093EA
:10AEF000990E70939A0E80939B0E90939C0E88E50A
:10AF00000E947BB8882351F00E9444B86093890E58
:10AF100070938A0E80938B0E90938C0E89E50E941D
:10AF20007BB8882351F00E9444B860938D0E7093D3
:10AF30008E0E80938F0E9093900E8AE50E947BB8C0
:10AF4000882351F00E9444B86093910E7093920E42
:10AF50008093930E9093940E85E40E947BB888238F
:10AF600051F00E9444B86093950E7093960E8093B2
:10AF7000970E9093980E08950F931F93462F50E0CD
:10AF800060E070E022E0440F551F661F771F2A958E
:10AF9000D1F74470552766277727FC010385148570
:10AFA000258536850B7F402B512B622B732B4387D6
:10AFB000548765877687AC01455F5F4F60E81F91D6
:10AFC0000F910D94821DCF92DF92EF92FF920F931B
:10AFD0001F93AC014D5A5F4F062F10E020E030E088
:10AFE000980111270027002711272F773327FA010F
:10AFF000C080D180E280F380F0E8EF220C291D2987
:10B000002E293F29FA0100831183228333836DEEB9
:10B010001F910F91FF90EF90DF90CF900D94821DC4
:10B02000CF93DF931F92CDB7DEB7789484B582605B
:10B0300084BD84B5816084BD85B5826085BD85B5DC
:10B04000816085BD80916E00816080936E0010925A
:10B0500081008091810082608093810080918100D5
:10B060008160809381008091800081608093800066
:10B070008091B10084608093B1008091B0008160C4
:10B080008093B000809191008260809391008091C4
:10B090009100816080939100809190008160809305
:10B0A00090008091A10082608093A1008091A10016
:10B0B00081608093A1008091A00081608093A000B6
:10B0C0008091210182608093210180912101816022
:10B0D00080932101809120018160809320018091E3
:10B0E0007A00846080937A0080917A0082608093F5
:10B0F0007A0080917A00816080937A0080917A0052
:10B10000806880937A001092C10082E08093C00032
:10B110001092C50087E08093C4008091C1008061D7
:10B120008093C1008091C10088608093C1008091AC
:10B13000C10080688093C1008091C1008F7D8093A1
:10B14000C10010926504EEE4FAE084918F010F5F74
:10B150001F4F882321F00E944961F801F6CFEEE4E9
:10B16000FBE284918F010F5F1F4F882321F00E9423
:10B170004961F801F6CF14B710FF0DC0E5E4FAE01D
:10B1800084917F019FEFE91AF90A882321F00E9438
:10B190004961F701F5CF11FF0DC0E4E3FAE08491B6
:10B1A0007F019FEFE91AF90A882321F00E94496183
:10B1B000F701F5CF12FF0DC0E2E2FAE084917F01C2
:10B1C0009FEFE91AF90A882321F00E944961F701EB
:10B1D000F5CF13FF0DC0E1E1FAE084917F019FEF0D
:10B1E000E91AF90A882321F00E944961F701F5CF95
:10B1F00015FF0CC0E0E0FAE084918F010F5F1F4F54
:10B20000882321F00E944961F801F6CF14BEE9EFCE
:10B21000F9E084918F010F5F1F4F882321F00E9476
:10B220004961F801F6CF80E20E944961E2EFF9E05E
:10B2300084918F010F5F1F4F882321F00E94496185
:10B24000F801F6CF8AE00E944961EEE4FBE28491C6
:10B250008F010F5F1F4F882321F00E944961F80181
:10B26000F6CFE2EEF9E084918F010F5F1F4F882344
:10B2700021F00E944961F801F6CFEEECF9E08491EB
:10B280008F010F5F1F4F882321F00E944961F80151
:10B29000F6CFE5E9F9E084918F010F5F1F4F882316
:10B2A00019F0F7D7F801F7CFEEE4FBE284918F01B4
:10B2B0000F5F1F4F882319F0ECD7F801F7CFEEE7A7
:10B2C000F9E084918F010F5F1F4F882319F0E1D7B8
:10B2D000F801F7CFEEE4FBE284918F010F5F1F4F7F
:10B2E000882319F0D6D7F801F7CF80915E18909196
:10B2F0005F18BE016F5F7F4F009719F0681B790BD5
:10B3000002C0645678418FE699E00E94C0A560E2D1
:10B3100075E088E599E00E94C0A58AE0BAD781E08F
:10B3200080938004809381048093820480938304BB
:10B33000809384040F94BA0C8CE0E4E7F4E0A7EF68
:10B34000BEE001900D928A95E1F70E94D8B66D9A01
:10B350009D9A8091010180628093010188E00F94A1
:10B3600056258091010188608093010186E00F9449
:10B37000562587ED80937A0010927E0010927D0012
:10B3800080917E00816080937E0080917E00846049
:10B3900080937E0080E888BD80916E0084608093F9
:10B3A0006E006AEF70E080E090E00E944C4C85E017
:10B3B00090E090936B0480936A0460E080911602A1
:10B3C000909117020E94D07320E030E040EA50E4F0
:10B3D0000F94172A87FF0AC08091160290911702D6
:10B3E00040979093170280931602E7CF81E391E094
:10B3F000909319028093180260E080916804909104
:10B4000069040E94D07320E030E848E953E40F94C7
:10B41000A730181654F480916804909169044096FE
:10B420009093690480936804E7CF8091140290910F
:10B4300015020E9477BD20E030E040EA50E40F940E
:10B44000172A87FF0AC08091140290911502409735
:10B450009093150280931402E8CF80916604909136
:10B4600067040E9477BD20E030E046E153E40F948A
:10B47000A730181654F480916604909167044096A2
:10B480009093670480936604E8CF98E288E10FB652
:10B49000F894A895809360000FBE9093600080910F
:10B4A0000A01886080930A0180910A01806180937B
:10B4B0000A0180910A01806280930A010E944EDF96
:10B4C00080912101887F816080932101E090070FA6
:10B4D000F090080F0091090F10910A0F28E430E056
:10B4E00040E050E060E170E08DE694E169D5E090E5
:10B4F0000B0FF0900C0F00910D0F10910E0F28E420
:10B5000030E040E050E060E170E088EF93E158D532
:10B51000E0900F0FF090100F0091110F1091120F8B
:10B5200023E030E040E050E060E270E083E893E147
:10B5300047D5E090130FF090140F0091150F109164
:10B54000160F2EE130E040E050E060E170E08EE068
:10B5500093E136D561E08DE694E10F94961E61E0AB
:10B5600088EF93E10F94961E61E08DE694E10F94CD
:10B57000291F61E088EF93E10F94291F64E08DE6B5
:10B5800094E10F94F91E64E088EF93E10F94F91EA3
:10B5900060E08DE694E10F94C61E60E088EF93E1D1
:10B5A0000F94C61E61E083E893E10F94291F60E0C9
:10B5B00083E893E10F94F91E60E083E893E10F9430
:10B5C000C61E61E083E893E10F94961E64E083E871
:10B5D00093E1F9DC61E083E893E1CEDC40E050E008
:10B5E000BA0183E893E10F94651F60E083E893E17B
:10B5F0000F94541E60E083E893E10F94271E61E0EE
:10B6000083E893E10F94291F60E083E893E10F94AE
:10B61000F91E60E083E893E10F94C61E61E083E8C1
:10B6200093E10F94961E60E08EE093E1A5DC4FEF6E
:10B630005FEF6FE070E08EE093E10F94651F61E0D3
:10B640008EE093E10F94541E63E08EE093E10F943B
:10B65000271E80910A01816080930A0180910A016E
:10B66000826080930A0180910A01846080930A01BC
:10B6700080910A01806480930A010F9A179A0E9AAA
:10B68000169A0D9A159A0C9A149A809107018B7F3D
:10B69000809307019FB7F89480910801846080939C
:10B6A00008019FBF24982C9A809107018F7780937F
:10B6B00007019FB7F8948091080180688093080182
:10B6C0009FBF809101018F7E809301019FB7F89405
:10B6D000809102018061809302019FBF389A409857
:10B6E000179A10927004399A4198169A1092710420
:10B6F0003A9A4298159A109272043B9A4398149A77
:10B70000809180008C7F8093800080918100877E73
:10B71000886080938100809180008F738093800087
:10B7200080918100887F82608093810080E090E436
:10B730009093890080938800109285001092840075
:10B7400080916F00826080936F0010926F0410925E
:10B750006E0410926D0410926C0481E080934C187A
:10B7600078940E94B8DF1092730480910101886080
:10B77000809301010E94B3AF0F94421420911118DD
:10B7800030E0790188E3E81AF108F7FE04C0790196
:10B7900097E3E91AF108F594E7942E5131093695AB
:10B7A0002795F22E0F943C0403ED18E023E147E0C7
:10B7B0006CE08E2D0F94781B84E00F947D14009123
:10B7C000111810E00257110916950795609112188B
:10B7D00062514AE853E08F2D0F94F51B60911218C7
:10B7E000665040E953E0802F0F94F51B0F943E1BE9
:10B7F0008111DACF64EC79E080E090E00E946798F4
:10B80000159840E6542E5DE0452E6CE6C62E6AE0A3
:10B81000D62E70E0A72E70E0B72E2AE0722E30E20E
:10B82000632E80918306853010F40E9456B4809177
:10B8300005188823F1F00E94844C009101181091A2
:10B8400002182091031830910418DC01CB01801BF1
:10B85000910BA20BB30BB7FD0CC010920518809191
:10B860005B1581110BC10E94BAF180915B158111AA
:10B8700005C180918306882309F494C080915815EE
:10B88000882309F47CC000918206509E8001112417
:10B890000E551B4F6FEA7AE0C8010F949629892B49
:10B8A000E9F08CE497E186D78CE497E10E949A6FE7
:10B8B0001092591510925815ECE9FAE084918F0115
:10B8C0000F5F1F4F882339F0E4D4F801F7CF809140
:10B8D0005915811154C00F94BA1853C0F801019042
:10B8E0000020E9F731977F01E01AF10A10924C1716
:10B8F0006EE470E0C8010F94C6314C01009729F442
:10B90000F7013197E00FF11F0EC060E270E00F9475
:10B91000C6318C010F5F1F4F6AE270E0C4010F94C3
:10B92000C631FC013197418272821382F801019085
:10B930000020E9F73197AF01401B510BB8018CE4AF
:10B9400097E10E94A36480914C17882309F4BFCF2C
:10B95000E3E3FBE284918F010F5F1F4F882319F00F
:10B9600098D4F801F7CFE5E5FAE084918F010F5FF5
:10B970001F4F882309F4ABCF8CD4F801F6CF0F9476
:10B98000521980918306882369F081508093830641
:10B99000809182068F5F853018F48093820602C002
:10B9A000109282068091E20E882309F45DC0EEE4D5
:10B9B000FBE284918F010F5F1F4F882319F069D438
:10B9C000F801F7CFEDE8FAE084918F010F5F1F4F88
:10B9D000882319F05ED4F801F7CF8091E20E80FD44
:10B9E00050C08091E20E84FD4CC090E2F92E80910F
:10B9F000E20E81FD63C08091E20E85FD5FC000E232
:10BA00008091E20E82FD76C08091E20E86FD72C0CA
:10BA100010E28AE03ED41F926F921F921F931F92F2
:10BA20000F931F92FF92DF92CF921F920F944E1DA1
:10BA30001092E20E0FB6F894DEBF0FBECDBF80911C
:10BA40008504882389F010925A158CE497E1B2D6C8
:10BA50008CE497E10E949A6F109259151092581534
:10BA60000E94854E0E94B07680E00F943116A1149A
:10BA7000B10409F4D6CE0E940000CFCE0E9408F196
:10BA8000F8CE6091960470919704809198049091FB
:10BA900099040F941D2A20918604309187044091C7
:10BAA0008804509189040F947C2AAB01BC0189E879
:10BAB0009AE00E94A3A588E5F82E99CF60919A0498
:10BAC00070919B0480919C0490919D040F941D2A79
:10BAD00020918A0430918B0440918C0450918D0404
:10BAE0000F947C2AAB01BC0185E89AE00E94A3A5D3
:10BAF00009E586CF60919E0470919F048091A00417
:10BB00009091A1040F941D2A20918E0430918F04EE
:10BB100040919004509191040F947C2AAB01BC0198
:10BB200081E89AE00E94A3A51AE573CF4F925F9235
:10BB30006F927F92AF92BF92CF92DF92EF92FF927D
:10BB40000F931F93CF93DF93009709F456C0FC0126
:10BB5000208121FD52C0EB018C0144A455A466A4B0
:10BB600077A4ACA4BDA4CEA4DFA49501A601C30113
:10BB7000B2010F94172A87FF40C0A3019201C301AD
:10BB8000B2010F947C2A2B013C01F80180AD91ADEC
:10BB9000A2ADB3ADBC01CD0190589B01AC010F9497
:10BBA000812EF80124A935A946A957A90F947C2A0A
:10BBB0009B01AC01C301B2010F94802E0F94EC30B5
:10BBC0007B018C019B01AC01B501C6010F94172AC2
:10BBD00087FF02C0750186019701A801B501C60162
:10BBE0000F94172A882349F0A701B8014CA75DA735
:10BBF0006EA77FA7888181608883DF91CF911F9195
:10BC00000F91FF90EF90DF90CF90BF90AF907F901B
:10BC10006F905F904F9008952F923F924F925F9256
:10BC20006F927F928F929F92AF92BF92CF92DF924C
:10BC3000EF92FF920F931F93CF93DF93CDB7DEB7B1
:10BC400068970FB6F894DEBF0FBECDBF1C015B0135
:10BC50008A01DC01DC966D917D918D919C91DF973D
:10BC60000F941B2A6B017C01F501208131814281F7
:10BC700053810F947C2A0F94472F0F94CA2F698702
:10BC80007A878B879C87D8012D913D914D915C914E
:10BC9000C701B6010F947C2A0F94472F0F94CA2F27
:10BCA0006D877E878F87988B29853A854B855C8544
:10BCB000283731054105510540F488E790E0A0E0C0
:10BCC000B0E089879A87AB87BC872D853E854F85F5
:10BCD0005889283731054105510540F488E790E03F
:10BCE000A0E0B0E08D879E87AF87B88B9101285B7D
:10BCF0003F4FD9018D919D910D90BC91A02D8D83C9
:10BD00009E83AF83B887BC01CD010F941D2A698340
:10BD10007A838B839C8369857A858B859C850F9438
:10BD20001B2A698B7A8B8B8B9C8B20E030E0A901DE
:10BD300069817A818B819C810F94172A882339F13C
:10BD4000A7019601C701B6010F947C2A4B015C0143
:10BD500029893A894B895C89CA01B9010F947C2AE7
:10BD60009B01AC01C501B4010F94802E4B015C0115
:10BD700029813A814B815C81CA01B9010F94812EDE
:10BD80009B01AC01C501B4010F945D2F03C060E0BD
:10BD900070E0CB010F94472F0F94C52F2B013C016E
:10BDA0006D817E818F819885909580957095619544
:10BDB0007F4F8F4F9F4F0F941D2A4B015C016D8564
:10BDC0007E858F8598890F941B2A6D837E838F8350
:10BDD000988720E030E0A901C501B4010F94172A2B
:10BDE000882349F12D813E814F815885CA01B901CF
:10BDF0000F947C2A6D8B7E8B8F8B988FA701960179
:10BE0000C701B6010F947C2A9B01AC016D897E8924
:10BE10008F89988D0F94802E6B017C01A501940170
:10BE2000C501B4010F94812E9B01AC01C701B6017D
:10BE30000F945D2F03C060E070E0CB010F94F62FEC
:10BE4000F10182889388A488B58875016401C418BB
:10BE5000D508E608F7080F94C52FC61AD70AE80ACE
:10BE6000F90AF7FE6BC020E030E0A90169817A8110
:10BE70008B819C810F94172A882309F447C029815C
:10BE80003A814B815C81CA01B9010F94812E6B010B
:10BE90007C01C501B4010F941B2A9B01AC01C701B1
:10BEA000B6010F947C2A6B017C0129893A894B8960
:10BEB0005C89CA01B9010F947C2A9B01AC01C701BE
:10BEC000B6010F94802E6B017C012D813E814F8144
:10BED0005885CA01B9010F947C2A9B01AC01C701A6
:10BEE000B6010F94812E6B017C0120E030E040E828
:10BEF00050E469817A818B819C810F947C2A9B011B
:10BF0000AC01C701B6010F945D2F03C060E070E083
:10BF1000CB010F94472F0F94C52F2B013C0197FFA6
:10BF200003C0412C512C3201481459046A047B048B
:10BF300010F024013501C12CD12C76018FB7F89473
:10BF4000D1019C9193FD22C0F101468A578A608EEF
:10BF5000718EC40CD51CE61CF71C5A96CD92DD924E
:10BF6000ED92FC925D97E05CFF4F29853A854B8509
:10BF70005C85208331834283538334962D853E85AF
:10BF80004F85588920833183428353838FBF6896BE
:10BF90000FB6F894DEBF0FBECDBFDF91CF911F91DA
:10BFA0000F91FF90EF90DF90CF90BF90AF909F9058
:10BFB0008F907F906F905F904F903F902F9008955B
:10BFC0004F925F926F927F928F929F92AF92BF92A9
:10BFD000CF92DF92EF92FF920F931F93CF93DF9355
:10BFE000EC016B0149015A01270138010F946F1FC1
:10BFF000FE01ED58FF4F60817181CE010E9431F644
:10C0000080E1C816D10471F1A0F4F2E0CF16D1049A
:10C0100069F128F4C114D10469F568E028C0E4E0AE
:10C02000CE16D10409F1F8E0CF16D10419F565E078
:10C030001EC080E4C816D10499F030F4F0E2CF16A7
:10C04000D104C1F463E013C080E8C816D10431F014
:10C05000C114E1E0DE0671F460E009C061E007C0F0
:10C0600062E005C064E003C066E001C067E0CE01A5
:10C070000F94691E61E0CE010F94961E65E0CE011B
:10C080000F94291FAE01415B5F4FFA0180819181BE
:10C09000A281B381B06180839183A283B3836CEE6C
:10C0A000CE010F94821DAE014D595F4F80E890E0A4
:10C0B000A0E0B0E0FA0180839183A283B38361E9B9
:10C0C000CE010F94821D62E0CE010F94F91E65E04F
:10C0D000CE010F94C61E8B859C85AD85BE859F7E47
:10C0E0008B879C87AD87BE878E01055F1F4FA80198
:10C0F00060E8CE010F94821D8B859C85AD85BE8541
:10C100009F7D8B879C87AD87BE87A80160E8CE01A5
:10C110000F94821D8B859C85AD85BE8591608B8734
:10C120009C87AD87BE87A80160E8CE010F94821D71
:10C130008B859C85AD85BE8580618B879C87AD870F
:10C14000BE87A80160E8CE010F94821D8B859C8577
:10C15000AD85BE858E7F8B879C87AD87BE87A80106
:10C1600060E8CE010F94821D8B859C85AD85BE85D0
:10C170008D7F8B879C87AD87BE87A80160E8CE0145
:10C180000F94821D005B1F4FF80180819181A28175
:10C19000B381AC7F80839183A283B383A80160EFD6
:10C1A000CE010F94821DF80180819181A281B3811B
:10C1B000A46080839183A283B383A80160EFCE0142
:10C1C0000F94821DF80180819181A281B38199270A
:10C1D000956080839183A283B383A80160EFCE0131
:10C1E0000F94821DF80180819181A281B3818F6FAC
:10C1F00080839183A283B383A80160EFCE010F9463
:10C20000821D61E0CE010E94BC57D60120E136E0DC
:10C2100041EC50E00F94612E0F941B2A6B017C01BE
:10C220009A2D892D782D66270F941B2AA301920140
:10C230000F947C2A9B01AC01C701B6010F945D2FBE
:10C240000F94CA2F6F8B788F898F9A8FAE01495EBA
:10C250005F4F63E9CE010F94821DAE01415A5F4FDB
:10C26000FA01108211821282138261E0CE01DF9105
:10C27000CF911F910F91FF90EF90DF90CF90BF90E3
:10C28000AF909F908F907F906F905F904F900D94A4
:10C29000821D91E0909365043FB7F89420912807A0
:10C2A000909129073FBF291304C09091C00095FDCC
:10C2B0003EC0909128079F5F9F712091290792139C
:10C2C00025C00FB607FCF9CF2091C00025FFF5CFA0
:10C2D00020912907E22FF0E0E85FF84F30812F5FCF
:10C2E0002F71209329073093C6002091C00020644D
:10C2F0002093C00030912807209129073213DDCF09
:10C300002091C1002F7D2093C100D7CFE091280755
:10C31000F0E0E85FF84F80832FB7F89490932807F8
:10C320008091C10080628093C1002FBF08959FB7A4
:10C33000F8948093C6008091C00080648093C00010
:10C340009FBF08958F929F92AF92BF92EF92FF92FC
:10C350001F93CF93DF93CDB7DEB7A0970FB6F894B6
:10C36000DEBF0FBECDBF611571058105910579F165
:10C3700010E0842E912CA12CB12CEE24E394F12C0E
:10C38000EC0EFD1EE10EF11C17FDFA94A5019401BF
:10C390000F94232EF7016083B901CA011F5F611555
:10C3A00071058105910549F7115010F1E1E0F0E0C8
:10C3B000EC0FFD1FE10FF11D17FDFA9580818A300A
:10C3C00010F097E301C090E3890F63DFEDCF80E3C6
:10C3D000A0960FB6F894DEBF0FBECDBFDF91CF9110
:10C3E0001F91FF90EF90BF90AF909F908F9051CF93
:10C3F000A0960FB6F894DEBF0FBECDBFDF91CF91F0
:10C400001F91FF90EF90BF90AF909F908F900895F5
:10C41000CF92DF92EF92FF926B017C0197FF0AC0EF
:10C420008DE237DFF094E094D094C094C11CD11C0D
:10C43000E11CF11C4AE0C701B601FF90EF90DF90CC
:10C44000CF9080CF8F929F92AF92BF92CF92DF9288
:10C45000EF92FF92CF936B017C01B42E20E030E08D
:10C46000A9010F94172A87FF06C08DE212DFF7FAA1
:10C47000F094F7F8F094C0E060E070E080E09FE3B3
:10C48000CB1541F02DEC3CEC4CEC5DE30F947C2A99
:10C49000CF5FF6CF9B01AC01C701B6010F94812E8F
:10C4A0006B017C010F94CA2F4B015C014AE04ADF0B
:10C4B000CC2379F1C501B4010F941B2A9B01AC0177
:10C4C000C701B6010F94802E6B017C018EE2E1DE84
:10C4D00020E030E040E251E4C701B6010F947C2A2D
:10C4E0004B015C010F94C52F6B01770FEE08FF081D
:10C4F000C701B6018DDFC701B6010F941D2A9B014C
:10C50000AC01C501B4010F94802E6B017C01C150B8
:10C51000F9F6CF91FF90EF90DF90CF90BF90AF9062
:10C520009F908F9008958FB7F8949091070720916E
:10C530000607291759F0E92FF0E0EA57F94F208153
:10C5400030E09F5F9F779093070702C02FEF3FEF88
:10C550008FBFC90108951F920F920FB60F92112439
:10C560000BB60F922F933F934F935F936F937F93ED
:10C570008F939F93AF93BF93EF93FF93E091060741
:10C5800081E08E0F8F779091C60020910707821768
:10C5900031F0F0E0EA57F94F90838093060720913D
:10C5A0008506422F50E04C30510508F046C0FA0194
:10C5B0008827EA56FF4F8F4F0D947C319D3441F010
:10C5C0009E34B9F481E005C09A3330F09D3471F5A2
:10C5D00082E08093850646C0903308F043C09032D5
:10C5E00009F440C09D3211F53DC0913329F09433D8
:10C5F00029F09032D9F436C083E0EBCF88E0E9CF60
:10C60000903321F0913391F486E0E3CF84E0E1CFE1
:10C61000983361F485E0DDCF923341F487E0D9CFE0
:10C62000913321F489E0D5CF903311F08BE0D1CF55
:10C630008AE0CFCF9A30B1F413C09A3099F4273002
:10C6400049F02A3059F0253059F410921A0210920C
:10C65000840606C083EB9AE00F9475150E94854E00
:10C6600010928506FF91EF91BF91AF919F918F91AD
:10C670007F916F915F914F913F912F910F900BBEE2
:10C680000F900FBE0F901F9018951F920F920FB62C
:10C690000F9211240BB60F928F939F93EF93FF93FA
:10C6A00080912907E82FF0E0E85FF84F90818F5FD5
:10C6B0008F71809329079093C6008091C000806499
:10C6C0008093C0009091280780912907981305C096
:10C6D0008091C1008F7D8093C100FF91EF919F9168
:10C6E0008F910F900BBE0F900FBE0F901F9018955B
:10C6F000DF92EF92FF920F931F93CF93DF937C0112
:10C70000EB018A018DE0D82E40E250E0BE01C70166
:10C710000E94236E8032910539F021E0892B09F4C3
:10C7200020E0822F81953EC02881222399F1253E69
:10C7300059F32E3249F30115110541F13B853F7341
:10C740003F3021F54A8D5B8D452B01F52F713FEF71
:10C75000320F3530D8F430E021503109D29EC0017B
:10C76000D39E900D1124D801A80FB91FFE0120E01F
:10C77000AD01253088F431813D932F5F32962D3005
:10C78000C1F7288126FF02C0FA0115862B8523FDFB
:10C79000BBCF08C080E006C02B3010F43481ECCF52
:10C7A0003681EACFDF91CF911F910F91FF90EF90EB
:10C7B000DF900895CF93DF93EC018B81882339F1CB
:10C7C000898187FF20C061E0CE010E94A36FFC0138
:10C7D000892BE9F08081853ED1F08B81823040F455
:10C7E00089899A89AB89BC89848F958FA68FB78FE9
:10C7F0008D899E89AF89B88D938F828FB58BA48BDD
:10C8000089818F778983DF91CF910D945B2081E0BF
:10C81000888380E0DF91CF9108958F929F92AF92AD
:10C82000BF92CF92DF92EF92FF920F931F93CF931D
:10C83000DF93EC018B81811102C080E077C0098910
:10C840001A892B893C890417150726073707A8F38F
:10C850006A017B01823029F4C886D986EA86FB8684
:10C860000DC0C114D104E104F10451F418861986F5
:10C870001A861B861C821D821E821F8281E056C082
:10C8800088849984AA84BB84E98DFA8D258530E05B
:10C89000275F3F4FB501A40141505109610971095A
:10C8A000022E04C076956795579547950A94D2F75E
:10C8B000D701C6010197A109B10904C0B695A79592
:10C8C000979587952A95D2F784179507A607B707F6
:10C8D00020F089288A288B2849F44D895E896F8940
:10C8E000788D4C835D836E837F8304C0841B950B9E
:10C8F000A60BB70B4C015D018E010C5F1F4F81141D
:10C900009104A104B10409F4A7CF4C815D816E812B
:10C910007F819801898D9A8D0F94642191E0891A05
:10C920009108A108B1088111EACF87CFDF91CF919B
:10C930001F910F91FF90EF90DF90CF90BF90AF903D
:10C940009F908F9008952F923F924F925F926F9297
:10C950007F928F929F92AF92BF92CF92DF92EF928F
:10C96000FF920F931F93CF93DF9300D01F92CDB709
:10C97000DEB78C014B011A01DC0113968C911397E1
:10C980008130C1F411968C9181FF14C082FF18C0D0
:10C99000F801418952896389748980859185A285CE
:10C9A000B38584179507A607B70751F0C80135DF8F
:10C9B000811106C081E0F80180838FEF9FEF2FC1C6
:10C9C000610185C0D80159968D919C915A97FC01BF
:10C9D000248121502A013B0139E0769467945794D1
:10C9E00047943A95D1F7722E74207A01F1E0FF2234
:10C9F000772009F478C080E092E08E199F095601F3
:10CA00008C159D0508F45C01D80159962D913C9137
:10CA10005A9714968D919D910D90BC91A02D0297DF
:10CA2000A109B109F901058404C0880F991FAA1F43
:10CA3000BB1F0A94D2F74685578560897189840F98
:10CA4000951FA61FB71F9C01AD01270D311D411D6C
:10CA5000511D29013A01A11432E0B30609F08AC040
:10CA60008091311190913211A0913311B091341114
:10CA700084159505A605B70569F4109239118FEF55
:10CA80009FEFDC018093311190933211A093331109
:10CA9000B09334119401B301A20180913A119091A5
:10CAA0003B110E945495882309F484CFF8018085B6
:10CAB0009185A285B3858A0D9B1DA11DB11D80871F
:10CAC0009187A287B3878A0C9B1CCA18DB08D80100
:10CAD00018964D915D916D917C911B97C114D10475
:10CAE00009F070CF7DC0E114F10409F084CF1496F1
:10CAF0004D915D916D917C9117974115510561059F
:10CB0000710559F455968D919D910D90BC91A02D74
:10CB10000097A105B10541F521C09E012F5F3F4F50
:10CB20000F946421882309F445CF89819A81AB81D0
:10CB3000BC81F801218D328DF9012789203139F42A
:10CB4000883FFFEF9F07A105B10540F40DC0883F66
:10CB50002FEF9207A2072FE0B20730F0C8010E9422
:10CB6000F26F811148CF26CFF80184839583A68385
:10CB7000B78341CFE114F10419F5D80118964D910E
:10CB80005D916D917C911B9751968D919D910D902A
:10CB9000BC91A02D481759076A077B0788F00F94AE
:10CBA0005B20882309F406CF81E0809339114092FD
:10CBB000311150923211609233117092341108C0C9
:10CBC00041E0C301B2010F949B20882309F4F2CE07
:10CBD000A501B401C7018F5C904F0F949F3166CFC0
:10CBE00051968D919D910D90BC91A02D8417950724
:10CBF000A607B70740F4F801418B528B638B748B07
:10CC0000818180688183D80111968C9183FD02C057
:10CC1000C10105C0C801CEDD8111FACFCBCE0F9086
:10CC20000F900F900F90DF91CF911F910F91FF9078
:10CC3000EF90DF90CF90BF90AF909F908F907F90BC
:10CC40006F905F904F903F902F900895EF92FF92DA
:10CC50000F931F93CF93DF931F92CDB7DEB7082FAB
:10CC6000162FEFE3FBE084917F012FEFE21AF20A27
:10CC7000882329F099830DDBF7019981F4CFE02F08
:10CC8000F92F84917F019FEFE91AF90A882319F09F
:10CC900000DBF701F6CFEDE3FBE084917F012FEF9E
:10CCA000E21AF20A882319F0F4DAF701F6CF612FBD
:10CCB00070E080E090E0ACDB8AE00F90DF91CF91F4
:10CCC0001F910F91FF90EF90E4CA83E50E947BB81B
:10CCD0008823D1F00E9444B8AB01BC014093AD0E53
:10CCE0005093AE0E6093AF0E7093B00E4093A50EAE
:10CCF0005093A60E6093A70E7093A80E81E59DE059
:10CD00000E94A3A58AE0C5DA80E50E947BB888234B
:10CD100091F00E9444B8AB01BC014093AD0E50931A
:10CD2000AE0E6093AF0E7093B00E84E39DE00E9450
:10CD3000A3A58AE0AEDA82E50E947BB8882391F051
:10CD40000E9444B8AB01BC014093A90E5093AA0EB7
:10CD50006093AB0E7093AC0E85E19DE00E94A3A59D
:10CD60008AE097DA84E50E947BB8882391F00E94DC
:10CD700044B8AB01BC014093A50E5093A60E60933E
:10CD8000A70E7093A80E87EF9CE00E94A3A58AE0EF
:10CD900080CA0895FF920F931F93CF93DF9301EC06
:10CDA0001EE0C3E3D3E0FC2E84E0F80E89910E94DC
:10CDB0007BB8882339F00E9444B8F80160837183FE
:10CDC000828393830C5F1F4FFC12F0CFDF91CF91D2
:10CDD0001F910F91FF900895FF920F931F93CF9390
:10CDE000DF9301EB1EE0C3E3D3E0FC2E84E0F80EFA
:10CDF00089910E947BB8882349F00E9444B80F941F
:10CE0000CA2FF80160837183828393830C5F1F4F65
:10CE1000FC12EECFDF91CF911F910F91FF900C94F8
:10CE200058E9CF9388EC90E00E9476B9811140C018
:10CE300084E40E947BB88823C1F10E9444B8C1E019
:10CE400020E030E0A9010F94172A811101C0C0E051
:10CE5000C093D50ECC2349F10E9444B8E0914C0711
:10CE600024E0E29FF0011124EF52F14F60837183BF
:10CE70008283938320E030E0A9016091D10E70910C
:10CE8000D20E8091D30E9091D40E0F94172A811157
:10CE90000CC080E090E0A0E4B0E48093D10E9093C9
:10CEA000D20EA093D30EB093D40ECF910C94E9DEA2
:10CEB000CF9108950F93CF93DF93CDB7DEB76497EB
:10CEC0000FB6F894DEBF0FBECDBF8CE40E947BB8D6
:10CED000882319F00E9444B804C060E070E080E04C
:10CEE00090EC6D877E878F87988B80E090E0A0E242
:10CEF000B1E489839A83AB83BC8380E090E0A6E3AE
:10CF0000B3E48D839E83AF83B88780E090E0A0EA8E
:10CF1000B1E489879A87AB87BC8788E50E94AAB865
:10CF2000882379F088E50E94AAB8882319F00E9426
:10CF300044B803C060E070E0CB0169837A838B83DF
:10CF40009C8389E50E94AAB8882379F089E50E942C
:10CF5000AAB8882319F00E9444B803C060E070E0CA
:10CF6000CB016D837E838F8398878AE50E94AAB860
:10CF7000882379F08AE50E94AAB8882319F00E94D4
:10CF800044B803C060E070E0CB0169877A878B8783
:10CF90009C87198A1A8A1B8A1C8A80912F08811102
:10CFA0000CC000E020E0AE014F5E5F4FBE016F5F3E
:10CFB0007F4FCE010D960E94ACC264960FB6F894D6
:10CFC000DEBF0FBECDBFDF91CF910F910895CF93FC
:10CFD000DF9385E40E94AAB8882319F00E9435B82F
:10CFE00003C085E40E947BB8882351F0EEE4FBE2A5
:10CFF0008491EF012196882319F04BD9FE01F8CFD7
:10D0000081E40E94AAB8882319F00E9435B803C0B1
:10D0100081E40E947BB8882351F0E3EFFCE0849127
:10D02000EF012196882319F034D9FE01F8CFC09181
:10D030006D08D0916E088991882311F02AD9FBCF11
:10D040008AE0DF91CF9125C9CF93DF93EBEFFBE02F
:10D050008491EF012196882319F01BD9FE01F8CFA6
:10D0600060E08BEE9BE0F2DD61E084EE9BE0EEDDC4
:10D0700061E089ED9BE0EADD61E089EC9BE0E6DDC3
:10D0800060E080EC9BE0E2DD61E086EB9BE0DEDDD2
:10D0900061E08CEA9BE0DADD61E084EA9BE0D6DDCA
:10D0A00061E086E99BE0D2DD61E088E89BE0CEDDCF
:10D0B00060E089E79BE0CADD60E08BE69BE0C6DDCF
:10D0C00060E085E59BE0C2DD61E084E49BE0DF9108
:10D0D000CF91BCCD4F925F926F927F928F929F9231
:10D0E000AF92BF92CF92DF92EF92FF92CF93DF93F6
:10D0F000EAE3FBE08491EF012196882319F0C9D877
:10D10000FE01F8CF209152183091531840915418D5
:10D11000509155186091F70E7091F80E8091F90EAC
:10D120009091FA0E0F94812E42E08CD9E6E3FBE059
:10D130008491EF012196882319F0ABD8FE01F8CF36
:10D1400020915618309157184091581850915918FD
:10D150006091FB0E7091FC0E8091FD0E9091FE0E81
:10D160000F94812E42E06ED9E2E3FBE08491EF015F
:10D170002196882319F08DD8FE01F8CF20915A18F6
:10D1800030915B1840915C1850915D186091FF0ED2
:10D190007091000F8091010F9091020F0F94812EDA
:10D1A00042E050D9EEE2FBE08491EF012196882322
:10D1B00019F06FD8FE01F8CF6091030F7091040F42
:10D1C0008091050F9091060F42E03CD98FB7F894FB
:10D1D0004090E70E5090E80E6090E90E7090EA0ED5
:10D1E0008090EB0E9090EC0EA090ED0EB090EE0EB5
:10D1F000C090EF0ED090F00EE090F10EF090F20E95
:10D200008FBFE4E2FBE08491EF012196882319F0BF
:10D2100040D8FE01F8CFC301B201FAD8E0E2FBE04A
:10D220008491EF012196882319F033D8FE01F8CFBD
:10D23000C501B401EDD8ECE1FBE08491EF0121964A
:10D24000882319F026D8FE01F8CFC701B601E0D82F
:10D250008AE0DF91CF91FF90EF90DF90CF90BF9069
:10D26000AF909F908F907F906F905F904F9011C87C
:10D270004F925F926F927F92AF92BF92CF92DF9266
:10D28000EF92FF920F931F93CF9383E3A82E83E037
:10D29000B82E07E01FE0C0E0F50181915F010E9418
:10D2A0007BB8882309F46DC0C33009F063C00E94C5
:10D2B00044B86B017C0120E030E040EA51E40F9477
:10D2C000172A87FF4EC0A70196016091130F709136
:10D2D000140F8091150F9091160F0F945D2F2B0155
:10D2E0003C019B01AC016091950E7091960E80916E
:10D2F000970E9091980E0F947C2A6093950E7093E0
:10D30000960E8093970E9093980EA30192016091D0
:10D31000CD0E7091CE0E8091CF0E9091D00E0F94C5
:10D320007C2A6093CD0E7093CE0E8093CF0E909397
:10D33000D00E6091F6087091F7088091F8089091EE
:10D34000F9080F941B2AA30192010F947C2A0F94D1
:10D35000CA2F6093F6087093F7088093F8089093AB
:10D36000F908C092130FD092140FE092150FF092AB
:10D37000160F07C00E9444B8F8016083718382834E
:10D380009383CF5F0C5F1F4FC43009F085CFCF91DF
:10D390001F910F91FF90EF90DF90CF90BF90AF90D3
:10D3A0007F906F905F904F900C94C2E983E50E944C
:10D3B0007BB8882391F00E9444B820E030E04AE72F
:10D3C00054E40F947C2A0F94CA2F609380127093B8
:10D3D00081128093821290938312089583E50E94B4
:10D3E000AAB8882399F00E9444B820E030E04AE7C8
:10D3F00054E40F947C2A0F94CA2F609357027093C1
:10D4000058028093590290935A02089588E50E9429
:10D410007BB8811113C089E50E947BB881110EC0D1
:10D420008AE50E947BB8811109C085E40E947BB81F
:10D43000811104C00E94A9DF0D946C150E94A9DF20
:10D4400088E50E947BB8882319F0179A109270041F
:10D4500089E50E947BB8882319F0169A109271040E
:10D460008AE50E947BB8882319F0159A10927204FD
:10D4700085E40E947BB881110D946A1508950E947D
:10D48000B0760E94A9DF0F946C151092D708109205
:10D49000D60868EE73E080E090E00E94679860E054
:10D4A00086E09BE00C94A2ABCF93DF9383E50E94D0
:10D4B000AAB8882321F00E9414B8EB0102C0C0E092
:10D4C000D0E0DD27C230D105BCF0E3E3FBE284917C
:10D4D000EF012196882321F00E944961FE01F7CFD8
:10D4E000E4EEFAE08491EF012196882309F450C01C
:10D4F0000E944961FE01F6CF88E40E94AAB8882301
:10D50000A9F00E9414B8683771053CF0633281E0DD
:10D5100078072CF062E271E002C068E770E0FE017B
:10D52000EE0FFF1FEC57F14F7183608386E40E947A
:10D53000AAB88823A9F00E9414B8FE01EE0FFF1FBD
:10D54000E458F14F718360836F3F710519F014F057
:10D550006FEF70E077FF02C060E070E0718360837E
:10D5600082E40E94AAB8882399F00E9414B865301A
:10D57000710534F0683871052CF067E870E002C07E
:10D5800065E070E0CC0FDD1FC058D14F7983688310
:10D59000DF91CF9108952F923F924F925F926F92B9
:10D5A0007F928F929F92AF92BF92CF92DF92EF9233
:10D5B000FF920F931F93CF93DF93CDB7DEB72E97D4
:10D5C0000FB6F894DEBF0FBECDBF8091E50883FD96
:10D5D0006CC183E50E94AAB8482E811106C082E57D
:10D5E0000E94AAB8882309F460C10E9444B80F942D
:10D5F000C52F6739710514F066E970E07093520722
:10D60000609351070E94E1BC6091510770915207ED
:10D61000072E000C880B990B0F941D2A20914D07A3
:10D6200030914E0740914F07509150070F94172AA1
:10D6300087FF04C060E087ED9AE003C060E08AECF9
:10D640009AE00E94A2AB81E080931A0280914F047D
:10D6500080934C0719821A821B821C821D821E82B3
:10D660001F821886512C19862CE32A873CE13B87C0
:10D6700046E44C87E12CF12C00E81FEB812C912C27
:10D6800054016091510770915207072E000C880BCE
:10D69000990B0F941D2A6D877E87782E692E9B012A
:10D6A000482F592FB701C8010F94172A8823C1F1B9
:10D6B00020914D0730914E0740914F0750915007F0
:10D6C0006D857E85872D962D0F94172A582E551C13
:10D6D0005524551C442041F1552031F180911A0206
:10D6E000882309F4E2C060E08CEB9AE02E960FB636
:10D6F000F894DEBF0FBECDBFDF91CF911F910F9188
:10D70000FF90EF90DF90CF90BF90AF909F908F9061
:10D710007F906F905F904F903F902F900C94A2ABB2
:10D72000ED86FE86702E612E0E94844C6B017C017A
:10D73000DC01CB012D813E814F815885821B930BEB
:10D74000A40BB50BB7FD3AC0D701C60188519C4F59
:10D75000AF4FBF4F8D839E83AF83B8870E9478748D
:10D76000E6ECFAE084918F010F5F1F4F882321F0D0
:10D770000E944961F801F6CF81149104A104B1041B
:10D78000B9F0D501C40188519C4FAF4FBF4FBC01C8
:10D79000CD016C197D098E099F0928EE33E040E028
:10D7A00050E00F94232ECA01B9010E94086203C001
:10D7B0008FE30E9449618AE00E94496180E00F94F2
:10D7C00031160E945EA520904D0730904E070091C3
:10D7D0004F07109150079101A8016D857E85872D17
:10D7E000962D0F94802E9F7720E030E040EA50E4A1
:10D7F00081149104A104B10429F40F94172A87FF1E
:10D8000007C004C00F94A730181614F4460157013E
:10D81000552079F129813A814B815C8121153105AF
:10D820004105510541F0D701C601821B930BA40BA2
:10D83000B50BB7FD1EC09101A80169857A858B855E
:10D840009C850F94802E20E030E040EC5FE30F9445
:10D85000172A87FD43CFD701C601805A9541AF4FA4
:10D86000BF4F89839A83AB83BC8329863A860B8713
:10D870001C8780911A02882309F430CF8114910407
:10D88000A104B10429F4ED84FE84072D162DF9CEF0
:10D8900098EEC91A93E0D90AE108F108C818D90826
:10D8A000EA08FB08F7FE1ACFEECF2E960FB6F894D3
:10D8B000DEBF0FBECDBFDF91CF911F910F91FF90C3
:10D8C000EF90DF90CF90BF90AF909F908F907F9020
:10D8D0006F905F904F903F902F90089580E50E9449
:10D8E000AAB8811105C01092D7081092D6080895E1
:10D8F0000E9414B8672BB9F3089580E50E94AAB876
:10D90000811108C083E50E94AAB8811108C03FEFC9
:10D9100020E009C00E9424B8811111C0F3CF0E94F9
:10D9200014B8362F272F832F922F8F3F910519F090
:10D9300010F08FEF90E09093D7088093D608089569
:10D94000CF9380915A1581110E94A9DF80915B15B8
:10D950008823A9F180E50E94AAB8882319F00E94C3
:10D9600035B803C080E50E947BB8C82F482F61E01E
:10D9700080916D0890916E080F946E0883E50E9467
:10D98000AAB8882381F00E9414B8AB01BC0140936F
:10D99000FD175093FE176093FF17709300188CE4E7
:10D9A00097E10E940D6480915B15882319F081E056
:10D9B00080935A15C11103C0CF910D94821CCF9151
:10D9C0000895CF92DF92EF92FF92CF93DF936A0197
:10D9D0007B01C7EFDEE0E0914F0424E0E29FF0011D
:10D9E0001124E55DFD4F2081318142815381FC018D
:10D9F00060817181828193810F945D2F9B01AC01C5
:10DA00006C857D858E859F850F94812E6C877D87A3
:10DA10008E879F870E94C5B9C701B6010E9449B38E
:10DA2000DF91CF91FF90EF90DF90CF900C94A9DF22
:10DA3000CF92DF92EF92FF92CF93DF9381E08093BA
:10DA40001A02D1E0C1E080911A02882309F446C08D
:10DA5000CC2309F443C080E00F9431166091530742
:10DA600070915407C0E06115710569F3072E000C31
:10DA7000880B990B0F941D2A9B01AC016091D8086B
:10DA80007091D9088091DA089091DB080F94802E6C
:10DA90006B017C0120E030E0A9010F94A73018163B
:10DAA0005CF020E030E040E251ECC701B6010F9499
:10DAB000172A87FFC8CF0BC020E030E040E251E4D6
:10DAC000C701B6010F94A73018160CF0BCCFD09345
:10DAD000641180EA9BE90F947104B4CFDF91CF9178
:10DAE000FF90EF90DF90CF900895CF92DF92EF926A
:10DAF000FF920F931F93CF93DF9300D01F92CDB768
:10DB0000DEB7182F662351F010922E0710922A07C5
:10DB100010922B0710922C0710922D070E94844C14
:10DB2000C0902A07D0902B07E0902C07F0902D078B
:10DB30009B01AC012C193D094E095F0957FD3EC000
:10DB400017FD16C040912E07212F012E000C330B1C
:10DB50002C5F3F4FE42F042E000CFF0B2E173F07C6
:10DB60006CF141172CF000E911E020E030E004C036
:10DB700004EC19E020E030E0DC01CB01800F911FC4
:10DB8000A21FB31F80932A0790932B07A0932C0703
:10DB9000B0932D0780ED97E09C838B838CE291E01E
:10DBA0009A838983BE016D5F7F4FCE0101960E94EB
:10DBB00040F380912E078F5F80932E070F900F9078
:10DBC0000F900F90DF91CF911F910F91FF90EF90E9
:10DBD000DF90CF900895EF92FF920F931F93CF9312
:10DBE000DF931F92CDB7DEB78C017B0180E24983C2
:10DBF0000E94496149814F3F11F084E501C082E4F0
:10DC00000E9449618AE30E944961F8016081718143
:10DC10008281938142E00E942262F701408151811A
:10DC2000628173818FE79EE00E94A3A562E070E0AD
:10DC300080E090E00F90DF91CF911F910F91FF90C6
:10DC4000EF900C944C4C2F923F924F925F926F92B8
:10DC50007F928F929F92AF92BF92CF92DF92EF927C
:10DC6000FF920F931F93CF93DF9300D01F92CDB7F6
:10DC7000DEB79C838B834B015A01DC0113968C9198
:10DC8000811103C08FEF9FEFEBC0EB81FC8181819D
:10DC900080FFF8CFAB81BC8151960D911D912D91E4
:10DCA0003C91549718964D915D916D917C911B9785
:10DCB000C501A0E0B0E068017901C41AD50AE60AFE
:10DCC000F70AC816D906EA06FB0618F45801A41A82
:10DCD000B50A75018B819C8104969A838983612C96
:10DCE00092E0792EE114F10409F48BC0AB81BC8180
:10DCF00018964D915D916D917C911B976A01B1E0F1
:10DD0000DB22EB81FC8123811A012B0189E05694EF
:10DD10004794379427948A95D1F7818D928D22303C
:10DD200061F4FC01828D938DA48DB58DBC01CD0174
:10DD3000620D731D841D951D4AC0DC0114961C9153
:10DD400011501221C114D10401F511111EC0452B2F
:10DD5000462B472B59F4EB81FC8185899689A7894D
:10DD6000B08D84839583A683B7830FC0AB81BC81BC
:10DD700014964D915D916D917C91179729813A810F
:10DD80000F946421882309F47DCFEB81FC81218DE0
:10DD9000328D84819581A681B7810297A109B1094D
:10DDA000F901058404C0880F991FAA1FBB1F0A949C
:10DDB000D2F74685578560897189840F951FA61F04
:10DDC000B71FBC01CD01610F711D811D911D930114
:10DDD0002C193D0987012E153F0508F4890101150D
:10DDE000F2E01F0779F52091311130913211409105
:10DDF000331150913411621773078407950719F492
:10DE000021C0C5012DC09401AB01BC0180913A1124
:10DE100090913B110E94B695882309F433CF800E70
:10DE2000911EEB81FC8180859185A285B385800F51
:10DE3000911FA11DB11D80879187A287B387E01A2A
:10DE4000F10A50CF40E00F949B20882309F41ACFA9
:10DE5000B6016F5C704FA801C4010F949F31DFCFF2
:10DE60000F900F900F900F90DF91CF911F910F9116
:10DE7000FF90EF90DF90CF90BF90AF909F908F90EA
:10DE80007F906F905F904F903F902F9008950F93E9
:10DE90001F93CF93DF93FC012381222311F080E0B5
:10DEA00044C08B01EC01FB018789803139F180325C
:10DEB000B1F783E08B83F801428D538D648D758DAE
:10DEC0004D8B5E8B6F8B788F9E012F5E3F4FC8010D
:10DED0000F94E421882319F31A8F098F81E0898335
:10DEE000188619861A861B861C821D821E821F8236
:10DEF000188A1C861D861E861F8617C082E08B83AB
:10DF00001D8A1E8A1F8A188EFB01808D918DA0E0CC
:10DF1000B0E025E0880F991FAA1FBB1F2A95D1F7F3
:10DF2000898B9A8BAB8BBC8BD7CFDF91CF911F9115
:10DF30000F910895CF93DF93EC010E94DA631B8267
:10DF4000DF91CF910895CF93DF93EC0141E0611110
:10DF500001C040E06C857D858E859F850F949B2058
:10DF6000882341F0888920E2829FC00111248F5CC0
:10DF7000904F02C080E090E0DF91CF910895CF9361
:10DF8000DF93EB01FC012381211102C080E027C057
:10DF90002250223020F48FE2888319821FC060E073
:10DFA000D2DF009799F3FC0190E080E02EE230810F
:10DFB000303269F0883029F4DE01A90FB11D2C93AD
:10DFC0009F5F3081DE01A90FB11D3C939F5F8F5F82
:10DFD00031968B3061F7C90FD11D188281E0DF9136
:10DFE000CF9108953F924F925F926F927F928F925E
:10DFF0009F92AF92BF92CF92DF92EF92FF920F93D8
:10E000001F93CF93DF93CDB7DEB72C970FB6F8945D
:10E01000DEBF0FBECDBF5C01DC0159968D909C9098
:10E020005A97F40181859285A385B4859C01AD0141
:10E030002F5F3F4F4F4F5F4F29873A874B875C8752
:10E04000D5011496CD90DD90ED90FC901797C114FA
:10E05000D104E104F10439F0BFEFCB1ADB0AEB0A7B
:10E06000FB0A312C07C0F401C080D180E280F3802C
:10E0700033243394260137011D821E821F821886A5
:10E08000F40181859285A385B4852D813E814F81E0
:10E090005885281739074A075B0708F064C0898547
:10E0A0009A85AB85BC858C159D05AE05BF0550F4E2
:10E0B00082E0C82ED12CE12CF12C92E0492E512C7B
:10E0C000612C712C9E012F5F3F4FB701A601C40147
:10E0D0000F946421882309F446C089819A81AB8119
:10E0E000BC81892B8A2B8B2B41F0260137019FEFB6
:10E0F000491A590A690A790A05C0C414D504E60404
:10E10000F70491F02D813E814F8158852F5F3F4F5D
:10E110004F4F5F4F2D833E834F8358873FEFC31A86
:10E12000D30AE30AF30AACCF0FEF1FEF2FEF3FE064
:10E13000B301A201C4010F94D320F82E882399F0D3
:10E14000D50114964D915D916D917C911797411574
:10E1500051056105710549F093018201C4010F94D5
:10E16000D320811102C0F12C29C0D50114964D9203
:10E170005D926D927C921797332051F0D301C201CA
:10E180000196A11DB11DF40180839183A283B38305
:10E19000F50185899689A789B08D892B8A2B8B2BD0
:10E1A00069F4D50155964D925D926D927C92589787
:10E1B00011968C911197806811968C938F2D2C96C7
:10E1C0000FB6F894DEBF0FBECDBFDF91CF911F9188
:10E1D0000F91FF90EF90DF90CF90BF90AF909F9006
:10E1E0008F907F906F905F904F903F9008954F92E7
:10E1F0005F926F927F92AF92BF92CF92DF92EF9237
:10E20000FF920F931F93CF93DF931F92CDB7DEB78B
:10E210008C017B015A01D22EDB0159968D919C9184
:10E220005A97F801928F818F40E050E0BA01C70100
:10E230000E940D64C12CF70180859185A285B3856C
:10E24000418952896389748984179507A607B7079E
:10E2500008F062C025E0B695A795979587952A9511
:10E26000D1F7F82FFF707F2ED70113968C91823053
:10E2700008F462C041E050E0BE016F5F7F4FC7010C
:10E28000E2DC019719F4898190E002C08FEF9FEFE3
:10E29000019609F451C0F70180859185A285B38567
:10E2A0004F96A11DB11D80879187A287B387F0E2A9
:10E2B0007F9EC0011124BC016F5C704F6115710518
:10E2C000D9F1DB012C91222319F0253ED1F467C14D
:10E2D000C1100EC040913111509132116091331133
:10E2E00070913411F8014487558766877787708A63
:10E2F000FC01EF5CF04F8081882361F0CC24C39453
:10E300009ACF4BE050E0C5010F949231892B09F070
:10E3100092CF14C0CC24C3948D2D8274823461F4C6
:10E32000CC2009F489C0D80150967C9061E0C801E6
:10E330000ADE009709F006C180E034C1D7FCFCCFAB
:10E34000F0E27F9EA00111249A012F5C304FD90189
:10E350001B968C91817121F08D2D827109F068C01E
:10E360008091311190913211A0913311B0913411FB
:10E37000F80184879587A687B787708AFA01EF5CD2
:10E38000F04F4489558960E070E0BA015527442771
:10E39000D80155964D935D936D937C935897828DDC
:10E3A000938DA0E0B0E0482B592B6A2B7B2BD80132
:10E3B00055964D935D936D937C935897D9011B9619
:10E3C0008C91887159F4848D958DA68DB78DF80147
:10E3D000818B928BA38BB48B81E010C0803141F58F
:10E3E00098012F5E3F4FD80159968D919C915A9775
:10E3F0000F94E4218823E1F084E0F80183838D2DDC
:10E400008F70D80111968C931197F80114821582A0
:10E410001682178218961D921D921D921C921B97B0
:10E42000D4FEB0C0C8010F94A2058111ABC084CF47
:10E43000D80113961C9280CFF7018381823009F4B2
:10E440007BCF81899289A389B489803E9F4FAF4158
:10E45000B10508F071CFC701C5DD882309F46CCF81
:10E460000F945B20882309F467CFD70159962D912B
:10E470003C915A9714968D919D910D90BC91A02D31
:10E480000297A109B109F901058404C0880F991FF9
:10E49000AA1FBB1F0A94D2F74684578460887188EC
:10E4A000480E591E6A1E7B1E81E0809339114092EE
:10E4B000311150923211609233117092341180E018
:10E4C00092E0E1E3FFE0DF019C011D92215030402A
:10E4D000E1F7CC24C394D7015996ED91FC915A975A
:10E4E0008481C81698F421E33FE0B301A2014C0DEA
:10E4F000511D611D711D80913A1190913B110E9437
:10E500005495882309F418CFC394E5CF80E092E0B6
:10E51000A0E0B0E0058404C0880F991FAA1FBB1FAC
:10E520000A94D2F7F7014189528963897489840F6B
:10E53000951FA61FB71F818B928BA38BB48B81E392
:10E540009FE0712C20E2DC011D922A95E9F72BE077
:10E55000F501DC0101900D922A95E1F721E238E204
:10E56000FC01318B208B40E058E057874687338B86
:10E57000228B318F208F578B468B0F945B2081111C
:10E58000DFCEDACED5FE09C0F80141895289638910
:10E590007489C8010E940D6405C081E003C0C110E8
:10E5A000ADCE98CE0F90DF91CF911F910F91FF903C
:10E5B000EF90DF90CF90BF90AF907F906F905F9083
:10E5C0004F9008952F923F924F925F926F927F9259
:10E5D0008F929F92AF92BF92CF92DF92EF92FF9273
:10E5E0000F931F93CF93DF93CDB7DEB7C254D109FA
:10E5F0000FB6F894DEBF0FBECDBF4C015B018A01A0
:10E60000322E1C8E1F8E19821C826115710511F429
:10E6100010E0A3C0FC0183818111FACFFA0180814F
:10E620008F3209F098C0F50183818250823058F012
:10E63000618D728DCE0101962ADC882349F3CE01CB
:10E6400001967C0101C07501C8018C010196F80199
:10E6500020812F32D1F36E01FCE1CF0ED11C3601A7
:10E66000CE0101962C012396CFAE23972D2C9BE053
:10E670009150E7E3F0E0EC0FFD1FE90FF11D80E2A0
:10E6800080839111F5CFD80127E04A2F3B2F8D9140
:10E69000811107C08FA9803209F4BACF842F932F3C
:10E6A0002CC08F32B9F38E3231F42A3009F4B0CF56
:10E6B00098E02AE0EACFEBE8FEE03491332321F042
:10E6C00031963813FACFA4CF291708F4A1CF81329D
:10E6D00008F49ECF8F3709F49BCF31E0390FE7E381
:10E6E000F0E0EC0FFD1FE90FF11D9FE9980F9A3143
:10E6F00008F480528083932FC8CF8C01FC012081C5
:10E7000001962F32D1F32223E9F021E0AE01495CDA
:10E710005F4FB701C6016BDD882309F479CFEA1496
:10E72000FB0411F0C70106DCC614D70441F02396A0
:10E730009FAD2397822D7601C92ED82E98CF942D88
:10E74000852DF9CF232DAE01495C5F4FB701C40180
:10E750004EDD182F02C07B017ECFCE0101960E94B4
:10E76000B6B9CE014C960E94B6B9812FCE5BDF4F71
:10E770000FB6F894DEBF0FBECDBFDF91CF911F91D2
:10E780000F91FF90EF90DF90CF90BF90AF909F9050
:10E790008F907F906F905F904F903F902F90089553
:10E7A0002F923F924F925F926F927F928F929F92A1
:10E7B000AF92BF92CF92DF92EF92FF920F931F938F
:10E7C000CF93DF93EC014DE75DE081E090E0FA014B
:10E7D00025913491C217D3070CF05DC09C012150E4
:10E7E0003109220F331F220F331FD901A558B24F11
:10E7F000FD01659174912758324FF901A590B490AD
:10E80000FC01EE0FFF1FEE0FFF1FE558F24FE590E2
:10E81000F490FD01C590D490FA0105911491F9018D
:10E8200025903490072E000C880B990B0F941D2A0D
:10E830002B013C01CA19DB09BE01DD0F880B990BC6
:10E840000F941D2A4B015C01B7016C197D09072E3D
:10E85000000C880B990B0F941D2A9B01AC01C5017C
:10E86000B4010F947C2A6B017C01B8016219730911
:10E87000072E000C880B990B0F941D2A9B01AC01ED
:10E88000C701B6010F945D2F9B01AC01C301B2011A
:10E890000F94812E11C001964C5F5F4F803291051D
:10E8A00009F095CFE7EFFDE065917491072E000C1C
:10E8B000880B990B0F941D2ADF91CF911F910F9117
:10E8C000FF90EF90DF90CF90BF90AF909F908F9090
:10E8D0007F906F905F904F903F902F900895609140
:10E8E000D8087091D9088091DA089091DB080895D2
:10E8F0000F931F93CF93DF93CDB7DEB728970FB653
:10E90000F894DEBF0FBECDBF6091530770915407DE
:10E91000072E000C880B990B0F941D2A6D837E83A4
:10E920008F8398878091D8089091D908A091DA08B0
:10E93000B091DB0889839A83AB83BC834EEFBE0121
:10E940006B5F7F4FCE01019646D960915107709160
:10E950005207072E000C880B990B0F941D2A6D830C
:10E960007E838F83988780914D0790914E07A09169
:10E970004F07B091500789839A83AB83BC834FEFD5
:10E98000BE016B5F7F4FCE01019625D9E7E8FEE01F
:10E9900084918F010F5F1F4F882321F00E944961EE
:10E9A000F801F6CFE0914C07F0E0E65BF84F6081AC
:10E9B00070E080E090E00E940862E2E8FEE084916E
:10E9C0008F010F5F1F4F882321F00E944961F801DA
:10E9D000F6CF60914B0770E080E090E00E94086203
:10E9E00028960FB6F894DEBF0FBECDBFDF91CF9152
:10E9F0001F910F9108951F920F920FB60F9211243D
:10EA00000BB60F921F932F933F934F935F936F9388
:10EA10007F938F939F93AF93BF93CF93DF93EF93A6
:10EA2000FF938091450E811185C181E08093450E51
:10EA300080916E008B7F80936E00789480911D0290
:10EA40008F3790F08F5790914A07909349079923F9
:10EA500011F0759A01C0759890914B0790934807F3
:10EA6000992359F0A59A0AC090914907891708F08F
:10EA7000759890914807891708F0A5988F5F809343
:10EA80001D029091470781E08927809347078111F4
:10EA90000E942BAB80911C02823079F1A0F4882374
:10EAA00041F1813009F042C0809178009091790065
:10EAB00020913C0730913D07820F931F90933D07B3
:10EAC00080933C0733C0833019F1843079F580910D
:10EAD0004607811103C086E0809346078091460770
:10EAE000815080934607882309F183E080931C02BC
:10EAF0001DC010927B0080E403C010927B0082E472
:10EB000080937C0080917A00806480937A000EC0AC
:10EB1000809178009091790020913A0730913B07DD
:10EB2000820F931F90933B0780933A0780911C02BA
:10EB300081116DC080911B028F5F80311CF4809326
:10EB40001B0265C010921B0280913907811113C00E
:10EB500080913C0790913D07909338078093370749
:10EB600080913A0790913B07909336078093350741
:10EB700081E0809339078AE0ECE3F7E0DF011D9242
:10EB80008A95E9F710923B0710923A07C091370730
:10EB9000D0913807D195C195D10911E080914A07EC
:10EBA000811101C010E080916804909169049195F1
:10EBB000819591098C179D070CF490C080911602E5
:10EBC00090911702919581959109C817D9070CF476
:10EBD00090C0C1E080914B07811101C0C0E020913D
:10EBE000350730913607809166049091670482174B
:10EBF00093070CF089C02091140230911502809186
:10EC0000350790913607821793070CF088C08091E2
:10EC10001C028F5F853018F480931C0202C0109292
:10EC20001C0220E030E0ABE0B0E0C901880F991F82
:10EC3000FC01E15DF84F408151814115510509F416
:10EC40003EC0F894223041F5609109016470159836
:10EC5000EFB7141615062CF4F89470910B0174603C
:10EC600004C0F89470910B017B7F70930B01EFBF90
:10EC7000429AFD013197F1F742987FB7662329F058
:10EC8000F89460910B01646004C0F89460910B01EA
:10EC90006B7F60930B017FBF7894FC01E15DF84FBF
:10ECA000141615063CF4408151814150510951839D
:10ECB000408305C0808191810196918380832F5F7D
:10ECC0003F4F2330310509F0B0CFF8941092450E34
:10ECD00080916E00846080936E002CC0112309F433
:10ECE0006DCF4FE65EE06DE47EE080E00E9439BECD
:10ECF00065CF112309F46DCF4CE25EE06AE07EE05F
:10ED000080E00E9439BE65CFCC2309F474CF4CE378
:10ED10005EE06DE47EE08FEF0E9439BE6CCFCC23C5
:10ED200009F475CF49EF5DE06AE07EE08FEF0E9465
:10ED300039BE6DCFFF91EF91DF91CF91BF91AF9130
:10ED40009F918F917F916F915F914F913F912F9103
:10ED50001F910F900BBE0F900FBE0F901F90189534
:10ED6000109254071092530780E00E942CBD10921D
:10ED70005207109251070E94E1BC0F94D51C1092CB
:10ED800054071092530780E00E942CBD10924A074E
:10ED90007598109252071092510710924B07A59840
:10EDA0000895EF92FF921F93CF93DF931F92CDB7F9
:10EDB000DEB7182FE4EBFEE084917F012FEFE21A1B
:10EDC000F20A882331F099830E944961F701998101
:10EDD000F3CFE12FF92F84917F019FEFE91AF90A10
:10EDE000882321F00E944961F701F5CFEBE9FEE0AD
:10EDF00084917F012FEFE21AF20A882321F00E940A
:10EE00004961F701F5CF0F90DF91CF911F91FF90EE
:10EE1000EF9008952F923F924F925F926F927F9260
:10EE20008F929F92AF92BF92CF92DF92EF92FF921A
:10EE30000F931F93CF93DF93CDB7DEB7C251D1406D
:10EE40000FB6F894DEBF0FBECDBF41E061E081E0B8
:10EE50000E942DB181110C945587FE0131968CE3EF
:10EE6000DF011D928A95E9F70091880EC453DF4FA8
:10EE70000883CC5CD0408AE40E947BB8882321F0D0
:10EE80000E94D7B70C94558786E50E94AAB88823BC
:10EE900049F00E9414B8C652DF4F79836883CA5D77
:10EEA000D04006C0C652DF4F19821882CA5DD040DA
:10EEB000C652DF4F08811981CA5DD0400530110567
:10EEC00070F0E0EAF0E184918F010F5F1F4F88231B
:10EED00011F40C9455870E944961F801F4CF84E441
:10EEE0000E94AAB8882319F00E9435B803C084E4B0
:10EEF0000E947BB8C851DF4F8883C85ED040C6529D
:10EF0000DF4F08811981CA5DD040033011058CF4B0
:10EF100084E50E94AAB8882319F00E9435B803C07E
:10EF200084E50E947BB8CE51DF4F8883C25ED0401B
:10EF300006C011E0CE51DF4F1883C25ED04088E595
:10EF40000E94AAB8882321F00E9414B8162F01C08D
:10EF500012E089E50E94AAB8882321F00E9414B823
:10EF6000062F01C002E080E50E94AAB881110BC003
:10EF7000C752DF4F1883C95DD040C553DF4F0883A8
:10EF8000CB5CD0400CC00E9414B8C752DF4F6883DE
:10EF9000C95DD040C553DF4F6883CB5CD040C752BA
:10EFA000DF4F0881C95DD040023018F4EBE6F0E194
:10EFB00008C0C553DF4F1881CB5CD040123068F4D5
:10EFC000F5CF84918F010F5F1F4F882311F40C94AC
:10EFD00055870E944961F801F4CF83E50E94AAB8E1
:10EFE000882319F00E9444B804C060E070E88BEBFD
:10EFF00095E420E030E040E752E40F945D2F609309
:10F000009F027093A0028093A1029093A2028CE4CD
:10F010000E94AAB8882381F00E9444B82091521817
:10F020003091531840915418509155180F94802ED8
:10F030000F94C52F7B0104C05DEFE52EFF24FA94E9
:10F0400082E50E94AAB8882381F00E9444B82091EA
:10F0500052183091531840915418509155180F94EC
:10F06000802E0F94C52F5B0103C043EAA42EB12C60
:10F0700086E40E94AAB8882381F00E9444B82091B7
:10F0800056183091571840915818509159180F94AC
:10F09000802E0F94C52F8B0102C00CEF1FEF82E46E
:10F0A0000E94AAB8882381F00E9444B82091561883
:10F0B0003091571840915818509159180F94802E3C
:10F0C0000F94C52F6B0103C038EAC32ED12C81E009
:10F0D0002DEFE2162FEFF2063CF095012950310991
:10F0E000E216F3060CF480E021E034EAA316B10442
:10F0F0003CF4A701475F5F4F4A155B050CF420E025
:10F10000882483940C3F4FEF14073CF0A60149502C
:10F110005109041715070CF4812C9924939459EA8A
:10F12000C516D1043CF4A801475F5F4F4C155D053F
:10F130000CF4912C81110BC0222321F08CE590E17D
:10F1400030DE14C0811012C0911015C01DC084E6BD
:10F1500090E1CE5EDE4F2883C251D14022DECE5EEA
:10F16000DE4F2881C251D1402111E8CF882019F00B
:10F1700084E590E116DE992011F40C9455878DE416
:10F1800090E10FDE0C945587C652DF4F888199813C
:10F19000CA5DD040892B21F1E7E3F0E184914F0172
:10F1A0009FEF891A990A882321F00E944961F4018E
:10F1B000F5CFC851DF4FA881C85ED040AA2369F0BF
:10F1C000EDE2F0E184914F01BFEF8B1A9B0A882397
:10F1D00021F00E944961F401F5CF8AE00E94496163
:10F1E0000E94A9DF80E00E94C0B781E00E94F8B2CF
:10F1F000882349F0C453DF4F8881CC5CD0400E9403
:10F20000C0B70C9455870E94F3B185E40E94AAB858
:10F21000882319F00E9435B803C085E40E947BB8AA
:10F22000CC51DF4F8883C45ED040C752DF4FF88196
:10F23000C95DD040EF2FF0E0C751DF4FF983E8837D
:10F24000C95ED040C553DF4F3881CB5CD040232FFF
:10F2500030E0C351DF4F39832883CD5ED040C752A1
:10F26000DF4F5881C95DD040C553DF4F4881CB5C2B
:10F27000D040549FA0011124C052DF4F59834883CE
:10F28000C05ED040C752DF4F5881C95DD040517039
:10F29000CB52DF4F5883C55DD040C052DF4F8881CD
:10F2A0009981C05ED040880F991FC750DF4F998366
:10F2B0008883C95FD040CD53DF4F19821882C35C69
:10F2C000D040C452DF4F188219821A821B82CC5D53
:10F2D000D040C554DF4F188219821A821B82CB5B43
:10F2E000D040AFEFBFEFC954DF4FB983A883C75BEE
:10F2F000D04097010F2C000C440B550BCB5FDE4F19
:10F30000288339834A835B83C550D140A5014E19B8
:10F310005F09C75FDE4F59834883C950D140C80198
:10F32000012E000CAA0BBB0BC55FDE4F88839983AF
:10F33000AA83BB83CB50D140D601A01BB10BC15FC8
:10F34000DE4FB983A883CF50D140CB52DF4F088125
:10F35000C55DD040002391F0C553DF4F0881CB5CE1
:10F36000D040C353DF4F0883CD5CD04011E0CF5273
:10F37000DF4F1883C15DD04010E011C0C553DF4F8F
:10F380001881CB5CD04011500FEFCF52DF4F088374
:10F39000C15DD040C353DF4F0883CD5CD04081E0D6
:10F3A000CB52DF4F0881C55DD0400827CB52DF4FDD
:10F3B0000883C55DD0402CE0C954DF4F4881598196
:10F3C000C75BD040249FC001259F900D1124DC0114
:10F3D000A85DBA4EC154DF4FB983A883CF5BD0403C
:10F3E000440F551F440F551FCF50DF4F598348839B
:10F3F000C15FD040C954DF4F88819981C75BD0403D
:10F40000C052DF4FE881F981C05ED0408E0F9F1F50
:10F410009C01220F331F220F331FCB50DF4F398344
:10F420002883C55FD040C954DF4F88819981C75B6D
:10F43000D040C750DF4F48815981C95FD040840F09
:10F44000951FDC01AA0FBB1FAA0FBB1FC550DF4FC2
:10F45000B983A883CB5FD040C953DF4F198218828C
:10F46000C75CD040C751DF4FE881F981C95ED04009
:10F470003197C350DF4FF983E883CD5FD040CD5340
:10F48000DF4F28813981C35CD040032E000C440B30
:10F49000550BC150DF4F288339834A835B83CF5F8D
:10F4A000D040CD53DF4F48815981C35CD040440FD9
:10F4B000551FCD5FDE4F59834883C350D140C3539E
:10F4C000DF4F0881CD5CD040101709F4C9C2CB5F73
:10F4D000DE4F688179818A819B81C550D1400F942C
:10F4E0001D2A6B017C01C75FDE4F88819981C9505D
:10F4F000D140C350DF4F68817981CD5FD0400F94F8
:10F500006931072E000C880B990B0F941D2A4B01B3
:10F510005C01C150DF4F688179818A819B81CF5F17
:10F52000D0400F941D2A9B01AC01C501B4010F947A
:10F530007C2A9B01AC01C701B6010F94812E6B019F
:10F540007C01C55FDE4F688179818A819B81CB50C8
:10F55000D1400F941D2A4B015C01C15FDE4F8881B1
:10F560009981CF50D140C351DF4F68817981CD5E01
:10F57000D040615071090F946931072E000C880B3F
:10F58000990B0F941D2A2B013C01612F012E000CB9
:10F59000770B880B990B0F941D2A9B01AC01C301BB
:10F5A000B2010F947C2A9B01AC01C501B4010F94F8
:10F5B000812E4B015C0120E030E0A901C701B601BA
:10F5C0000F94172A87FD05C020E030E040E05FE39C
:10F5D00003C020E030E0A901C701B6010F94812EDD
:10F5E0000F94F62FC355DF4F688379838A839B83FB
:10F5F000CD5AD04020E030E0A901C501B4010F94FC
:10F60000172A87FD05C020E030E040E05FE303C03B
:10F6100020E030E0A901C501B4010F94812E0F94C0
:10F62000F62FC755DF4F688379838A839B83C95A36
:10F63000D040C954DF4F88819981C75BD040019683
:10F64000C954DF4F99838883C75BD040CD5FDE4FBD
:10F65000E881F981C350D140E10FF11D17FDFA9502
:10F66000EE0FFF1FA1EAB0E0AC0FBD1FEA0FFB1FBA
:10F6700091838083C652DF4F2881CA5DD040CC5130
:10F68000DF4F4881C45ED040BE0167557F4FCE0139
:10F6900083559F4F0F94DF22C554DF4F68837983D2
:10F6A0008A839B83CB5BD0409B01AC010F942D31AF
:10F6B000882341F0C453DF4F8881CC5CD0400E9446
:10F6C000C0B7CEC1C554DF4F288139814A815B81E3
:10F6D000CB5BD040C452DF4F688179818A819B81A6
:10F6E000CC5DD0400F94812EC452DF4F6883798364
:10F6F0008A839B83CC5DD040C953DF4F8881998139
:10F70000C75CD040CF50DF4FE881F981C15FD04066
:10F710008E0F9F1FEDE6F0E0EC0FFD1FE80FF91FC5
:10F72000C554DF4F288139814A815B81CB5BD04052
:10F730002483358346835783C355DF4F2880398020
:10F740004A805B80CD5AD040EDE3F0E0EC0FFD1F26
:10F75000E80FF91F2482358246825782C755DF4F52
:10F7600088809980AA80BB80C95AD040C953DF4F96
:10F77000E881F981C75CD040CB50DF4F4881598187
:10F78000C55FD040E40FF51F8DE390E08C0F9D1F07
:10F79000E80FF91F84829582A682B782C953DF4F92
:10F7A000E881F981C75CD040C550DF4FA881B9819D
:10F7B000CB5FD040EA0FFB1FE80FF91F20E030E0DD
:10F7C00040E85FE32483358346835783A201910198
:10F7D00069817A818B819C810F94812E69837A83E0
:10F7E0008B839C83A50194016D817E818F81988597
:10F7F0000F94812E6D837E838F839887C554DF4F4E
:10F80000288139814A815B81CB5BD04069857A85CB
:10F810008B859C850F94812E69877A878B879C873F
:10F82000A2019101C201B1010F947C2A9B01AC019C
:10F830006D857E858F8598890F94812E6D877E8753
:10F840008F87988BA5019401C501B4010F947C2A80
:10F850009B01AC0169897A898B899C890F94812EDF
:10F86000698B7A8B8B8B9C8BC554DF4F28813981B8
:10F870004A815B81CB5BD040CA01B9010F947C2ADD
:10F880009B01AC016D897E898F89988D0F94812EA3
:10F890006D8B7E8B8F8B988FA5019401C201B10176
:10F8A0000F947C2A9B01AC01698D7A8D8B8D9C8D88
:10F8B0000F94812E698F7A8F8B8F9C8FC554DF4F69
:10F8C000288139814A815B81CB5BD040C201B10183
:10F8D0000F947C2A9B01AC016D8D7E8D8F8D98A13C
:10F8E0000F94812E6D8F7E8F8F8F98A3C554DF4F1D
:10F8F000288139814A815B81CB5BD040C501B4014D
:10F900000F947C2A9B01AC0169A17AA18BA19CA1D7
:10F910000F94812E69A37AA38BA39CA3720161012A
:10F92000E894F7F86DA07EA00FA138A5C453DF4F6F
:10F930003883CC5CD0409301402FC453DF4F5881B3
:10F94000CC5CD040C701B6010F94A73018163CF02C
:10F950006301E02EC453DF4FF880CC5CD040CDA2D1
:10F96000DEA2EFA2F8A675016401E894F7F869A495
:10F970007AA40BA54CA5C453DF4F4883CC5CD04080
:10F980009301402FC453DF4F5881CC5CD040C70156
:10F99000B6010F94A73018163CF06301E02EC45353
:10F9A000DF4FF880CC5CD040C9A6DAA6EBA6FCA657
:10F9B00020E030E040E85FE369AD7AAD8BAD9CAD0F
:10F9C0000F94812E69AF7AAF8BAF9CAFC154DF4FDC
:10F9D000A881B981CF5BD0401C962D923D924D926B
:10F9E0005C921F97FD01808A918AA28AB38AC554CE
:10F9F000DF4F288139814A815B81CB5BD0405496AF
:10FA00002D933D934D935C93579780E00F9431165F
:10FA1000CF52DF4F0881C15DD040100FC154DF4F7E
:10FA200028813981CF5BD040245F3F4FC154DF4FE5
:10FA300039832883CF5BD040C953DF4F4881598138
:10FA4000C75CD0404C5F5F4FC953DF4F5983488339
:10FA5000C75CD040C453DF4F1882CC5CD0402FCD60
:10FA6000CD53DF4F8881C35CD0408F5FC752DF4FDB
:10FA70001881C95DD0408117E8F4CD53DF4F08816C
:10FA80001981C35CD0400F5F1F4FCD53DF4F1983E7
:10FA90000883C35CD040C554DF4F288139814A8137
:10FAA0005B81CB5BD040CA01B9010F942D31882313
:10FAB00009F44BCC80E00E94F8B2882349F0C4538B
:10FAC000DF4F8881CC5CD0400E94C0B70C944C873B
:10FAD000C554DF4F288139814A815B81CB5BD0409F
:10FAE000CA01B9010F942D3181110C944C8789AC56
:10FAF0009AACABACBCAC20E030E0A901C501B401CC
:10FB00000F94172A882309F408C2A501940169817A
:10FB10007A818B819C810F945D2FC954DF4F68835C
:10FB200079838A839B83C75BD04069837A838B8385
:10FB30009C83A50194016D817E818F8198850F94AE
:10FB40005D2FC154DF4F688379838A839B83CF5BAA
:10FB5000D0406D837E838F839887A501940169854A
:10FB60007A858B859C850F945D2FCD53DF4F6883FD
:10FB700079838A839B83C35CD04069877A878B872C
:10FB80009C87A50194016D857E858F8598890F944A
:10FB90005D2F6B017C01C954DF4F288139814A8177
:10FBA0005B81C75BD040CA01B9010F947C2A9B01DD
:10FBB000AC01C701B6010F94802ECB52DF4F688392
:10FBC00079838A839B83C55DD0406D877E878F87CD
:10FBD000988BA501940169897A898B899C890F94F6
:10FBE0005D2F6B017C01C154DF4F288139814A812F
:10FBF0005B81CF5BD040CA01B9010F947C2A9B0185
:10FC0000AC01C701B6010F94802EC353DF4F688348
:10FC100079838A839B83CD5CD040698B7A8B8B8B75
:10FC20009C8BA50194016D897E898F89988D0F9495
:10FC30005D2F6B017C01CD53DF4F288139814A81D3
:10FC40005B81C35CD040CA01B9010F947C2A9B013F
:10FC5000AC01C701B6010F94802E6D8B7E8B8F8B0C
:10FC6000988FA5019401698D7A8D8B8D9C8D0F9451
:10FC70005D2F6B017C01C154DF4F288139814A819E
:10FC80005B81CF5BD040C954DF4F688179818A8125
:10FC90009B81C75BD0400F947C2A9B01AC01C701BC
:10FCA000B6010F94802EC953DF4F688379838A830E
:10FCB0009B83C75CD040698F7A8F8B8F9C8FA50107
:10FCC000940169A17AA18BA19CA10F945D2F6B0176
:10FCD0007C01CD53DF4F288139814A815B81C35C30
:10FCE000D040C154DF4F688179818A819B81CF5B8D
:10FCF000D0400F947C2A9B01AC01C701B6010F9440
:10FD0000802E6B017C0169A37AA38BA39CA3A50120
:10FD100094016D8D7E8D8F8D98A10F945D2F4B0179
:10FD20005C01CD53DF4F288139814A815B81C35CFF
:10FD3000D040C954DF4F688179818A819B81C75B3C
:10FD4000D0400F947C2A9B01AC01C501B4010F94F3
:10FD5000802E4B015C016D8F7E8F8F8F98A3C353D4
:10FD6000DF4F288139814A815B81CD5CD040CB5205
:10FD7000DF4F688179818A819B81C55DD0400F9476
:10FD80007C2A2B013C01C953DF4F288139814A81EC
:10FD90005B81C75CD040CA01B9010F947C2A9B01EA
:10FDA000AC01C301B2010F94802ECF52DF4F6883A4
:10FDB00079838A839B83C15DD0402B013C01E89409
:10FDC00077F829A53AA54BA55CA56DA17EA18FA1C9
:10FDD00098A50F94812E2FEF36EE4BED5EE20F9437
:10FDE0007C2A9B01AC01C301B2010F94172A18169B
:10FDF0000CF093C0C953DF4F288139814A815B8160
:10FE0000C75CD040C701B6010F947C2A2B013C018E
:10FE1000C353DF4F288139814A815B81CD5CD0405B
:10FE2000C501B4010F947C2A9B01AC01C301B2014E
:10FE30000F94802ECF52DF4F288139814A815B8118
:10FE4000C15DD0400F945D2F2B013C016DA77EA7B3
:10FE50008FA798ABC953DF4F288139814A815B81D5
:10FE6000C75CD040C501B4010F947C2A4B015C01F2
:10FE7000CB52DF4F288139814A815B81C55DD040FB
:10FE8000C701B6010F947C2A9B01AC01C501B401E6
:10FE90000F94802ECF52DF4F288139814A815B81B8
:10FEA000C15DD0400F945D2F6B017C0169AB7AABD3
:10FEB0008BAB9CABC954DF4F288139814A815B8170
:10FEC000C75BD040C301B2010F947C2A9B01AC01F7
:10FED000CD53DF4F688179818A819B81C35CD0409B
:10FEE0000F94812E4B015C01C154DF4F2881398171
:10FEF0004A815B81CF5BD040C701B6010F947C2A59
:10FF00009B01AC01C501B4010F94812EDC01CB0132
:10FF1000B0588DAB9EABAFABB8AF2DA53EA54FA5EE
:10FF200058A9C154DF4F288339834A835B83CF5B51
:10FF3000D0405058CD53DF4F288339834A835B83A9
:10FF4000C35CD04089A99AA9ABA9BCA9C953DF4F0A
:10FF500088839983AA83BB83C75CD0400DA91EA95F
:10FF60002FA938ADCB50DF4F088319832A833B83F9
:10FF7000C55FD040C052DF4F08811981C05ED040BC
:10FF8000B801110F880B990B0F941D2A9B01AC012E
:10FF9000C452DF4F688179818A819B81CC5DD040DA
:10FFA0000F945D2FCB52DF4F688379838A839B83C5
:10FFB000C55DD040C652DF4F08811981CA5DD0406F
:10FFC000012B09F46DC240903C1550903D15609096
:10FFD0003E1570903F15209148153091491540917C
:10FFE0004A1550914B15C301B2010F94802ECC518C
:10FFF000DF4F688379838A839B83C45ED040C0903F
:020000021000EC
:100000003815D0903915E0903A15F0903B152091B5
:100010004415309145154091461550914715C7013B
:10002000B6010F94802EC751DF4F688379838A838E
:100030009B83C95ED0408090341590903515A09078
:100040003615B090371520914015309141154091EB
:10005000421550914315C501B4010F94802EC35130
:10006000DF4F688379838A839B83CD5ED040209164
:100070003015309131154091321550913315C452DD
:10008000DF4F288339834A835B83CC5DD040A30153
:100090009201C452DF4F688179818A819B81CC5D56
:1000A000D0400F94802ECF50DF4F688379838A83AE
:1000B0009B83C15FD04080912C1590912D15A0910C
:1000C0002E15B0912F15C353DF4F88839983AA83D0
:1000D000BB83CD5CD040A7019601BC01CD010F943C
:1000E000802E6B017C01009128151091291520911B
:1000F0002A1530912B15CF52DF4F088319832A839D
:100100003B83C15DD040A5019401CF52DF4F688190
:1001100079818A819B81C15DD0400F94802E4B01F3
:100120005C01C751DF4F288139814A815B81C95EFB
:10013000D0400F947C2A2B013C01C351DF4F288112
:1001400039814A815B81CD5ED040C701B6010F94F1
:100150007C2A9B01AC01C301B2010F94802EC954CB
:10016000DF4F688379838A839B83C75BD040C35109
:10017000DF4F288139814A815B81CD5ED040CF50ED
:10018000DF4F688179818A819B81C15FD0400F9464
:100190007C2A2B013C01CC51DF4F288139814A81D7
:1001A0005B81C45ED040C501B4010F947C2A9B01E1
:1001B000AC01C301B2010F94802E2B013C01CC5144
:1001C000DF4F288139814A815B81C45ED040C701FD
:1001D000B6010F947C2A6B017C01C751DF4F288147
:1001E00039814A815B81C95ED040CF50DF4F688141
:1001F00079818A819B81C15FD0400F947C2A9B01C9
:10020000AC01C701B6010F94802E6B017C012091D7
:100210004C1530914D1540914E1550914F150F943E
:100220007C2A4B015C012091501530915115409171
:10023000521550915315C301B2010F947C2A9B01B2
:10024000AC01C501B4010F94812E4B015C012091DA
:100250005415309155154091561550915715C95464
:10026000DF4F688179818A819B81C75BD0400F9481
:100270007C2A9B01AC01C501B4010F94812E4B0176
:100280005C01CF52DF4F688179818A819B81C15D9A
:10029000D0409058A70196010F947C2ACF52DF4F8F
:1002A000688379838A839B83C15DD040A3019201D7
:1002B000C353DF4F688179818A819B81CD5CD040B7
:1002C0000F947C2A9B01AC01CF52DF4F688179816A
:1002D0008A819B81C15DD0400F94802EC353DF4F34
:1002E000688379838A839B83CD5CD040C954DF4F78
:1002F000288139814A815B81C75BD040C452DF4F7E
:10030000688179818A819B81CC5DD0400F947C2A61
:100310009B01AC01C353DF4F688179818A819B8146
:10032000CD5CD0400F94802E9B01AC01C501B4017F
:100330000F94812E4B015C0120E030E0A9010F9465
:10034000A730181624F0B7FAB094B7F8B094A70104
:100350009601C701B6010F947C2A6B017C01A301B1
:100360009201C301B2010F947C2A9B01AC01C70129
:10037000B6010F94812E6B017C01C954DF4F288197
:1003800039814A815B81C75BD040CA01B9010F94B2
:100390007C2A9B01AC01C701B6010F94812E0F94FA
:1003A000EC309B01AC01C501B4010F945D2FAB0192
:1003B000BC0186E090E10E94A3A58AE00E94496109
:1003C0008AE00E944961E0EFFFE084918F010F5FB6
:1003D0001F4F882321F00E944961F801F6CF48E0C1
:1003E000CD53DF4F688179818A819B81C35CD04086
:1003F0000E942262EBEEFFE084918F010F5F1F4F9E
:10040000882321F00E944961F801F6CF48E0C953E2
:10041000DF4F688179818A819B81C75CD040905889
:100420000E942262E6EEFFE084918F010F5F1F4F72
:10043000882321F00E944961F801F6CFCB50DF4FAD
:10044000688179818A819B81C55FD040905848E05E
:100450000E9422628AE00E944961C652DF4F0881F1
:100460001981CA5DD04003301105D4F0EDECFFE0F6
:1004700084918F010F5F1F4F882321F00E944961F3
:10048000F801F6CF48E0CB52DF4F688179818A814D
:100490009B81C55DD0400E9422628AE00E94496132
:1004A000C851DF4F1881C85ED0401111E9C1C15455
:1004B000DF4F288139814A815B81CF5BD040CB56A9
:1004C000DF4F288339834A835B83C559D040C953A2
:1004D000DF4F88819981AA81BB81C75CD040C75614
:1004E000DF4F88839983AA83BB83C959D040C12C2D
:1004F000D12C60E8E62E6FE3F62EC356DF4FC8829C
:10050000D982EA82FB82CD59D040CE018B569F4FD3
:100510000E947099C757DF4FC882D982EA82FB8256
:10052000C958D040C357DF4F188219821A821B82E4
:10053000CD58D040CD53DF4F088119812A813B81AE
:10054000C35CD040CF56DF4F088319832A833B8397
:10055000C159D040CE0187579F4F0E947099CB560A
:10056000DF4F288139814A815B81C559D040CD5305
:10057000DF4F288339834A835B83C35CD040C756EF
:10058000DF4F488059806A807B80C959D040C3566C
:10059000DF4F88809980AA80BB80CD59D040C75753
:1005A000DF4F88819981AA81BB81C958D040C1544D
:1005B000DF4F88839983AA83BB83CF5BD040C35727
:1005C000DF4F088119812A813B81CD58D040C95421
:1005D000DF4F088319832A833B83C75BD040CF5604
:1005E000DF4FC880D980EA80FB80C159D040A70185
:1005F0009601C301B2010F947C2AC953DF4F68836F
:1006000079838A839B83C75CD040C954DF4F28819C
:1006100039814A815B81C75BD040C501B4010F9429
:100620007C2A9B01AC01C953DF4F688179818A81A3
:100630009B81C75CD0400F94802EC358DF4F6883E6
:1006400079838A839B83CD57D040C154DF4F288163
:1006500039814A815B81CF5BD040C501B4010F94E1
:100660007C2A4B015C01A7019601CD53DF4F6881C5
:1006700079818A819B81C35CD0400F947C2A9B0145
:10068000AC01C501B4010F94802ECF57DF4F6883B2
:1006900079838A839B83C158D040C954DF4F288116
:1006A00039814A815B81C75BD040CD53DF4F688180
:1006B00079818A819B81C35CD0400F947C2A6B0135
:1006C0007C01C154DF4F288139814A815B81CF5B36
:1006D000D040C301B2010F947C2A9B01AC01C70139
:1006E000B6010F94802ECB57DF4F688379838A83BE
:1006F0009B83C558D040CE0183589F4F0E9470996C
:10070000C757DF4F088119812A813B81C958D040E2
:10071000C357DF4F488059806A807B80CD58D040D6
:10072000CF56DF4F88809980AA80BB80C159D040C6
:10073000C358DF4F88819981AA81BB81CD57D040B2
:10074000C954DF4F88839983AA83BB83C75BD0409A
:10075000CF57DF4F88819981AA81BB81C158D04092
:10076000C154DF4F88839983AA83BB83CF5BD0407A
:10077000CB57DF4F88819981AA81BB81C558D04072
:10078000CD53DF4F88839983AA83BB83C35CD0405A
:10079000CB56DF4FC880D980EA80FB80C559D04056
:1007A000C756DF4F488159816A817B81C959D04042
:1007B000C356DF4F88819981AA81BB81CD59D04032
:1007C0000093B4121093B5122093B6123093B7125F
:1007D0004092B8125092B9126092BA127092BB1243
:1007E0008092BC129092BD12A092BE12B092BF1223
:1007F000C954DF4F088119812A813B81C75BD040F2
:100800000093C0121093C1122093C2123093C312EE
:10081000C154DF4F088119812A813B81CF5BD040D1
:100820000093C4121093C5122093C6123093C712BE
:10083000CD53DF4F088119812A813B81C35CD040B1
:100840000093C8121093C9122093CA123093CB128E
:10085000C092CC12D092CD12E092CE12F092CF1272
:100860004093D0125093D1126093D2127093D3124E
:100870008093D4129093D512A093D612B093D7122E
:10088000CE51DF4F1881C25ED040112309F465C2FA
:10089000EAE0FFE084918F010F5F1F4F882321F072
:1008A0000E944961F801F6CFC553DF4FC880CB5C89
:1008B000D040CA94DC2CC553DF4F1882CB5CD040AB
:1008C00000ECC154DF4F0883CF5BD04019E7CD5314
:1008D000DF4F1883C35CD04004E4C953DF4F088363
:1008E000C75CD0408E010B561F4FCF54DF4F19838A
:1008F0000883C15BD0400C501109CD54DF4F1983E0
:100900000883C35BD0400C501109CB54DF4F1983CF
:100910000883C55BD040D7FC27C10D2D000F110BFC
:10092000CE51DF4F19830883C25ED040212C312C79
:10093000C954DF4F1882C75BD040CE51DF4FE881EA
:10094000F981C25ED040E20DF31D21EA30E02C0FA8
:100950003D1FE20FF31F008111817801EE0CFF1C97
:10096000EE0CFF1CEDE6F0E0EC0FFD1FEE0DFF1DA1
:100970004080518062807380CB52DF4F2881398163
:100980004A815B81C55DD040C301B2010F94802EC6
:100990004B015C01E1E0F0E0EC0FFD1FEE0DFF1DEF
:1009A00084AD95ADA6ADB7ADCB56DF4F88839983A7
:1009B000AA83BB83C559D040C052DF4FE881F9817B
:1009C000C05ED040E00FF11FEE0FFF1FEE0FFF1FC4
:1009D00041E050E04C0F5D1FE40FF51F84AD95AD75
:1009E000A6ADB7ADC757DF4F88839983AA83BB8372
:1009F000C958D040C358DF4F188219821A821B820F
:100A0000CD57D040CA54DF4F5881C65BD0405F936A
:100A1000CB54DF4F8881C55BD0408F93CC54DF4FE0
:100A20009881C45BD0409F93CD54DF4FA881C35BB6
:100A3000D040AF93CE54DF4FB881C25BD040BF935C
:100A4000CF54DF4FE881C15BD040EF930DB71EB7A5
:100A5000045211090FB6F8941EBF0FBE0DBFADB7FB
:100A6000BEB71196E4EBF2E184E201900D928A9513
:100A7000E1F70E948B98C358DF4F288139814A8162
:100A80005B81CD57D040C301B2010F94802E7B0112
:100A90008C010FB6F894DEBF0FBECDBF9B01AC0139
:100AA000C553DF4F6881CB5CD040C154DF4F7881A4
:100AB000CF5BD040CD53DF4F8881C35CD040C9535A
:100AC000DF4F9881C75CD0400F94A7301816A4F46C
:100AD000C553DF4FE882CB5CD040C154DF4FF88272
:100AE000CF5BD040CD53DF4F0883C35CD040C953A8
:100AF000DF4F1883C75CD04020E030E0A901C5017A
:100B0000B4010F94A73087FD0CC0E7E0FFE08491AB
:100B10008F010F5F1F4F882339F00E944961F80150
:100B2000F6CF80E20E94496145E0C501B4010E9410
:100B30002262C954DF4F0881C75BD0400F5FC954A0
:100B4000DF4F0883C75BD04014E0210E311CC75231
:100B5000DF4F1881C95DD040011708F4EECE8AE05E
:100B60000E944961DA94D7CE8AE00E944961C65258
:100B7000DF4F08811981CA5DD0400430110509F0AA
:100B8000ECC0EEEDFEE084918F010F5F1F4F8111ED
:100B90000CC01E0115E9210E311C2E0129E8420E60
:100BA000511C8E0103581F4F1BC00E944961F80160
:100BB000EACF80E20E94496145E0C501B4010E948C
:100BC0002262D394F4E0EF0EF11CC752DF4F28816C
:100BD000C95DD040D21660F08AE00E944961CA9493
:100BE000C7FCB7C06C2C660C7708E12CF12CD12C1B
:100BF000F701E60DF71D41EA50E04C0F5D1FE40FD1
:100C0000F51F808191815C01AA0CBB1CAA0CBB1C46
:100C1000E1E0F0E0EC0FFD1FEA0DFB1D44AD55AD2A
:100C200066AD77ADD1014D935D936D937C93139732
:100C3000C052DF4FE881F981C05ED040E80FF91F54
:100C4000EE0FFF1FEE0FFF1F21E030E02C0F3D1FC6
:100C5000E20FF31F84AD95ADA6ADB7ADF201808371
:100C60009183A283B383D8011D921D921D921C9281
:100C700013971F930F935F924F923F922F92EDB76E
:100C8000FEB7B4970FB6F894FEBF0FBEEDBFADB779
:100C9000BEB71196E4EBF2E184E201900D928A95E1
:100CA000E1F70E948B98EDE6F0E0EC0FFD1FEA0DF6
:100CB000FB1DD8012D913D914D915C916081718119
:100CC000828193810F94802EC553DF4F2881CB5CA6
:100CD000D040C154DF4F3881CF5BD040CD53DF4F80
:100CE0004881C35CD040C953DF4F5881C75CD040B6
:100CF0000F94802E4B015C010FB6F894DEBF0FBE3F
:100D0000CDBF20E030E0A9010F94A73087FD51CF7F
:100D1000EBEDFEE084919F012F5F3F4F882309F4A4
:100D20004BCFCE5EDE4F2883C251D140CF5EDE4F27
:100D30003883C151D1400E944961CE5EDE4F288187
:100D4000C251D140CF5EDE4F3881C151D140F9014F
:100D5000E1CF8AE00E94496108C0C652DF4F088196
:100D60001981CA5DD040012B21F08CEB9EE00F94DD
:100D70001625C851DF4F1881C85ED040111185C0BB
:100D80008CE0E7EFFEE0DE01A358BF4F01900D922B
:100D90008A95E1F781E08093880ECE0183589F4FBA
:100DA0000E9445DDC355DF4F288139814A815B812F
:100DB000CD5AD0406091F70E7091F80E8091F90EE7
:100DC0009091FA0E0F94802E6B017C012DEB37E38E
:100DD00046E855EB0F94A73087FD4BC02DEB37E36A
:100DE00046E855E3C701B6010F94172A18160CF40C
:100DF00040C0C755DF4F288139814A815B81C95A7C
:100E0000D0406091FB0E7091FC0E8091FD0E909190
:100E1000FE0E0F94802E6B017C012DEB37E346E82C
:100E200055EB0F94A73087FD24C02DEB37E346E840
:100E300055E3C701B6010F94172A1816D4F0C5540C
:100E4000DF4F288139814A815B81CB5BD040609143
:100E5000FF0E7091000F8091010F9091020F0F947F
:100E6000802ECB57DF4F688379838A839B83C55855
:100E7000D0408CE0FE01E358FF4FA7EFBEE00190A9
:100E80000D928A95E1F781E005C0C453DF4F888158
:100E9000CC5CD0408093880E0E94D9B10E946A68D1
:100EA0008091880E81110E94D8B6CE5EDE4F0FB6BB
:100EB000F894DEBF0FBECDBFDF91CF911F910F9190
:100EC000FF90EF90DF90CF90BF90AF909F908F906A
:100ED0007F906F905F904F903F902F900895DF929A
:100EE000EF92FF920F931F93CF93DF93CDB7DEB7AF
:100EF0002C970FB6F894DEBF0FBECDBF182F0E94FF
:100F0000A9DFD090880E80E00E94C0B70E94F3B1A4
:100F100081E080934C18111119C088E50E947BB8BC
:100F2000F82E89E50E947BB8082F8AE50E947BB8DD
:100F3000E82EF11006C0011113C0882369F0F02ECD
:100F400010C0002369F0F02E182F0BC0FF24F3947B
:100F500001E0EE24E39402C0F82E082F11E001C056
:100F600010E00E94C5B9111105C0E11003C0F110D5
:100F700006C02BC082E00E94A1C11123C1F380E012
:100F800090E0A0E8B0E48093470890934808A093CD
:100F90004908B0934A089C01AD016091FF0E709121
:100FA000000F8091010F9091020F0F94172A87FF75
:100FB0000FC019821A821B821C82BE016F5F7F4F95
:100FC00087E498E00E9442B303C00111D8CF0CC05F
:100FD000111102C0FF20A9F080E00E94A1C11123DD
:100FE00081F081E00E94A1C10E94D8B61D821E82BC
:100FF0001F821886112369F080E090E0A5E3B3E436
:1010000012C00111EECF0E94D8B61D821E821F822F
:101010001886E110F1CF8091FF0E9091000FA09102
:10102000010FB091020F89839A83AB83BC83BE0109
:101030006B5F7F4FCE0101960E9442B380E090E04B
:10104000A0EAB0E489879A87AB87BC8711110BC0EF
:10105000011109C04091FB0E5091FC0E6091FD0EF4
:101060007091FE0E04C040E050E06BE373E44D83EA
:101070005E836F83788711110BC0F11009C0409116
:10108000F70E5091F80E6091F90E7091FA0E04C0AF
:1010900040E050E060EA70E449835A836B837C83CC
:1010A000AE01475F5F4FBE016B5F7F4FCE01019680
:1010B0000E943EB380914B1880934C188D2D0E9456
:1010C000C0B70E94D9B183E080935B020E946A6836
:1010D0002C960FB6F894DEBF0FBECDBFDF91CF9137
:1010E0001F910F91FF90EF90DF9008951092A0074D
:1010F0008091A607882331F00F94211483E39BE8A5
:101100000D94710420910102309102024091651109
:10111000509166116091671170916811C901840F37
:10112000951F2436310524F4853691053CF416C00C
:101130002436310531F08436910584F484E690E05C
:101140000DC0473051056105710514F0069706C0C2
:101150004A3F5F4F6F4F7F4F6CF4069690930202A9
:10116000809301021092651110926611109267111E
:101170001092681180910102909102028A309105CB
:101180003CF0883E23E092072CF087EE93E002C00B
:101190008AE090E0909302028093010280E00C9438
:1011A0006EA2CF93DF9300D01F92CDB7DEB75C83E2
:1011B0004B837A836983BE016D5F7F4FCE010196B9
:1011C0000E9440F30F900F900F900F90DF91CF91FE
:1011D0000895282F8091651190916611A091671153
:1011E000B091681181309048A105B10540F010928E
:1011F000651110926611109267111092681180911A
:101200009507882331F080916511809381071092B2
:101210006211809189071816FCF4082E000C990BB6
:10122000821B910920918107022E000C330B281795
:10123000390794F097FF02C080E090E08093810727
:10124000092E000CAA0BBB0B8093651190936611BD
:10125000A0936711B0936811809181076623A9F06C
:1012600090918A07891714F480938A0720918A073E
:10127000022E000C330B2C5F3F4F482F082E000C22
:10128000550B241735071CF4845080938A07089562
:10129000809163118630D8F496E0899FF001112483
:1012A000EB5AF84F2091450230914602318320835A
:1012B00040916511509166116091671170916811AC
:1012C00042835383648375838F5F80936311089592
:1012D00086E798E80D947104E0916311EE2369F0BC
:1012E000E150E093631186E0E89FF0011124EB5A8E
:1012F000F84F808191810D947104EACF10926411AE
:10130000EBCF0F931F93CF93DF9361E081E061DF19
:10131000D0918A07C0E002E612E1D1111DC0809190
:10132000A607811106C080915B02882309F4B6C02C
:101330000AC0809181078111F6CFE0DF80916211B0
:10134000882389F3B2C081E090918107911180E0F8
:1013500024E04CEA52E19FC0D13009F58091A60704
:10136000811106C080915B02882309F497C00DC0EB
:10137000809181078130B1F78AEA9FE90E94ECAF42
:1013800080916211882371F390C081E09091810770
:10139000913009F080E023E04AE952E17CC0D2308C
:1013A00051F58091A607811106C080915B028823C8
:1013B00009F474C016C0809181078230B1F7C1D59D
:1013C000882319F00E94D9B907C048EB51E064E1C5
:1013D00070E080E090E0E5DE80916211882329F3DF
:1013E00064C081E090918107923009F080E020E2B2
:1013F0004BE852E150C0D33059F58091A6078111D6
:1014000006C080915B02882309F448C017C0809110
:1014100081078330B1F70F94BA0C882319F00E942A
:10142000D9B907C048EB51E064E170E080E090E09A
:10143000B8DE80916211882321F337C081E090915A
:101440008107933009F080E020E24CE652E123C0AE
:10145000D43021F58091A607811105C080915B02EF
:101460008823E1F00FC0809181078430B9F7109391
:101470005411009353110E94F7B380916211882395
:1014800069F313C081E090918107943009F080E006
:1014900020E24AE752E16C2F0E94E9B9CF5FDF5F9B
:1014A000C53009F03ACFC0938907DF91CF911F91E2
:1014B0000F910895CF92DF92EF92FF920F931F93B7
:1014C000CF93DF9361E081E084DED0918A07C0E0B2
:1014D00000EA11E181EBE82E81E1F82E99E5C92EB1
:1014E00092E1D92ED1111DC08091A607811106C0AD
:1014F00080915B02882309F4A6C00AC0809181070D
:101500008111F6CFFBDE80916211882389F3A2C09E
:1015100081E090918107911180E024E04DE552E156
:101520008FC0D13019F58091A607811106C0809136
:101530005B02882309F487C00FC080918107813046
:10154000B1F7D0925411C09253110E94F7B3809119
:101550006211882361F37EC081E090918107913010
:1015600009F080E020E24FE452E16AC0D23019F580
:101570008091A607811106C080915B02882309F43F
:1015800062C00FC0809181078230B1F7F092541190
:10159000E09253110E94F7B380916211882361F3A6
:1015A00059C081E090918107923009F080E020E2FB
:1015B00044EA51E145C0D33011F58091A60781116D
:1015C00005C080915B028823F1F10FC080918107F3
:1015D0008330B9F710935411009353110E94F7B35D
:1015E00080916211882369F335C081E09091810771
:1015F000933009F080E020E24FE851E121C0D4307F
:1016000011F58091A607811105C080915B028823A6
:10161000D1F00DC0809181078430B9F785E39CEF4C
:101620000E94ECAF80916211882379F313C081E0AE
:1016300090918107943009F080E023E045E851E182
:101640006C2F0E94E9B9CF5FDF5FC53009F04ACF48
:10165000C0938907DF91CF911F910F91FF90EF9079
:10166000DF90CF9008958F929F92AF92BF92CF92CA
:10167000DF92EF92FF920F931F93CF93DF9361E07E
:1016800081E0A7DDC0918A0700E09924939488EC5B
:10169000E82E80E1F82E93EEC92E90E1D92E2DEDA3
:1016A000A22E20E1B22EC1111EC08091A607811189
:1016B00005C080915B028823B1F00AC08091810748
:1016C0008111F7CF1BDE80916211882391F32DC227
:1016D00081E090918107911180E024E049E751E198
:1016E000602F0E94E9B980910C1390910D13891B12
:1016F0008F7009F0E6C180915A158111E2C1809185
:101700005B15882321F080914F178111DAC1C13018
:1017100009F58091A607811106C080915B0288239C
:1017200009F45EC00DC0809181078130B1F78AE570
:101730009AE80E94ECAF80916211882371F3F5C1A1
:1017400081E090918107913009F080E023E04BE641
:1017500051E143C0C23001F58091A607811105C057
:1017600080915B028823E1F10DC080918107823076
:10177000B9F787EC9AEC0E94ECAF80916211882354
:1017800079F3D3C181E090918107923009F080E034
:1017900023E04FE551E121C0C33011F58091A60748
:1017A000811105C080915B028823D1F00DC080912A
:1017B00081078330B9F781E899E80E94ECAF809106
:1017C0006211882379F3B1C181E090918107933050
:1017D00009F080E023E041E551E1602F0E94E9B982
:1017E00010E0D4E08090DC08811018C060912902DC
:1017F00070912A02072E000C880B990B0F941D2A5A
:101800009B01AC016091D8087091D9088091DA08E9
:101810009091DB080F94172A87FD37C0CD1334C091
:101820008091A607811105C080915B02882361F138
:1018300020C0809181078C13F7CF8091E50883FD4C
:1018400067C1811065C12091530730915407809181
:10185000290290912A02281739070CF059C118DD86
:101860008FE29DE90F947104809162118823E1F267
:101870005CC181E0909181079C1380E020E241E40B
:1018800051E1602F0E94E9B9DF5F80915B158823E9
:1018900009F4C5C080914F17882309F49CC080913A
:1018A0005A15882379F1CD1357C08091A60781116D
:1018B00006C080915B02882309F44EC01AC0809153
:1018C00081078C13F6CF10925A1580E095E10E94A3
:1018D000BB4CB0925411A09253110E94F7B36FEF1A
:1018E00080ED90E10E94A2AB80916211882309F300
:1018F0001CC181E0909181079C1380E020E245E3C8
:1019000051E127C0CD1328C08091A607811105C0E1
:1019100080915B02882301F114C0809181078C13B0
:10192000F7CFD0925411C09253110E94F7B36FEFCA
:1019300082EE90E10E94A2AB80916211882341F374
:10194000F4C081E0909181079C1380E020E249E19E
:1019500051E1602F0E94E9B9DF5FCD1337C080915C
:10196000A607811105C080915B02882379F123C00D
:10197000809181078C13F7CF0F946308809114082E
:1019800080938206109283060E94854E0F94D51C88
:101990000E94B0761092D7081092D60810921A02C0
:1019A0006FEF87EE90E10E94A2AB92DC8091621112
:1019B0008823C9F2BAC081E0909181079C1380E02E
:1019C00020E24EE051E1602F0E94E9B9DF5F112370
:1019D00009F44BC06EC011116CC0CD1345C080918D
:1019E000A607811106C080915B02882309F43CC0E0
:1019F0000DC0809181078C13F6CF8CED9DE90E947C
:101A0000ECAF80916211882371F38FC081E09091D7
:101A100081079C1380E023E040E051E122C01111D6
:101A200048C0CD1321C08091A607811105C08091C7
:101A30005B028823C9F00DC0809181078C13F7CF1A
:101A40008CED9DE90E94ECAF80916211882379F3BF
:101A50006CC081E0909181079C1380E023E045EF0A
:101A600050E1602F0E94E9B9DF5FCD1321C0809162
:101A7000A607811105C080915B028823C9F00DC0C3
:101A8000809181078C13F7CF82EF90E00E94ECAF3A
:101A900080916211882379F348C081E09091810799
:101AA0009C1380E023E046E251E1602F0E94E9B9F7
:101AB000DF5F0F5FCF5F053009F0F5CDD093890769
:101AC00034C0C13011F58091A607811105C0809105
:101AD0005B028823D1F00DC0809181078130B9F776
:101AE00086ED90E00E94ECAF80916211882379F33B
:101AF0001CC081E090918107913009F080E023E0E3
:101B000044E751E1602F0E94E9B911E0D2E06ACECA
:101B1000909264118EE49CE90F947104F092541138
:101B2000E09253110E94F7B39FCEDF91CF911F91A6
:101B30000F91FF90EF90DF90CF90BF90AF909F906C
:101B40008F900895AF92BF92CF92DF92EF92FF9263
:101B50000F931F93CF93DF935C017B0120E030E074
:101B6000F501E20FF31FE491EE2319F02F5F3F4FD1
:101B7000F7CFF701CF018E199F0941914111FACF9B
:101B800004E110E0081B11093327021713071CF0AA
:101B9000DD24D39402C082E0D82E8091121890E008
:101BA0006D2D70E06F5F7F4F0F946931C62EC6E0D8
:101BB000C60F80914518C81750F08091471890E0E3
:101BC0002C2F30E02B503109821793079CF5D0E081
:101BD000E114F104C1F18AE30F94771C82E0D8127A
:101BE0000FC0CC0D80914518C81768F12091471897
:101BF00030E08C2F90E00B97281739071CF423C096
:101C0000DD2309F1802F880F080F000F009348187B
